:020000021000EC
:10F00000F0FF002039F5010061F5010063F5010012
:10F0100065F5010067F5010069F5010000000000D9
:10F020000000000000000000000000006BF501007F
:10F030006DF50100000000006FF50100351A0400B5
:10F040007954020073F501006D560200D954020094
:10F05000255502004D6702001D58020073F501009E
:10F0600073F50100791A040073F5010073F50100CE
:10F0700073F501008961020073F5010073F5010069
:10F08000751A0400452D020073F5010073F50100A7
:10F090004D2E0200D1DB0300C91E020073F50100F2
:10F0A00073F5010073F5010073F50100AD6902000D
:10F0B00073F5010073F5010000000000000000007E
:10F0C00073F5010073F5010073F5010073F501009C
:10F0D00073F501005563020073F5010000000000A4
:10F0E0000000000000000000000000000000000020
:10F0F0000000000000000000000000000000000010
:10F1000000000000000000000000000000000000FF
:10F1100000000000000000000000000000000000EF
:10F4000010B5054C237833B9044B13B10448AFF35E
:10F4100000800123237010BD202E0020000000007A
:10F42000E850060008B5034B1BB103490348AFF38E
:10F43000008008BD00000000242E0020E8500600D7
:10F44000154B002B08BF134B9D46A3F5803A0021B6
:10F450008B460F461348144A121A00F063F80F4BFC
:10F46000002B00D098470E4B002B00D0984700206F
:10F47000002104000D000D48002802D00C48AFF315
:10F48000008000F02BF82000290026F015FB00F08A
:10F4900011F800BF00000800F0FF0020000000008D
:10F4A00000000000202E0020ACE200200000000040
:10F4B0000000000008B5074B044613B10021AFF36C
:10F4C0000080054B1868836A03B19847204600F016
:10F4D00031F800BF000000004CBE050070B50D4DB6
:10F4E0000D4C641BA4100026A64209D10B4D0C4CF8
:10F4F0003CF0A0FC641BA4100026A64205D170BD00
:10F5000055F8043B98470136EEE755F8043B984719
:10F510000136F2E7082E0020082E0020082E0020D9
:10F520000C2E002002440346934200D1704703F89A
:10F53000011BF9E7FEE700BF0649074A074B9B1A84
:10F5400003DD043BC858D050FBDC07F003F8FFF79D
:10F5500077FF0000F4500600402C0020202E0020F1
:10F56000FEE7FEE7FEE7FEE7FEE7FEE7FEE7FEE773
:10F57000FEE7FEE71FB501238DF80030054B8DF83F
:10F58000080001916846D3E90012904705B05DF884
:10F5900004FB00BF60CB002061DF704748DF70478D
:10F5A00010B50388012B11D8094A02EB03124388D6
:10F5B0005189CC1A032C09D4C3F57F43FD330B4486
:10F5C0005381002303804380184610BD0420FCE7CC
:10F5D00060D0002010B5124A0B6802EB00104268A0
:10F5E00073B15888033003EB800302F580524FF665
:10F5F000FF749A4202D91868013004D1002009E052
:10F6000002F10803F1E79888A04204D0188810B1ED
:10F610000B60012010BD5888033003EB8003E8E73E
:10F6200060D0002073B5436804460D4613B31E4AEC
:10F6300011688B421ED3526893421BD813F003000B
:10F6400018D11A4A21891289914213D121689A68E6
:10F6500091420FD1164A5268934201D80A2004E021
:10F6600002F580529342F9D22880B0FA80F0400926
:10F6700002B070BD00232B801E46019601A9288888
:10F68000FFF7A8FF30B92B8801339BB22B80002BEA
:10F69000F3D0EDE7019B226899689142EED1636057
:10F6A000024B1B892381E3E7102E002024CD00208C
:10F6B00060D00020033083B240F2FD32934230B577
:10F6C0000ED909200BE0228965892A441A4492B296
:10F6D000B2F5806F08D2088062891344638130BD1F
:10F6E000024C20780028EED00720F8E760D00020F8
:10F6F00010B50A494A788C78531CDBB29C4208BF8B
:10F7000000230C789C421FBF0370486802EB420242
:10F7100000EBC20008BF002010BD00BFDCCF0020FE
:10F72000AADF7047A9DF7047A7DF704785DF704702
:10F730007FDF70477EDF7047084A30B500230C2416
:10F7400004FB03F18D5A854202D10A44508830BD32
:10F750000133082BF4D14FF6FF70F8E78ECC002070
:10F760006EDF7047012804D0043804288CBF0020C5
:10F77000012070478378013B072B07D8DFE803F0AF
:10F7800007060606060704091423038070470123B1
:10F79000FBE743689B8809339B08F6E770B5054D86
:10F7A0000646002455F8043B304601349847052CA2
:10F7B000F8D170BD18C00500114BF0B50022142619
:10F7C0001D4606FB02F4E75A874212D12344142651
:10F7D00000249A788A420AD001342246072A0BD89C
:10F7E00006FB02F3EF5A874208D1EB18F1D1184615
:10F7F000F0BD0132082AE4D10023F8E70132EDE739
:10F80000FCD10020F8B5074D074E07460024337899
:10F81000A34200DCF8BD55F8043B38469847013454
:10F82000F5E700BF00CD0020B1CE00207DDF70479E
:10F8300079DF70476DDF704758B1CB0801F00701E1
:10F84000C25C012303FA01F10A4214BF18460020EA
:10F85000704701207047000070B50A4E34680546B5
:10F8600054B1706860B1FF2D08D02946FFF7E4FF5E
:10F8700030B1F36803FB0544204670BD0024FBE76C
:10F880000446F9E7ECD1002030B5072185B0FFF739
:10F8900093FF044600283AD04568002D39D1007CFA
:10F8A000FFF7DAFF0721CDE902558DF80A1040B3C2
:10F8B000E368039003EB83031B019BB29B0802A840
:10F8C000ADF80830FFF756FF9DF80A00FFF74AFF32
:10F8D000D8B1114B1B789B0715D5BDF808500DF119
:10F8E00006012846FFF7E6FE48B9BDF80630A380BA
:10F8F000E5800A4B185C092803D005B030BD092803
:10F90000F7D90320F9E70220F3E70846F5E70520D9
:10F91000F3E70020F1E700BF21CD002068BE05001D
:10F9200038B54FF6FF73984218BF01300D4614BF2B
:10F9300084B20024FF2C03D94FF6FF74204638BD53
:10F9400021462846FFF778FF0028F7D10134A4B2FA
:10F95000F0E7000038B5074C051E04F1080318BF96
:10F960001C4623682BB11A6822605B6828469847BA
:10F97000F7E738BD38CC002040DF70473FDF7047E5
:10F980000023435082B043580193019B02B070475B
:10F990002DE9F0470D789DF820609DF824A00446DD
:10F9A0000F469946002D60D1D0F8243192F800809E
:10F9B0009BB14FF49271FFF7E3FF012363613B704A
:10F9C000B04550D1D4F80431002B4CD04FF48271A3
:10F9D0002046FFF7D5FF00251DE0D0F81C31FBB114
:10F9E0004FF48E71FFF7CCFFD0F824311BB14FF4E8
:10F9F00092712046DFE713789E4207D919F8033049
:10FA0000C0F81C35137801331370D9E70123BAF11C
:10FA1000000F03D0C3612846BDE8F0874361CFE7FC
:10FA2000D0F80831002BCBD04FF48471FFF7A8FF3A
:10FA3000D0F82431002BDAD113789E42C0D9D0F807
:10FA4000181509F8031013780133DBB21370721E16
:10FA5000934205D10223C0F8003201232362AFE7AD
:10FA60009E42FAD1ACE70125D5E74FF49271FFF73A
:10FA700087FF4FF48E71FFF783FF4FF48471FFF718
:10FA80007FFF9FE72DE9F3470C4605464FF482714F
:10FA900020461F469046FFF773FF4FF49271FFF721
:10FAA0006FFF4FF48E71FFF76BFF4FF48471FFF718
:10FAB00067FF0023012F85F8263085F8233008BF23
:10FAC00002224FF001030CBFC4F80022C4F8003238
:10FAD000236223602E6846BB05F1260A05F123093F
:10FAE000CDE900764346524649462046FFF750FF8F
:10FAF0000028F5D195F82330EBB1D4F8C434C4F81C
:10FB0000C434C3B113F0010F14BF4FF402400320FB
:10FB100048F2012213F0020F18BF104613F0040F31
:10FB200048F2022318BF184606E040F28623AB6075
:10FB3000AB68C4F80433002002B0BDE8F0872DE9BB
:10FB4000F3470C4605464FF4827120461F46164681
:10FB50009DF82880FFF714FF4FF49271FFF710FF14
:10FB60004FF48E71FFF70CFF4FF48471FFF708FF1D
:10FB70000023C4F8003285F8263085F823300123AD
:10FB80002362A36095F82620974232D9B35CC4F86B
:10FB90001C3595F82630013385F826302B687BBB61
:10FBA00005F1260A05F12309CDE9007833465246CE
:10FBB00049462046FFF7ECFE0028F5D195F82330A2
:10FBC00023B3D4F8C434C4F8C434FBB113F0010F28
:10FBD00014BF4FF40240032048F2012213F0020F39
:10FBE00018BF104613F0040F48F2022318BF18463E
:10FBF0000DE0B8F1000F01D0E361CFE76361CDE71D
:10FC000040F28623AB60AB68C4F80433002002B036
:10FC1000BDE8F0870023435082B043580193019B15
:10FC200002B0704708B502464FF492710068FFF7C2
:10FC3000F1FF4FF484711068FFF7ECFF13680122A5
:10FC40001A6008BD10B5CB7D0A464FF4847123B904
:10FC5000FFF7E0FFD0F8183510BDFFF7DBFF537E4C
:10FC6000D168D0F81805C854537E0133DBB25376FF
:10FC7000F2E70A4610B54FF48E71FFF7CBFF938A77
:10FC800091689BB2C95C938A01339BB29382C0F89E
:10FC90001C1510BD2DE9F04793F9005090B00024D9
:10FCA000013D6E46AD002746A446A0465FF0000E1B
:10FCB00003E05FEA080EBEEB050EB8EB0E0952F842
:10FCC00009A051F80E90A9FB0A9A14EB090457EB0E
:10FCD0000A075CF1000C1EF1040EAE4501DCC645BE
:10FCE000EBDD46F808403C4667465FF0000C18F133
:10FCF0000408A845DADDB8EB450FDADD46F8084020
:10FD0000D3F8B0303146984710B0BDE8F0871346BD
:10FD10000A46FFF7BFBFF0B5154689B01C46074637
:10FD20000E461A4629466846FFF7F1FF23466A4603
:10FD300039463846FFF7AEFF23462A4669466846ED
:10FD4000FFF7A8FF23466A4631463046FFF7A2FF79
:10FD500009B0F0BD00EB81010023884200D3704759
:10FD600051F8042D43EA52030B60D307F5E710B5B1
:10FD7000013A52B2130601D5002010BD50F82240BE
:10FD800051F822309C4205D802F1FF32F2D24FF0F6
:10FD9000FF30F2E70120F0E710B500235CB2A24289
:10FDA00000DC10BD51F8234040F823400133F5E753
:10FDB000013910B549B2041D0A06CBB204D4013989
:10FDC00054F82120002AF7D001335BB273B103F15C
:10FDD0008042013A50F82220002022B9013B00EB7A
:10FDE000431318B210BD52080130F6E71846F9E780
:10FDF000002310B51C465AB2914200DC10BD40F8F9
:10FE000023400133F7E7000000000000000000007D
:10FE1000C3F10803DB0070B50133002403A500BF64
:10FE20005B1920C940CAAD1B20C0184720C940CA71
:10FE3000B54120C020C940CAB54120C020C940CA30
:10FE4000B54120C020C940CAB54120C020C940CA20
:10FE5000B54120C020C940CAB54120C020C940CA10
:10FE6000B54120C06441B4FA84F0400970BD00BFC0
:10FE7000C3F10803DB0070B50133002403A500BF04
:10FE80005B1920C940CAAD1920C0184720C940CA13
:10FE9000754120C020C940CA754120C020C940CA50
:10FEA000754120C020C940CA754120C020C940CA40
:10FEB000754120C020C940CA754120C020C940CA30
:10FEC000754120C06441204670BD00BFF0B50822D6
:10FED00089B00C460646FFF75FFFCB6A03930B6BB6
:10FEE00004934B6B05938B6B0693CB6B07930027A7
:10FEF00008236A4669466846CDE901770097FFF70F
:10FF0000B7FF082305466A4631463046FFF7B0FF83
:10FF1000236B0393636B0493A36B0593E36B05441B
:10FF2000CDE906376A46082369466846FFF7A0FF11
:10FF3000082305446A4631463046FFF799FF236A95
:10FF40000093636A0193A36A0293A36B0693E36B26
:10FF50000793054408236A4631463046CDE90477C5
:10FF60000397FFF785FF636A0093A36AA26B01936F
:10FF7000E36A02930492636BE26B0393CDE905237A
:10FF8000236A0793054408236A4631463046FFF743
:10FF90006FFFE36A0093236B0193636B0293236A01
:10FFA0000693A36A0793054408236A463146304600
:10FFB000CDE904770397FFF72BFF236B0093636B67
:10FFC0000193A36B0293E36B0393636A0693E36A63
:10FFD00007932D1A08236A4631463046CDE9047747
:10FFE000FFF716FF636B0093A36B0193E36B029320
:10FFF000236A0393636A0493A36ACDE90537236BED
:020000022000DC
:1000000007932D1A08236A4631463046FFF700FF52
:10001000A36B0093E36BCDE90137636A0393A36A93
:100020000493E36ACDE90537636B07932D1A082320
:100030006A4631463046FFF7EBFE2D1A0D4C0FD4C1
:1000400035B9082231462046FFF791FE01280FD02E
:100050000823224631463046FFF7DAFE2D1AEFE735
:100060000823224631463046FFF702FF2D18F7D409
:1000700009B0F0BD8CBE05002DE9F04391B00F46EC
:100080001C220021804609A8FFF74CFA01251C22FA
:10009000002101A80895FFF745FA394608AA11F989
:1000A000046B009533461046FFF7E2FE314608A880
:1000B000FFF77EFE013804B2012C07DC32466946A8
:1000C0004046FFF769FE11B0BDE8F0833A46684646
:1000D0006946FFF71CFE10AB601103EB80001FFAAE
:1000E00084F909F01F0350F8202C05FA03F313429A
:1000F00005D03B46424669466846FFF7CBFD09F10D
:10010000FF3424B2D8E770B5036813F00105064642
:10011000144605D013460A460146FFF7A9FE0546D8
:1001200021463046FFF716FE45B104F18042013A00
:1001300056F8223043F0004346F8223070BD70B5C7
:100140009DF910401E4623460546FFF761FE38B173
:100150002346324629462846BDE87040FFF788BE50
:1001600070BD2DE9F0438BB01446129D15F9046B58
:1001700000961F46804689462B460246214602A825
:10018000FFF7DDFF02A9129A0846FFF7C0FD129B98
:1001900002AA41464046FFF77DFD129B02AA214676
:1001A0002046FFF777FD2B464A46394638460096EB
:1001B000FFF7C5FF129A394602A8FFF7A8FD02A96A
:1001C0002B46424608460096FFF7B9FF02A92B4688
:1001D000224608460096FFF7B2FF2B4642462146CC
:1001E00020460096FFF7ABFF129B22464946484641
:1001F000FFF750FD2B4602AA414620460096FFF726
:100200009EFF129B224639463846FFF743FD2B4698
:100210004A46394638460096FFF791FF324602A912
:100220002046FFF7B9FD0BB0BDE8F08370B59DF92E
:1002300010401E4623460546FFF71AFE30B92246F7
:1002400029463046FFF793FD012807D02346324662
:1002500029462846BDE87040FFF7DABD70BD2DE99C
:10026000F0439BB01646229C14F9045B0095984617
:100270000746894623460246314612A8FFF75FFF2C
:1002800012A9229A0846FFF742FD229B12AA39467C
:100290003846FFF7FFFC229B12AA31463046FFF793
:1002A000F9FC23464A46414612A80095FFF7BEFFD7
:1002B00023464A46414640460095FFF740FF234605
:1002C0003A4631460AA80095FFF739FF229B0AAA51
:1002D00049464846FFF7DEFC2346324639460AA81F
:1002E0000095FFF7A3FF229A41463046FFF70FFD26
:1002F00023460AAA314630460095FFF720FF2346E1
:100300003246394602A80095FFF719FF229B02AA40
:1003100041464046FFF7BEFC23464A46414640461A
:100320000095FFF70CFF229A12A902A8FFF7EFFC35
:1003300002A923460AAA08460095FFF700FF2346B4
:100340003A4602A90AA80095FFF7F9FE0AA9229BDE
:1003500012AA0846FFF79EFC23464A460AA94846C9
:100360000095FFF7ECFE2A4602A93846FFF714FD78
:100370001BB0BDE8F0832DE9F04115468AB0044674
:1003800088461C22002103A8FFF7CCF82E1D95F902
:10039000007003232A46414620460293FFF7B7FC2C
:1003A000334602AA214620460097FFF7C8FE2B4697
:1003B000424621462046FFF76DFC0097334605F183
:1003C000840221462046FFF731FF0AB0BDE8F081E4
:1003D0000C4B1B78062B10D10B4B1B681A070CD14A
:1003E0000A4B186800F0F003302B08D000F0E00052
:1003F000A0F1400358425841704700207047012047
:10040000704700BFE00F00F0E40F00F0E80F00F0CD
:10041000094B1B78062B0CD1084B1B681A0708D117
:10042000074B186800F0F000A0F130035842584123
:1004300070470020704700BFE00F00F0E40F00F0AD
:10044000E80F00F010B9024B01221A60704700BF9C
:100450000050004010B50C494A6E042A044611D0E1
:100460000B6E1344032B02F101024A6688BF043B62
:10047000182202FB031318460021FFF753F82060EF
:10048000012010BD0020FCE700D1002010B504467B
:1004900086B01422002101A8FFF744F86088ADF867
:1004A0000800FFF749F92378ADF80600092B0CD8AE
:1004B000DFE803F005051014161B1D0E1F2107238E
:1004C0008DF8043008238DF80C3001A8FFF79AF955
:1004D00006B010BD0D238DF80430F6E70E23FAE7C1
:1004E00007238DF804300523EDE70F23F3E71023EE
:1004F000F1E70523EFE706238DF80430A3680393A3
:10050000A388ADF80630E0E72DE9F041067904460E
:10051000407B174603360023834204DB51B93E601B
:100520000020BDE8F081226912F833200132164420
:100530000133F1E73B68B34229D3237833F0030852
:1005400027D10B7022794A708D1C2846A1683BF098
:1005500019FC2279617BA954AB180133627B4245B7
:10056000DDDD226912F8382003F8012B226902EB45
:10057000C801184612F8382049683BF003FC22698C
:1005800012F838200346134408F10108E6E7042076
:10059000C7E70720C5E738B504461546084631B118
:1005A00062682B68934206D321683BF0EBFB6368DB
:1005B0002B60002038BD0420FCE708B5134644F248
:1005C0000102904203BF5A681988986800221AF005
:1005D00007F9000030B50B4B1B68012293F850104F
:1005E0000D338A4204DB405CB0FA80F0400930BD34
:1005F00013F8014B855CA54201D10132F1E70020DF
:10060000F5E700BFA0CA002003681A78302A27D176
:100610005A1C02605A7802F0DF024F2A03D10233DB
:10062000036008207047582A03D10233036010206A
:100630007047422A04D0082013F8012F22B97047CE
:1006400002330360022070472E2A07D0A2F138013E
:10065000012903D9303A092AEED970470A20EBE77D
:100660000A20704770B5244B0022C3F80025234AA6
:10067000516831B12249C3F8081322490420C1F856
:100680008000D3F80C55D3F81445D3F80815D3F8E7
:1006900010054FF0FF36B542C3F8146518BF05F5D5
:1006A000E075C3F80C65C3F80865C3F810651EBF94
:1006B0004FF0A043022643F82560651C1FBF4FF092
:1006C000A04304F5E074022543F82450441C1FBFE6
:1006D00000F5E0704FF0A043022443F820404B1C8B
:1006E0001FBF4FF0A04301F5E071022043F8210045
:1006F0000023D376536070BD0020004060CB002003
:100700008402020000E100E070B58AB00C460146A8
:1007100068461E462EF045F80022214605A82EF018
:1007200040F868462DF02BFF044605A82DF027FF62
:10073000844205460DD0039833F0B8FB089833F097
:10074000B5FB002C01DB002D00DA56B9601B0AB0A6
:1007500070BD002C07DA039833F0A8FB089833F03B
:10076000A5FB0020F3E768462DF0C1FC05A82DF09D
:10077000BEFCD6E7044A138A9BB223F0410343F040
:1007800040031382704700BF482E00200000000085
:100790002DE9F04F85B08A460390039C25782846C2
:1007A0002DF0FCFA0746C8B92D2D1AD101340123CA
:1007B00003940193DDF80CB0BAF1000F01D0CAF830
:1007C00000B003A8FFF720FF8046002835D1624D16
:1007D00000242046294605B0BDE8F08F013403947B
:1007E000DBE72B2D04BF013403940190E2E71846A8
:1007F00002932DF0A1FAB0F10009029B20DBC8455D
:100800001EDD40463AF040FD22462B463AF0A6FD5A
:1008100004460D4648463AF037FD22462B463AF04C
:10082000E7FB013604460D460396039E3378002B02
:10083000DDD1B8F10A0F37D113E000240025F4E729
:10084000B8F10A0F30D12E2B0BD10FF20419D9E9D0
:10085000008901360396039E30783038C3B2092BE5
:1008600039D9039B1A7802F0DF02452A1CD15A1CA1
:1008700003925A782D2A01D02B2A05D12D3A5742BE
:1008800003F10203574103934FF000080A20039A33
:100890001378303BD9B2092936D9002F39D12F4FDF
:1008A0000026B8F1000F46D1039BBAF1000F01D02A
:1008B000CAF800309B458AD09BF800202E2A03D12D
:1008C0000BF1010B5B4582D0019B002B81D005F120
:1008D00000431D467DE73AF0D7FC42464B463AF0CE
:1008E0003DFD02460B46204629463AF081FB002298
:1008F00004460D4640464946184B3AF059FE01362B
:10090000804689460396A6E7013200FB0838039229
:10091000BDE7124FC8F100080026B8F1000FC3D0A0
:100920002046294632463B463AF042FE08F101088D
:1009300004460D46F1E72046294632463B463AF04A
:100940000DFD08F1FF3804460D46AAE7AFF300801D
:100950009A9999999999B93F0000F87F000024402D
:1009600070B586B014460E460022014601A82DF04F
:1009700018FF2546DDE901239A4204D3049833F099
:1009800095FA601B04E02DB9049833F08FFA2046E5
:1009900006B070BD01A82DF0FDFD013D06F8010B6C
:1009A000E8E710B586B00A46014601A82DF0F9FE29
:1009B0000023DDE90112914203F1010401D2013368
:1009C0000AD1049833F072FA20202AF09DFA14F12B
:1009D000FF340AD206B010BD01A82DF0DBFD0A28B5
:1009E000EFD02AF091FA2346E3E70820EDE7000074
:1009F00070B50D2029F0DEFA0028264B46DB264C88
:100A00001871A17D01229A7000293DD1234DA18248
:100A100004334FF48E712846A360A275FFF7FAF8ED
:100A20002146AA60FFF725F9636893B92646A27D9F
:100A3000A38A9A420ED8A38A9BB2B3F5807F1BD0BB
:100A4000164BD3F81C21002AFBD00122DA600023C8
:100A5000A37570BDD5F81C3123B9A38A9BB2B3F539
:100A6000807FF7D1A38A9BB2B3F5807FE0D0314677
:100A70002846FFF7FEF8DAE70023A3750F210848A0
:100A8000BDE870402EF0CEB81121F8E700229A7030
:100A9000DFE700BFD9D2002060CB0020002000405B
:100AA0002EC1050030B58BB04FF4D8230193054615
:100AB00008B1002303602022002102A8FEF732FDC6
:100AC000002202A94FF4D82036F060F9D0B10024FA
:100AD000029B039A23F07F43033323F00303203365
:100AE00052B11C44032202A901A836F0D7F900280C
:100AF000EED120460BB030BD002DF3D02A68134450
:100B00002B60EFE70446F4E72DE9F04F202291B087
:100B100000244FF4D825824688460DEB020021467A
:100B2000CDE904540694FEF7FDFC012208A92846ED
:100B3000079536F02BF9A8B905AB019306AB5246E1
:100B40004FF4EC21009304A8434636F0E9FB0498E7
:100B5000013836F093F9049036F026FC012011B0EC
:100B6000BDE8F08F099B002B5DD0049E069BDDF84D
:100B70001C901E444E4523D0089B23F07F43203316
:100B80004B4401250D2702936A1E3E497A4302EB2E
:100B9000010B5846039232F08DFAA8B1DBF8001031
:100BA000894508D8029B994205D2A6EB09030B445C
:100BB000039A34495350013540F604439D42E3D92A
:100BC00020230DEB030214E0584632F07DFA002892
:100BD000F1D0DBF800300C33B3FBF7F31D44EAE748
:100BE00012F8011B0AF804100134B4FBF8F108FBF9
:100BF000114413F1FF33F3D2069B089E2033069372
:100C0000079B26F07F46033603F1200905AB26F04B
:100C10000306019306AF009743465246494604A88F
:100C200036F07EFB2EB9012208A907A836F036F966
:100C300081E7069B059AA8EB0300A8EB0405854213
:100C400028BF0546A24203D9121B954228BF15466C
:100C50000293ADB1B54228BF354649460AEB0400C0
:100C60002A463BF08FF8029B2C442B440693B4FB9E
:100C7000F8F308FB134405AB761BA9440193CAE7BC
:100C800028466CE7682E002030B58BB04FF4D8248E
:100C90002022002102A80194FEF744FC002202A9B0
:100CA000204636F08DF870B1032202A901A8DDE9D3
:100CB000015436F0F3F80028F6D124F07F442335B0
:100CC0002C4424F00304C4F5EC200BB030BD00002C
:100CD000F0B40023124D0D271C4640F6044607FBD6
:100CE00003519A1CC87ACC72087B0C73C2F30B00B8
:100CF0004A79087122F00F02013342EA1022B3420E
:100D00004A71ECD149F62B43064AEC54537823F050
:100D10000F035370044B01221A80F0BC32F01ABA50
:100D2000682E002093CA0020662E002037B50123CC
:100D3000009300231A460549054633F0B5FA0446E8
:100D4000284633F0B3F8204603B030BD0DC005008F
:100D5000F8B50646437A807A000150EA13100C4633
:100D600019D031F0DDFF074634F0CCF9451C384688
:100D700033F09CF8284632F085FF214633F09EFE82
:100D8000044638B10146304634F032FA204633F09A
:100D90008DF8681CF8BD0125ECE7000038B5074C5C
:100DA00025780023EDB202461946237035F0D6FBB4
:100DB00025700348BDE8384029F020BA642E002091
:100DC00040180600002370B50B6005460E4632F051
:100DD00021FE044670B1294633F071FD05462046D8
:100DE0001DB933F063F8284670BD32F077F93060F2
:100DF0002046F6E70546F6E72DE9F341002400F426
:100E00007F6715461470A7F54072502A0E4600F40D
:100E1000704312D8484A11F0100F484908BF1146D4
:100E2000002B79D0B3F5805F78D0B3F5005F444CE8
:100E300018BF00244FF440784BE0A7F50072202A39
:100E40000DD8002B6CD0B3F5805F6BD0B3F5005F8D
:100E50003C4C18BF00244FF400783B4939E0A7F51B
:100E60002072302A0AD8002B5ED0B3F5805F374C51
:100E700018BF00244FF4207835492AE0B7F5C07F29
:100E800009D1002B52D0B3F5805F324C18BF00243B
:100E9000B84631491DE0A7F11002B2F5887F47D866
:100EA00044F64302ADF80020C3F302321B0402F102
:100EB000310248BF4E2329494CBF8DF804408DF8BC
:100EC00003408DF8022048BF8DF803306C464FF088
:100ED0001008F00703D50F2228463AF095FFB20715
:100EE0000BD528463AF088FFA7EB08073F110122EF
:100EF00029180A23B8182CF010FD54B1330708D56F
:100F000028463AF079FF2146C0F10F0228463AF010
:100F10007BFF02B0BDE8F081114C8BE7114C89E7F3
:100F2000114C98E7114C96E7114CA3E7114CAFE731
:100F3000A0461149CDE700BF50BF050049BF0500DD
:100F4000B1E905006FBF0500FBE105007BBF0500AF
:100F500077BF05005ABF05005EBF050056BF0500FC
:100F600067E1050062BF050065BF05006ABF0500B7
:100F700073BF05007FBF0500411806002DE9F84347
:100F8000394F03791C2202FB03720646506820B1D8
:100F900032684FF40174C2F808431C2202FB037349
:100FA000DA7D52B11A7E002A41D020B133684FF465
:100FB0000172C3F80423112037E00120D875D960ED
:100FC0005A761A7635791C2303FB05739B7E1BB971
:100FD00012B93046FEF726FE4FF01C0808FB0578D4
:100FE0003068D8F80430002B35D14FF4A271FEF7E9
:100FF00011FEC5EBC50907EB89093068D0F824312B
:10100000D0F80821D0F84441A2B90CB9002BF4D093
:101010001C2202FB05750022EA750BBB14BBA97EDE
:1010200033680122A9B11A600020BDE8F883196174
:101030000122C6E7002BEBD1002CE9D14946FEF78F
:1010400001FE98F8193098F817209A42D5D823460F
:10105000DEE75A60E8E74FF40173C0F80433E3E7D2
:101060000320E2E70F20E0E760CB00200A490B48AD
:1010700008B5FFF783FF014610B109482DF0D2FDF6
:1010800008490648FFF77AFF014620B10648BDE847
:1010900008402DF0C7BD08BDD9D2002080BE050094
:1010A000E8C00500DAD200200BC1050038B50022E7
:1010B000054634F081FA044650B100231A46014631
:1010C00028462AF0F7FC2046BDE8384032F0EEBE54
:1010D00038BD0000F0B54FF080530220D3F8501413
:1010E000D3F85424284BC3F804032848C3F8040356
:1010F000274B93F800E093F801C09F78DE781D79C4
:101100005C7998794EEA0C033B4333432B432343EA
:101110000343204B2AD083F800E083F801C09F707E
:101120001E715D719C71D8711D789C785A785E79BA
:10113000586885EA0401514081F08801D970197915
:1011400071409E797140DE7971401972120203215B
:10115000597242EA05420C4B2243C3F8942500BA67
:101160004422C3F89005C3F8A025F0BD080A197001
:10117000090C9970110A1A715971110C120E5870DC
:101180009971DA71D0E700BF00500040800008007C
:10119000D4CF0020BFCF002038B50B4C0B4D2B789F
:1011A0005BB12CF0A1FB40B914F1FF34F7D2084930
:1011B0000420BDE838402DF075BE002CF7D02CF08F
:1011C00093FB0028F3D138BD80841E00C4D20020D8
:1011D00096BF050070B5EFF3108672B60D4A94689D
:1011E0000123A4B993600C4B0C4DD3F88010294017
:1011F0001160C3F88050D3F8841051604FF0FF3273
:10120000C3F88420047006B962B6002070BD037074
:10121000F9E700BFA4D2002000E100E0FC06FFBC1B
:10122000437882781B01120202F4E06203F030037B
:101230001343027802F003021343C278120302F44C
:10124000805213430279120402F4E02213434279DC
:10125000120502F4801213438279120602F08072A2
:101260001343054AC2F81835C379017AC2F8141538
:10127000C2F81035704700BF0070004010B588B04C
:1012800012788DF80C200021FF2202918DF80D209C
:1012900001214FF6FF72104C01908DF81C10ADF833
:1012A0000E208DF8103028F033FB70B12CF01CFBB1
:1012B00058B914F1FF34F6D2084904202DF0F2FD9C
:1012C00001A828F035FB08B010BD002CF4D02CF09C
:1012D0000BFB0028F0D1F3E780841E00F4BF05006B
:1012E000F7B5354F354C7E797601A31905465A7E00
:1012F000002A5FD1A2590AB101225A7695E80F005F
:1013000004EB060E0EF1080C8CE80F0006F1180332
:1013100023445A7922F003025A719EF81A20FF2AB8
:101320001FBF012393404FF0A042C2F80C352A683A
:1013300022B102F06043B3F1005F06D1AB6853B154
:1013400003F06043B3F1005F05D0344400236376BB
:10135000102003B0F0BD3B682979C3F84425C3F8D9
:1013600048152A7BA968C3F834150020C3F838252E
:10137000C3F81801D3F818210192019AC3F8500557
:101380000122C3F840051A61A2597AB9D3F818218D
:10139000002AFBD03444A27EFF2A05D001239340CB
:1013A0004FF0A042C2F808350020D2E74022C3F82F
:1013B0000423CEE71120CCE7B42C0020A4CB0020DE
:1013C000F0B5154685B01C4E07460C46FFF7E4FE07
:1013D0000123FF2D33702B4628BFFF231FB3FA18BC
:1013E00016490A600CB3E218154900970A60154ABD
:1013F0000294002CA5EB0305DBB21560684614BF10
:101400001A4600228DF80C208DF80430FFF768FF93
:10141000024660B1002404200B4934702DF042FDD7
:10142000204605B0F0BD3A46DAE72246DCE7FFF792
:10143000B3FE0120F5E700BFC4D20020C8D20020CF
:10144000C0D20020B8D2002083BF050013B51A4BCC
:101450001B78044663B3FFF79FFE184B1B680022FE
:1014600001200421C3F80025C3F80005C3F80813C0
:10147000C3F80821D3F80811009100991049E4B28B
:101480000870C3F81C45D3F808010028FBD0C3F846
:101490000821D3F8080101900198D3F818050A70C3
:1014A000C3F800250722C0B2C3F8002502B010BD62
:1014B0004FF0FF30FAE700BFBCD20020B42C002070
:1014C000C4D2002037B50B015BB249B2044643EAEF
:1014D00001008DF804001A4D50B20343120152B2BC
:1014E0008DF805302B78114302438DF806108DF8E6
:1014F000072013B302AB03EB941302AA13F8040CF6
:10150000C4F30113134413F8043C43EA00201AF017
:1015100027FC2B788BB102AAC4F3810304F00304E7
:101520001344144413F8040C14F8043C43EA002058
:1015300003B0BDE830401AF013BC03B030BD00BFAB
:10154000BCD20020C30914BF13020B0210F0400FDD
:1015500070B5064614BF10460846184314460D469B
:10156000FFF774FFB1064CBF23022B0216F0100FD9
:1015700014BF204628461843FFF768FF32074CBFC8
:1015800023022B0216F0040F14BF204628461843EE
:10159000FFF75CFFB3074CBF2002280216F0010FD3
:1015A00008BF2C462043BDE87040FFF74FBF000046
:1015B0002DE9F047FF2705463C4604264FF6FF7805
:1015C000296911B9002E61D051E0286822F02CFE63
:1015D000064600284BD168690378002B5ED0C27A9A
:1015E000E52B02F03F0247D022F02001082943D02A
:1015F0000F2A46D159063DD503F0BF04EB88477B3F
:101600002B84437BBB4237D10378EE69DFF890E04F
:1016100003F03F03013B0D2253434FF0010C002127
:101620001EF8019B00EB090292F801A010F80920B6
:1016300042EA0A22BCF1000F20D03E2B1CD826F82B
:1016400013209446013301310D29E9D10278520665
:1016500004D53E2B10D8002226F81320013CE4B21A
:101660000021284623F05EFA06460028A8D0002371
:101670002B610CE0A342C4D0FF24F1E74245E2D045
:10168000FAE73CB922F060FDB84203D100263046AB
:10169000BDE8F0874FF6FF732B84F8E70426E6E7F2
:1016A00072BE050020292DE9F0470BD9244A254EAA
:1016B0002139C9B200231446DFB2B94205D814F863
:1016C00001C0B6BB4008BDE8F08712F8017B0133CA
:1016D0003E44F1E7745CC82C1ED81EF80450DFF8B5
:1016E0006C90194B4FF000085FFA88FA54450DD8FA
:1016F00003EB0509994511D101316145EADB02325D
:10170000504320F0704007300009DCE719F801ABC6
:1017100008F101085344E7E70023E9E713F8018BD8
:10172000B8FBF7F407FB1484E4B2A242B8BF224628
:10173000E0E700210A46DFF814E00D27DDE700BFEF
:101740004FC105002EC2050052C4050089C3050023
:1017500010B5074A002332F8024B8C4203D11841DE
:1017600000F0010010BD0133082BF4D10020F9E78F
:10177000A8CA0020F0B5224B9F7C1C4600221D46C3
:10178000D6B2B7420ED895F878701D4C0022D6B26A
:10179000B74216D895F8DE500022D4B2A54220D820
:1017A00000200DE0B4F814C0844502F1010204F1F8
:1017B0000A04E5D142F64D2301200B808870CE70DB
:1017C000F0BDB4F87AC0604502F1010204F10A04E8
:1017D000DDD142F64D230B8002238B70CE700120A9
:1017E000EEE7B3F8E060B04202F1010203F10A0350
:1017F000D3D142F64D230B8003238B70CC70EEE7E0
:1018000030CD002010B50C4C226886B0034682B162
:1018100004208DF804000868D989ADF80C10123343
:1018200033F8021C0290ADF80E10049301A9204673
:10183000904706B010BD00BF30CD00207FB54B896A
:10184000022B0FD1094A136863B1097B006802902B
:1018500011F0010F14BF022103218DF8041010466E
:1018600001A9984707B05DF804FB00BF30CD002008
:1018700070B50D4D002435F8026B964210D101224F
:10188000A240D2B2D543EDB2014410F8014B2BB1C6
:101890001443884200F8014CF7D170BD2C40F8E7A2
:1018A0000134082CE7D1F8E7A8CA002070B500235E
:1018B000084C1A4641FA02F5ED0706D504EB42063C
:1018C00000EB4305B688AE8001330132082AF1D11E
:1018D000036070BDA4CA002010B586B00446002283
:1018E000684616F07FFF2046009916F043FD20461B
:1018F00006B010BD38B501230B7004460D4631F01B
:1019000086FB88B100220B49204633F055FE10B10A
:1019100034F0D3FA287020460022074933F04CFEF9
:10192000BDE8384034F090B92046BDE8384033F087
:10193000E9BB00BF3CBF050041BF05002DE9F04FEA
:101940002DED028B8DB0436A059390ED048B1F0241
:10195000836A07671E024667B0EE480AF0EE680A1F
:101960000446069337F070FB59EC108BB0EE480A32
:10197000F0EE680A37F058FC94ED067B404653ECD5
:10198000172B49465BEC10AB8DED007B39F010FE58
:101990000022614B39F0E2FC0022604B39F028FB59
:1019A00039F08CFFDDE900230790A06759465046C7
:1019B00039F0FEFD0022584B39F0D0FC0022574B85
:1019C00039F016FB39F07AFFE0670546059839F0E3
:1019D0005BFC29F00043CDE908010698CDF80880AA
:1019E000039339F051FCDDE90223CDE90A01DDE979
:1019F000080139F0B3FCD0462BF0004942468B4633
:101A00004B468246DDE90A0139F0A8FC02460B4646
:101A10005046594639F0ECFADDE9002339F09EFCD6
:101A200000223E4B39F0E4FA39F048FF42464B467B
:101A30008346DDE9080139F091FCDDE90A2380469F
:101A40008946DDE9020139F089FC02460B46404631
:101A5000494639F0CDFADDE9002339F07FFC2F4B00
:101A6000002239F0C5FA39F029FF94F820305BB133
:101A7000226863680BEBDB71A2EB6102226000EB72
:101A8000D072A3EB620363602368059A5B44A36092
:101A900063680344E360079B0BFB03F3013300FB24
:101AA000053303EBD373D201A2EB6303C4F8803098
:101AB000079B58430130069B0BFB150505EBD575BD
:101AC000D80194F82130A0EB6505C4F884503BB9E7
:101AD0000DB0BDEC028BBDE8F08F3B44C4F8803004
:101AE000D4F88030002BF8DBD4F880309F420BDD37
:101AF000D4F88430002B0BDBD4F884309E42E7DC32
:101B00009B1BC4F88430F7E7DB1BC4F88030EBE79D
:101B10003344C4F88430EBE7000070400000E03F3D
:101B20001F4B204A1B6800BF00BF00BF00BF00BFA3
:101B300000BF00BF00BF93422FD000BF00BF00BF57
:101B400000BF00BF00BF00BF00BF00BF00BF00BF9D
:101B500000BF00BF00BF00BF00BF00BF00BF00BF8D
:101B600000BF00BF00BF00BF00BF00BF00BF00BF7D
:101B700000BF00BF00BF00BF00BF00BF00BF00BF6D
:101B800000BF00BF00BF00BF00BF00BF00BF00BF5D
:101B900000BF00BF00BF00BF00BF0138C3D1704706
:101BA000A42C00200024F40008B1FFF7B9BF70474F
:101BB000084B5A6E013A5A6622B907490A7822F050
:101BC00002020A701A6E0132042A08BF00221A6645
:101BD000704700BF00D1002022CD002030B5044660
:101BE00085B00D46102200216846FDF79BFC237A44
:101BF000012B0AD0022B0ED063680193236829467B
:101C00009B686846984705B030BD23690293A38A54
:101C1000ADF80C30F0E70123A2898DF80030E3899C
:101C2000ADF80A20D31AADF80830E5E728DF704791
:101C300029DF704738B51C4B5A6E19465AB31C6ED3
:101C4000182202FB04331A7A012A07D0022A23D071
:101C500018460921BDE83840FFF7C0BF1825D88ACB
:101C60009A8A05FB0414D4E90314121AB2F5806FA2
:101C70004FEA80000144B4BF92B24FF48062204426
:101C8000FFF7D6FF11280BD1084A137823F002037F
:101C900043F00403137038BD9889FFF7C7FFF1E7DD
:101CA0000028F8D0D4E700BF00D1002022CD0020CA
:101CB000054A137813F0060F04D143F002031370A2
:101CC000FFF7B8BF704700BF22CD00202DE9F341D8
:101CD0001F4B1B781746DA07064688462BD51D4D45
:101CE0001D4B9D4229D31D4B9D4226D239B330B3A3
:101CF00041EA00039B0724D12B68984223D36A68EA
:101D000000EB87039A421ED3FFB101A8FEF7A2FBA6
:101D100078B1019B0024C3E90054019B01221A728F
:101D2000C3E903869F82FFF7C3FF204602B0BDE8E8
:101D3000F0810720FAE70120F8E70220F6E7032008
:101D4000F4E70620F2E70520F0E70420EEE700BF05
:101D500022CD0020102E0020102E0020202E00204A
:101D600038B5074B074A5968948810684A88033287
:101D7000032592B200EB84001D70FFF7A7FF38BD6A
:101D800024CD0020A4D1002010B501220C46064924
:101D9000FFF79CFF28B9054901EB041101238B7360
:101DA00010BD0E20FCE700BF2CC0050060D0002055
:101DB00008B502220149FFF789FF08BD30C00500C0
:101DC00008B5034B034918680222FFF77FFF08BDDF
:101DD000A4D1002038C0050073B51B4B1B78DB076E
:101DE00005462BD5194E1A4B9E4229D3194B9E42BC
:101DF00026D238B3C0F30B04D4B93368984219D350
:101E0000726800F580539A4214D301A8FEF722FBB2
:101E100090B1019BC3E90064019B02221A722D0B51
:101E200001229D811A82FFF743FF204602B070BD58
:101E30000620FBE70520F9E70720F7E70120F5E793
:101E40000220F3E70320F1E722CD0020102E00202E
:101E5000102E0020202E002010B50B4C0B4B62885A
:101E600003EB02139A892AB95868FFF7B5FF0423D8
:101E7000237010BD05232370054B022218689A8039
:101E8000FFF7AAFFF5E700BF24CD002060D00020B7
:101E9000A4D1002008B5074B191D5888FDF79AFBFF
:101EA00018B1BDE80840FFF75BBFBDE80840FFF789
:101EB000D3BF00BF24CD002010DF7047002208B53B
:101EC000114618F08DFC00002DE9F347254B1B68E7
:101ED0001BB1984730B3FFF7F1FF234B1B7803F09A
:101EE000FF07FBB1214D224E2C68DFF88C90B4FA2D
:101EF00084F46409B0463378A3B901A8FDF74EFB1A
:101F0000052812D00028E6D1019B0BB9FDF722FD70
:101F1000184B1B680BB1019898474CB10124EAE7B4
:101F2000002CFBD002B0BDE8F087002CFAD13C4673
:101F3000DFF848A098F80030002BF3D1B9F8003052
:101F4000ADF80430DAF8003001A91846FDF724FB9B
:101F50000528E5D00028BED12A6818469047002CF5
:101F6000E8D1C8E710CD0020A1D10020DCCA0020B4
:101F7000A2D10020ACD10020D8CA00209CD20020E1
:101F800010B5084B9A685AB150B9EFF3108172B688
:101F9000054A1C6814605C685460986001B962B6B8
:101FA000002010BDA4D2002000E100E073B505467A
:101FB000B8B1C1F3C70401F0070301269E40035DD9
:101FC00033420ED000230DF107008DF80730FFF7E4
:101FD00001F92B5D9DF8070023EA06062E55FFF751
:101FE000CFFF02B070BD000038B50A4B1A687AB155
:101FF0005D686DB1FF280BD084B221462846FDF7FD
:102000001BFC28B121462846BDE83840FFF7CEBF6B
:1020100038BD00BFECD1002038B504460025E36888
:10202000AB420ED84FF6FF732380A3700023C4E9A0
:102030000133E360238A03F4784343F0FF032382F0
:1020400038BD207C2844C0B2FFF7CEFF0135E6E75B
:1020500037B5FDF7B1FB0546A0B144682CB10A4B7A
:1020600001941B789B0706D403242846FFF7D4FF6E
:10207000204603B030BD01A8FDF792FA04460028BF
:10208000F3D0F1E70524F3E721CD0020FF2810B5B8
:10209000044609D801460548FFF788FF2146044851
:1020A000BDE81040FFF782BF10BD00BFB8D00020D0
:1020B000D8D000202DE9F3411D4F7B6806460D4620
:1020C0009BB304292FD943697BB3437C0024012BA4
:1020D0000DF107000CBF8846A0468DF80740FFF7BA
:1020E00079F80DF10600FDF703FBD0B10123037071
:1020F000104B4660D3F80435C0E90484C0E90235CA
:102100009DF806307B709DF80700FFF739FF24B972
:10211000094B4FF48012C3F80021204602B0BDE8FD
:10212000F0810424EFE70724F7E70824F5E700BF70
:10213000DCCF00200010014000E100E02DE9F34178
:10214000CE0801F007044FF0010808FA04F4855D99
:10215000E4B22540074613D10DF107008DF8075072
:10216000FFF738F8BB5D9DF807001C4202BF1C4317
:10217000BC554546FFF704FF284602B0BDE8F08194
:102180000025F9E72DE9F74F9846531E072B8146A6
:102190000F46154600F2BB80FF2800F2B8800146CA
:1021A0005E48FDF749FB0646002800F0B08039463E
:1021B0004846FDF701FB044600283ED0C3689D4217
:1021C00047D805D25FFA85F9E368207C994543D367
:1021D00094F81090B9F1FF0F40F09780504B1A68B7
:1021E0009B46002A41D14FF6FF732380A370002342
:1021F000C4E90133E360238A03F4784343F0FF0327
:102200002382112084E0237C1844C0B2FFF7ECFE47
:10221000E3685FFA8AF083420AF1010AF3D84FF6C5
:10222000FF732380A3700023C4E90133E360238A92
:1022300003F4784343F0FF032382FF214FF6FF703E
:10224000FDF7BAFA04460028DBD0A0F800908770AA
:10225000BEE74FF0000ADBE74844C0B209F10109CC
:10226000FFF7C2FE5FFA89F9AEE75B68002BBAD0D0
:102270000023DBF808205FFA83FA924502D34FF07F
:10228000FF0912E0DBF8040060B351460193FFF749
:1022900055FF019B30B3B9F1FF0F08BFD146AAEB40
:1022A000090A0AF1010AAA4521D1B9F1FF0F84F800
:1022B000109098D0E560207CFDF7CEFA58B305EB7E
:1022C00085052D01ADB2AD0888F80270C8F804008C
:1022D000A8F8005026B1082F02D1AD00063D858038
:1022E000002015E0B9F1FF0F0CD14FF0FF090133C9
:1022F000BFE74846019309F10109FFF775FE019B0D
:102300005FFA89F9D145F4D3EFE70026D2E7072039
:1023100003B0BDE8F08F0320FAE700BFB8D000207B
:10232000ECD100202DE9F3478146002701261FFA52
:1023300087F84FEAD80A08F0070406FA04F419F8F7
:102340000A50E4B2254008D00137B7F5807FEED1BE
:10235000B846404602B0BDE8F0870DF107008DF8A1
:102360000750FEF737FF19F80A309DF807001C42A6
:1023700002BF1C4309F80A400125FFF701FE002DAA
:10238000E2D0E6E713B50DF106010446FDF74AF980
:1023900070B1BDF80620084B03EB02139A894AB1CD
:1023A000A17A39B1013A00209A81A07202B010BD21
:1023B0000A20FBE70620F9E760D0002037B50D467C
:1023C0000DF106010446FDF72DF988B1BDF8062090
:1023D000084B616803EB021300209A8901329A814D
:1023E000296063680C336B600123A37203B030BDB6
:1023F0000A20FBE760D000202DE9F043DFF884805D
:10240000D8F874E0BEF1030F0F46944635D81C4E41
:10241000756CC1F108039D422FD8D8F87040744400
:102420001C2304F00304814603FB0484B9E80F0075
:102430000FC499E807000EF1010384E80700C8F80B
:102440007430C7B1336C2B4403F0070306EBC303AE
:10245000002206F138040CEBC20103C9A34202F1C9
:10246000010283E8030014BF0833054B9742F2D101
:10247000736C1F447764012000E00020BDE8F08306
:10248000E8CB0020E4CF00202DE9F0411C46184B9A
:102490001B789B0706460F46154627D5DFF8588060
:1024A000A3880BB10A201FE098F800302BB9214611
:1024B000A088FDF78FF820B92060A3880133A3809E
:1024C000EEE723681EB1998832889142EFD11FB19F
:1024D00019883A889142EAD19B682B6023686B6027
:1024E000044B1B892B810020BDE8F0810220FBE713
:1024F00021CD002024CD002060D0002030B587B051
:102500004CF2070305460C46ADF8043003AA0F4B06
:1025100001A90020FFF7B8FF10B1002007B030BDBF
:1025200001A903A8FFF74AFF0028F6D10723A370EB
:10253000019B5A882280029A62609B8803F580433F
:102540002B8003A8FFF71EFF0120E7E714CD002032
:102550001FB50023A0F58040A1F58041CDE90233ED
:10256000ADF80400ADF8061002AB0DF1060101A8AC
:10257000FFF78AFF002818BF052005B05DF804FBAF
:102580002DE9F04102230B80164B00251C6800F555
:10259000805E2F4608304FF6FF7870450AD305B1AC
:1025A0001C6002B11770BDE8F08101270EE03446CF
:1025B00001250BE006680136F1D086884645F4D047
:1025C0000688002EF1D08668A642F0D8468806F12B
:1025D000030C00EB8C00B1F800C00CF1030C664456
:1025E0000E80DAE7ACCE002070B5064D064600241A
:1025F00055F8043B0BB1304698470134082CF7D10D
:1026000070BD00BFC4CB00202DE9F047AA4C266F57
:102610001C2707FB06F586B0635D013B8046052B52
:1026200000F22A81DFE813F00600640064001D0157
:102630001D017E0130B1A14A137823F0010313700C
:1026400001201FE025442B79032B15D8DFE803F088
:1026500002072C34FFF7B4FB01232B7109E0984DDE
:102660002B78022B40F03C826868FFF7A1FB002327
:102670002B70002800F0F080904A137823F00103BB
:1026800013700E201C237343E218E35C0290023B9C
:10269000012B00F232818B4B907D196C5A6C0144F6
:1026A000121A19645A6428E1874F3868FFF794FBBF
:1026B0000223BB800023D0E7834FDFF80482386811
:1026C000FFF776FB814BD7F800E05B88B7F804C0D2
:1026D0001B0108EB03025168A2F808C0C2F804E02D
:1026E0000222BA800022396008F803202A71C0E76C
:1026F00007FB0647724BB7F812A04FEA0A1A03EB22
:102700000A029946118960B1FB8803F103088844E5
:10271000C3F57F435189A2F80880FD330B445381F0
:102720008EE7536803EB81083B7C062B00F2978011
:10273000DFE803F02D733C4D1F84040041F61D506B
:102740001C2303FB0643D144DB88B9F80810DA1CCC
:102750000A44A9F80820C3F57F43B9F80A20FD33DD
:102760001344A9F80A3041F61D53984200F0C38083
:1027700088E757485749002343601C2303FB06435F
:102780009B690360FCF74EFF002800F04C81291D77
:10279000012221444046FFF799FA1C2303FB06431C
:1027A00002221A74002857D00E20C9E705F10C0147
:1027B0000122214408F10800FFF788FA1C2303FBDB
:1027C00006439A7D002A14BF03220122E9E73D4B0C
:1027D0005A6C002A00F08C81196C1C2505FB0645FB
:1027E000481C00F0070003EBC1071864A88A53F8DF
:1027F0003110013A5A6408EB8000BA88FFF766FA94
:10280000AB8ABA881344AB82AB7D013BDBB2AB75BC
:10281000002BC7D101232B74C4E705F10801012265
:10282000214408F10400FFF751FA1C237343E25CD2
:10283000032A0CBF052206222344B2E7254B198840
:10284000234B5868FFF7A0FA1C2303FB064306221C
:102850001A7400287FF474AF06B0BDE8F0870F202B
:102860006EE700287FF4ECAE07FB06473B79012BAF
:1028700032D01BB1022B3ED00F2003E7CDE902007E
:10288000FB6801930DF1020101A8FCF7CBFE80B1BA
:102890000298BDF802108388FB8003883B81FFF714
:1028A00073FA1C2303FB064302221A710028D3D0BB
:1028B00059E70A20F5E700BFE4CF002021CD002032
:1028C00060D00020E8CB0020A4D1002024CD00203F
:1028D0003C2E0020B0D20020864FA81D3B4601AA06
:1028E00041462044FFF7D0FDB8B9B9880298FFF7F8
:1028F0004BFA0A28DAD1002302931C2303FB06F2C9
:10290000A25C013A052A00F2B580DFE812F08E00E1
:102910009200A000CB00D500E1000A28C7E900889A
:10292000E9D020E700287FF48BAE734BDA7AAAB1A6
:10293000D8721A78013A062A9ED801A151F822F0DD
:10294000F1290200EB290200012A0200072A0200F5
:10295000792802000D2A02001D2A02001A78072A8F
:10296000E7D801A151F822F0892902003329020099
:1029700033290200A5290200B9290200D729020043
:10298000D7290200A12902001A8901321A810022E6
:102990005A80DA72594A1278B2FA82F252099A725D
:1029A000012207E0564958688A8840880332024469
:1029B0008A8002221A70BCE75D88504A504902EBB7
:1029C00005120868556850608888108102228A8044
:1029D0000D600622EEE70722ECE7484900229A72D2
:1029E0008A8942B9897B31B15A80FFF753FA5DE792
:1029F0009A7A002AF1D100221A705A805A607AE736
:102A0000FFF7AEF952E7FFF727FA4FE75A883B4B3B
:102A100003EB02135868FFF7CBF947E700225A602F
:102A2000FFF7CEF942E70A202CE600238DF80430A8
:102A300020E003FB064301228DF804201A89ADF83B
:102A400010209A88ADF81220DB68039312E003FB94
:102A5000064302228DF804201A89ADF810209A88C6
:102A6000ADF81220DA681B7C03929A1F534253413F
:102A70008DF8143001A8FFF7B7FD206F1C2200214C
:102A800002FB0040FCF74EFD636F1BB3226F013267
:102A900002F00302013B22676367DBB10020FFF70E
:102AA000B3FDD9E603FB064303228DF80420DA8840
:102AB000ADF810201A89C5E703FB06430422DB8822
:102AC000ADF8103000238DF80420ADF81230D1E7B6
:102AD0000523ABE70B4A137823F004031370BBE61E
:102AE000084A137843F0020323F00103137002E74E
:102AF0001368FFDED0D2002024CD002060D000205B
:102B0000A4D1002021CD00200846FFF77DBD0000A4
:102B1000054A137813F0040004D143F00403137042
:102B2000FFF772BD704700BF21CD0020F0B51C46F5
:102B30003D4B1B789E0789B007460D466FD5098827
:102B40004FF6FF7399426CD06B88002B69D069688F
:102B5000B5F808C000239C4503D8BAB9164604311D
:102B60000AE051F83300800757D10133F3E731F819
:102B70003200304486B201329445F8D80DF102019A
:102B80003046FCF797FD28B109B0F0BD1388568890
:102B9000ADF8023000238DF81430BDF80230ADF8E6
:102BA00016300323ADF81830204B8DF804401A6816
:102BB00029898DF81A1001321A602B88ADF80C3073
:102BC000032C6B88ADF8083004BF04238DF8143053
:102BD000049208BF3B686A6808BF0793002401A8F5
:102BE000ADF80A60ADF80E40FFF706FC50B9BDF82D
:102BF00002200F4B03EB021358890338801B5881C6
:102C00000820C1E7049B3B600A4B7C601B89BC72B7
:102C10003B81FFF77DFF2046B6E70320B4E70220A3
:102C2000B2E70420B0E700BF21CD0020ACCE0020E9
:102C300060D0002024CD002030B58BB0FF280446A2
:102C400001921D4645D88B781846FCF78BFD00286D
:102C50003FD04A6802920A88ADF80C20A4F5804261
:102C6000ADF81C20A3F58042ADF81E2002AA089200
:102C70000122ADF82420194604AA2046FFF768FC7B
:102C80000528019A0ED1022352B907A904A8FFF71B
:102C90004DFF07281FD010D8B0B103200BB030BDB6
:102CA00001AAF2E732B10E4B1B789B0702D501A8AF
:102CB000FCF776FC03230022E7E708280DD00E2856
:102CC0000CBF11200320E9E7002DE7D0049B2B6007
:102CD000E4E70720E2E78620E0E71120DEE700BF17
:102CE00021CD002073B5154E736805461BB34369AB
:102CF0000BB3002404740DF107008DF80740FEF7B4
:102D000069FA0DF10600FCF7F3FC90B102230370A1
:102D10009DF80630456073709DF80700FFF730F9A5
:102D200024B9074B4FF48012C3F80021204602B0AB
:102D300070BD0424F0E70824F8E700BFDCCF0020D2
:102D400000E100E02DE9F8432649274B0025C1F8B2
:102D50004051C1F84451C1F84851C1F84C51C1F833
:102D60000051C1F804511B68002B39D0D1F804453B
:102D70001E49DFF88C800968641A24F07F442F46CE
:102D80001A68A24217D8A41A15441A7CDE6982B1C7
:102D9000D8F800901F74D3E90521B9F1000F06D0CF
:102DA0001046C84728B1FFF789F83346E8E70846D8
:102DB0009047002EF9D10E4A0E4B11781B788B42AA
:102DC00005D10133DBB2022B08BF00231370127848
:102DD000094B43F82250094B4FF48012C3F80021ED
:102DE000BDE8F88300100140A0D20020BCD1002033
:102DF000B9D10020B8D10020B0D1002000E100E01E
:102E00000CCD00200D4B0E494FF4003210B5C3F825
:102E1000802001244FF48033C1F848332F20C1F8BB
:102E200008334C60FEF77CFE064B8C602F2000219F
:102E30001960FEF775FE044B197010BD00E100E04B
:102E400000100140BCD1002099D100202DE9F04FA5
:102E5000B64AB74913780978B64D85B09942D5F886
:102E60000080019500F095800133DBB2022B08BF92
:102E7000002313701278B04B53F82260019A08EBCC
:102E8000060323F07F4313600127AC4BAC4A18685C
:102E90000290AC48117890F800904FF0000CE24698
:102EA0005078884278D1BCF1000F02D0A54981F852
:102EB0000090002F40F0BB801F6802997F1A18BF56
:102EC00001270020196802919E49039191F800E0C2
:102ED00000244FF00108002840F0AD8092F80190E6
:102EE000D2F804C092F802A01178494540F0C180A0
:102EF0001B68029A9A4201D1002F44D0002B00F0A7
:102F00001281D3F80090904C019BD4F804651968A5
:102F10008E4F751A3B7825F07F450335A3B94FF4E2
:102F20008033C4F84433C4F80433894B4FF400327F
:102F30004FF00108C3F880212F201A60C4F80080E8
:102F4000FEF7EEFD87F80080A9452CBF49444919DA
:102F500021F07F41C4F84015D4F804359B1B23F0C1
:102F60007F43891B033321F07F418B420BD9D4F877
:102F70000435C4F840352F20FEF7D2FD744B4FF4D2
:102F80000032C3F80021039A0023137005B0BDE896
:102F9000F08F0026374678E701EB4104506892F83D
:102FA00002B000EBC40E013110F834401868C9B209
:102FB0008B4508BF0021022C04D0032C7FF470AF96
:102FC000002410E0DEF804B004468646002C3FF4EE
:102FD00067AFA34500F0C080A646E469F6E780F835
:102FE00010A0C06901240028F9D1002C3FF458AF8B
:102FF000186055E7D4F80C90C4F800E0761A8C44B9
:10300000E1691960B9F1000F07D008EB0C0121F05C
:103010007F41C4E90119E06120461C68002C3FF49F
:1030200051AF2168B142E5D98E1B26604AE70020E6
:1030300084468646F1E70146C069019DD1F804A0A7
:103040002E68444DD1F80890AAEB060C2CF07F4C6A
:10305000AC4535D80CEB09060E60D3F800C081F8FA
:103060001080C1E90144CC61BCF1000F33D119607B
:1030700031E701EB410B0131C9B2514514BF117069
:1030800014701CF83B1001290CEBCB067FF42CAF1D
:10309000716891F810B0BBF1000F7FF425AFD6F83E
:1030A00008C0C1F804C0F5688D603569CD607669E7
:1030B0008E61BEF1000F0CBF66465E464E60BCE7F7
:1030C000A6EB0A0626F07F464E4502D2A9EB06067D
:1030D000C2E70C60C1E7D1F80090DCF80060B145B0
:1030E0001FD8A6EB0906CCF80060C1F81CC0BEE7EB
:1030F000A9EB0A09D6F81CA0B446BAF1000F0AD011
:103100005646D6F800A0CA45F2D3AAEB090AC6F87B
:1031100000A0B2466646C1F80090C1F81CA0F1615B
:10312000D9E66646EDE7FFF76DFE2CE7B8D1002043
:10313000B9D10020BCD10020B0D10020A0D2002005
:10314000DCCF002098D100200010014099D1002050
:1031500000E100E0FEFF7F0074450FD1D0F81CB005
:10316000C3F800B0BBF1000F08D10A4D0120A860E0
:1031700001984FF0010CC0F800B0E1462068E46906
:10318000CEF81C40002C3FF48BAE2568284420600C
:1031900086E600BF0010014037B5074B054693E8AF
:1031A00003006C46002384E803001A4621462846A3
:1031B000FFF742FD03B030BD50BE0500FDF766B914
:1031C00010B54FF6FF7304469C42084609D1FFF73D
:1031D000A9F8B0F5807F044601D14FF6FF74204670
:1031E00010BDFF2CF9D82146FEF7A8FF0028F6D124
:1031F000F3E710B5044601F0EFFC2046BDE81040AF
:1032000000F02EBF1FB5037893B90279072A0FD1BA
:10321000448803932046CDE901338DF80420FCF760
:103220008BFAADF8060001A8ADF80840FFF7E1FF02
:1032300004B010BD1FB50023CDE901330393ADF8F1
:103240000600022301A88DF804308DF80810FFF75E
:10325000D0FF05B05DF804FB86DF704738B5048801
:103260004CB9821C00F10A0512F8013B1BB99542CA
:10327000FAD100200AE00B88A342FAD108220231D9
:10328000023038F071FDB0FA80F0400938BD08B561
:1032900070B171B103780A78534013F0FE0F08D172
:1032A00006220131013038F05FFDB0FA80F04009AC
:1032B00008BD0020FCE710B5044600F0BDFF204625
:1032C000BDE8104000F04ABF43DF70476FDF704732
:1032D000024B0022C3E90022704700BF14CD00203A
:1032E000F0B5FF2887B004460E4615461F4629D87C
:1032F0000846FCF737FA28B303AA2046FFF728F957
:1033000018B10524204607B0F0BD01A903A8FFF7B6
:1033100055F804460028F4D1019BAE705A882A80E3
:103320005FB13B6892009A420AD30299686838F00C
:1033300029FD03A8FFF726F8E4E7029B6B60F8E796
:103340000424DFE70724DDE72DE9F041CEB020AE0D
:10335000502380460CADB8220021304601930395DE
:10336000FCF7E0F80DF1970305930DF1AE0306931A
:103370000DF1C503079337AB08930DF1F3030993E0
:103380000DF585730A931C4F04960DF221130B93D0
:103390000024444507D1E2B2002104A8FFF796FFBC
:1033A0004EB0BDE8F081502200212846FCF7BAF863
:1033B00001AB02AA072137F8020BFFF791FF20F0BB
:1033C00002000528ECD06B7C032B12D817230DF1DB
:1033D000310203FB04630DF1450152F8040B43F87D
:1033E000040B8A42F9D11188198092789A700134BD
:1033F000CFE743F20220D3E7CAD100202DE9F04104
:1034000010220546A6B000212D48FCF78BF835B9EF
:1034100029462846FCF7A4F926B0BDE8F0816A00E9
:1034200028492748DFF89C8004AE38F0ABFC3822EE
:1034300000213046FCF776F800245023CDE9013412
:1034400012AF0397502200213846FCF76BF801AB0E
:1034500002AA072138F8020BFFF742FF20F0020012
:103460000528D9D09DF85930032B26D8C4EBC402C7
:10347000B318DDF85910B1500134BDF85D209A80C1
:10348000A5429DF85F209A71DCD10DF117031393CB
:103490000DF11E0314930DF1250315930BAB169339
:1034A0000DF1330317930DF13A0318930DF1410316
:1034B00012961993E9B23846ACE743F20220ABE723
:1034C000DAD10020CAD100202DE9F043037889B079
:1034D0000546002B3FD1017907293CD104AA408839
:1034E000FFF7FEFEB8BBFFF7F3FE02A90DF10600E1
:1034F000FFF704F878B36E88BDF80670BE42F4D0CA
:10350000059C631C1846113413F8012B12B9A34211
:10351000FAD1EAE7DDF80C80102208F1010138F059
:1035200023FC08F1110181462046FFF7B0FEB9F1F6
:10353000000F01D00028D8D03046FCF7FDF800235A
:10354000ADF81A0006A88DF81830ADF81C60ADF87B
:103550001E70FFF7B0FE09B0BDE8F083CA1F012A54
:1035600073B5064654D80025CDE900558DF80210F4
:10357000FCF722F9044600284CD0437CDB074BD4EF
:10358000007CFCF769F910B9032002B070BDE36854
:10359000019003EB83031B019BB29B086846ADF8C7
:1035A0000030FCF7E7F8626804F10803694630462A
:1035B000FFF742FB637C03F00603062B01BF174AAB
:1035C000136803F1FF33136030B9637C23F0070302
:1035D00043F001036374D8E711280BD10F4A136835
:1035E00001331360637C23F0060343F00403637428
:1035F0000020CAE7862809D1084A136801331360FE
:10360000637C23F0060343F00203E3E70728BBD102
:103610000720BAE70520B8E72846B6E7B4CE002071
:103620002DE9FF410546102200216846FBF77AFF8D
:1036300068882979ADF802008DF80410FCF7BCF811
:103640002B78454E092B5ED8DFE803F00505684D61
:103650004D6C7173757D00283FD0437CDC073CD5F1
:10366000FEF7DAFC2B78581E43424341002468469B
:103670008DF800408DF80830FCF790F833684BB3B4
:10368000364E002537464FF0140808FB05735B7C67
:103690005A0703D49B0759D5002C57D0B1783088EE
:1036A000FFF75CFF002851D014235D437B19862867
:1036B0009B788DF804307A5B16BF029008230923AB
:1036C0006846ADF802200CBF8DF800308DF8003050
:1036D000FCF764F804B0BDE8F08101238DF80030F8
:1036E000AB68029316E080B18268AB689A420CD155
:1036F000437CD90709D5326823F00503013243F032
:103700000403326043740024B8E702238DF80030CC
:10371000EB6803936846FCF741F8F4E703238DF860
:103720000030F7E704238DF80030EB68D9E7052374
:10373000F5E70623F7E7072368468DF800300124F4
:10374000FCF72CF89AE7EB680293DCE70135082DCB
:1037500006F1140699D1BDE7B4CE0020FCD10020BB
:1037600070B500238CB02D492C4E4FF6FF70CDE97B
:103770000033FCF7D5F84FF6FF750446AC420BD08A
:10378000A4F58043ADF8143002AA6B46002105A8C9
:10379000FEF77AFE0A2822D0214B1A781846E2B9A1
:1037A0004FF6FF718C4218D01E4E367801251D70E1
:1037B000B607A4F580439BB21DD58B422CD00521C2
:1037C0008DF8141005A811468DF81850ADF81A3070
:1037D000FEF712FE60B1FFF79BF90CB070BD2046FA
:1037E000FEF754FC20463146FCF79AF80446C5E73C
:1037F0000D4B1D70F1E702230022092102708DF8A4
:10380000141005A8FF21ADF816408DF81810CDE969
:103810000723FFF705FFE0E70423EDE7D8D00020FA
:1038200071D0002021CD002072D00020F0B5426878
:1038300005783D4C85B0B2FA82F149090391691EC1
:103840000346042924D8DFE801F0030330496A0065
:103850009989DE8901F5804189B243F6FE77B94244
:1038600004D906F5804080B2B84211D8012DADF8D8
:1038700002108DF8046013D1002A14BF0321002127
:103880008DF8001003929B6802936846FFF7C8FE0C
:1038900023781BB100232370FFF762FF05B0F0BD52
:1038A000002A14BF04210121EAE79989DD8901F585
:1038B000804189B243F6FE76B14204D905F58040D5
:1038C00080B2B042E4D8002A0CBF02220522ADF833
:1038D00002108DF804508DF80020D4E7988900F587
:1038E000804080B243F6FE718842D1D8DB89002B3C
:1038F000CED1FF23ADF802008DF804305AB906236B
:103900008DF80030FEF7C2FB084A002323701370C5
:10391000FFF726FFB9E707238DF80030F4E7082307
:103920008DF80030B1E700BF72D0002071D00020C8
:10393000F8B50D490D4DFBF7F3FF4FF6FF76044642
:10394000A5F12007B44201D12046F8BDFF2CFBD8D9
:1039500021462846FBF770FF0028F5D0204639465F
:10396000FBF7DEFF0446EDE7B8D00020D8D00020FA
:1039700073B5104B104C93E803006D46002385E8A7
:1039800003001A4629462088FFF756F94FF6FF76BE
:103990002388B34201D0112801D102B070BD18466E
:1039A000FFF7C6FF00231A4629462080FFF744F997
:1039B000EEE700BF58BE0500FCCC00201FB5037821
:1039C000012B044615D10179012912D1002302AA45
:1039D0004088FFF785FC60B902238DF800306388CA
:1039E000ADF80230039B68461B788DF8043000F078
:1039F000B5FD054B1A884FF6FF739A4201D0FFF7C9
:103A0000B7FF04B010BD00BFFCCC002070B5044669
:103A10008AB0142200216846FBF784FD6588ADF862
:103A200004502846FBF788FE2378ADF80200092BE6
:103A300015D8DFE803F005163048525E8614A1A5BC
:103A400007238DF8003023798DF808309DF80A306F
:103A500043F001038DF80A306846FBF7D3FE0AB045
:103A600070BD07238DF8003023798DF808309DF85C
:103A70000A30444AA168039143F001038DF80A30EB
:103A80001368002BE8D09942E6D1002313603E4A28
:103A900003931580E0E708238DF8003023798DF833
:103AA0000830E3680493374BA1681A680391002A31
:103AB000D2D09142D0D1354900221A600B680392CE
:103AC000013B0B60C8E707238DF8003023798DF8A0
:103AD000083001238DF80930BEE708238DF8003047
:103AE00023798DF8083001238DF80930A3680493F9
:103AF000B2E7274D09238DF800302B78002BABD08F
:103B00004FF6FF70FFF714FF4FF6FF73984206461B
:103B1000A2D12049FBF704FFB04204469CD11422F5
:103B200000210DEB02002970FBF7FCFC0B238DF844
:103B30001430ADF81840ADF8164005A8FBF762FE4A
:103B40008AE70A238DF80030114BA4681A78029492
:103B5000002A81D0142200210DEB02001970FBF71E
:103B6000E1FC0C238DF814304FF6FF73ADF81830DC
:103B7000ADF816300794E0E705238DF800306BE7C9
:103B80000623FAE7B4D00020A8CE0020F8CC00200D
:103B9000FECC0020D8D000202DE9F047474B1B7801
:103BA0008AB00546002B00F08780454B454F93E8CF
:103BB00003003C7803AE86E80300BCB94FF6FF7003
:103BC000FFF7B6FE0123ADF8143001AB06930423D2
:103BD000029305AA02AB062180460194ADF8164077
:103BE000FFF77EFB07284AD101233B70364B1C6848
:103BF0009846002C5AD1354A354F12883B68AA4264
:103C000041D1002B3FD0142221460DEB0200FBF7DF
:103C100089FC072328468DF81430FBF78DFD062319
:103C2000ADF8160005A8ADF818508DF81C30FBF75C
:103C3000E9FD20460AB0BDE8F087CDF804A0019B5D
:103C40004046A34224BFC1461C46FFF771FEBDF8A3
:103C500014309B00029305AA02AB06218046FFF7B1
:103C60003FFB0028EBD00528E7D04FF6FF739845BF
:103C70001CD1164BA3F80090154B1C60B4E74FF60F
:103C8000FF79A246EDE701333B6000220E4B31463F
:103C90002846FEF7D1FF0028CCD00023C8F800301A
:103CA0003B68112803F1FF333B6001D11120C1E7CC
:103CB000862818BF0320BDE70820BBE7B0CE002050
:103CC00060BE0500B3D00020B4D00020A8CE0020F4
:103CD000F8CC002063DF7047A6DF7047A2DF704793
:103CE0002DE9F04391B0984611238DF804301378F4
:103CF0008DF805300024164601254FF0000365F3CA
:103D00004203074689461C22214609A88DF8063041
:103D1000FBF708FCB3788DF80930C3F30302A24225
:103D200014BF1A2212228DF8242001AA0E9203AB8E
:103D300072788DF808200493224602AB65F34202A4
:103D4000059308238DF80A20CDE9064404AAADF8AE
:103D50001C3009A9434638888DF80E50ADF80C90F8
:103D60000894FFF7BBFF11B0BDE8F083A0DF7047F8
:103D7000044A0123116883400B401ABF1218507E79
:103D800018467047A4CA002070B4094D1346012696
:103D90002A6806FA01F4144207D001F11904024618
:103DA0003146281970BCFDF763BD70BC704700BF79
:103DB000A4CA00201FB50023CDE9013303938DF879
:103DC0000A201A46074BADF8081006241978ADF8FA
:103DD00006008DF80440FFF7D7FF01A8FFF709FAA6
:103DE00004B010BDAF2C002010B4084A01231468A1
:103DF0008B40234006D00A445DF8044B0146507EB8
:103E0000FDF7A6BC18465DF8044B7047A4CA002015
:103E100010B50A4B19780446FFF7E6FF58B1084B76
:103E200000205A88A24201D1C0B210BD013008283A
:103E300003F10C03F5D1FF20F7E700BF8CCC002085
:103E40008ECC00202DE9F8430546FBF775FC234B8B
:103E5000074600221420984600FB02F1CC5AAC42DF
:103E60002AD10B44002634464FF014095BB19978EF
:103E70002846FEF7EDF810B1052818BF03240136D7
:103E80003246072A1DD9A4B9FF2D24D81449284643
:103E90004FF6FF75FFF794F9FFF762FCAF4208D0C9
:103EA0003846FFF7B5FFFF2803D00C2343430D4AE4
:103EB000D5522046BDE8F8830132082ACCD1002330
:103EC000D0E709FB02F338F80310A94201D14344BB
:103ED000CCE70132D5E70724EBE700BFFCD1002097
:103EE000D8D000208ECC00202DE9F0411F46154B84
:103EF0009DF818400E46904619780546FFF744FF96
:103F0000B8F1000F17D0104B3A4619782846FFF742
:103F10003BFF0E4B224619782846FFF735FF44B188
:103F20002846FFF775FFFF2803D00C234343084AB8
:103F3000D652BDE8F081002CFBD03046BDE8F04100
:103F4000FFF780BFAF2C0020B12C0020B02C002048
:103F50008ECC002008B5FFF75BFFFF281DBF0C23A8
:103F60004343034A4FF6FF7018BFD05A08BD00BF45
:103F70008ECC00202DE9F04385B00546FFF7EAFF1F
:103F80004FF6FF739842074641D001224FF00309D4
:103F900001AB0821384602F10108FEF7F3F81FFAD9
:103FA00088F8064648BB02990A46032342F8049B58
:103FB00006312846FBF7B4FB044660B908213846B1
:103FC000FFF7CCFA0446112C3FD01AD80CB30C2CB6
:103FD0002FD107231EE00C280DD0052800D1344630
:103FE00008213846FEF734F8002818BF032442465B
:103FF000002ECDD1E7E70126F2E70728E9D00446F5
:10400000E1E7862C13D043F202039C4211D1002237
:104010001CE0012328468DF80430ADF80850FFF766
:1040200099FFADF8060001A8FFF7C8F8EFE70823ED
:10403000F0E7092328468DF80430FFF78BFFADF831
:104040000850ADF806000394EDE70122034B284623
:104050001978FFF799FE05B0BDE8F0831ECD00206A
:104060000378072B02D14088FFF784BF7047000018
:104070002DE9F0434FF6FF75A84285B0044668D09D
:10408000FFF768FFA84227D100260327B0464FF06C
:1040900001093B46324641462046FBF743FB0428D4
:1040A00005464DD0082847D00B282DD117F0020324
:1040B0001FD1B8F1000F20D11EBB032320468DF87D
:1040C0000430FFF747FFADF80840ADF8060001A83F
:1040D000FFF774F8002237E0002301AA0821FFF758
:1040E000FFF80028D0D1029B03F106089E881F68C4
:1040F000CDE701274FF00009CBE703271E4698467E
:10410000F8E703274646F5E7B9F1000FD5D01128A7
:1041100019D043F202039842DCD008B90223CDE75C
:10412000092320468DF80430FFF714FFADF808404E
:10413000ADF806000395CAE7B9F1000FEED1BCE770
:10414000B9F1000FB9D00122034B20461978FFF7CF
:104150001BFE05B0BDE8F0831DCD002037B5057806
:10416000012D044614D14088FFF782FF6088FFF7D5
:10417000F1FE00236A462946FFF7B2F840B9019BD9
:104180001B782BB1034B608819782A46FFF7FCFD9A
:1041900003B030BD1FCD0020F0B587B004460E46F9
:1041A0001746FFF7D7FE4FF6FF739842054624D017
:1041B0001E4B20461978FFF717FE80B30023CDE988
:1041C0000033029304238DF80030194BADF8024000
:1041D0001978ADF8046020468DF80670FFF704FEEC
:1041E00068B12846FFF72EFE124B204600221978B0
:1041F000FFF7CAFD6846FEF7FCFF07B0F0BD0721D8
:104200002846FDF725FF0528EED10923049003A8D1
:104210008DF80C30ADF80E40FEF7EBFFE4E73A46C0
:1042200031462046FFF7C6FDE7E700BFB12C00206E
:10423000B02C0020AF2C002010B5027886B00446C8
:104240001AB1012A09D006B010BD0E4B1B78002B05
:10425000F9D0C088FFF7F6FDF5E70B4B40881978D9
:10426000FFF792FD1422002101A8FBF75BF960889B
:10427000ADF80600FFF76EFEADF8080001A8FBF7E9
:10428000C1FAE0E7B0CE0020E0CA002070B50446D5
:1042900086B01422002101A8FBF744F92378608836
:1042A000ADF80600013B0B2B00F29080DFE803F035
:1042B0002106233A4E585C68747A7C8C2679444BEC
:1042C000321C19784FF0010518BF01228DF80450F7
:1042D000FFF75AFD731B5A425A413E4B60881978CA
:1042E000FFF752FD6088FFF735FEADF80800002D9E
:1042F00042D106B070BD02238DF804302379002B23
:1043000014BF012302238DF80C30314B01221978A0
:10431000FFF73AFD2F4B227919786088FFF734FDBB
:104320000125DFE703238DF804302A4B1978FFF7C6
:104330005BFD002814BF012302238DF80C30A37904
:104340008DF81030A388ADF80E30E9E7204B1978CE
:10435000FFF74AFD0028CCD102238DF80430DFE7B7
:1043600003238DF80430EAE70723A2888DF8043090
:10437000ADF808208DF80C3001A8FBF743FAB8E738
:1043800008238DF80430A388ADF8083007238DF892
:104390000C30A3680593EFE706238DF804306368BB
:1043A0000393BDE70523D8E703238DF80430094BB9
:1043B0001978FFF719FD002814BF012302238DF897
:1043C0000C3041F20113BEE70423C6E7002589E75C
:1043D00070D00020E0CA00201FB50D294FF0000367
:1043E00001930393ADF80600029108D10B2301A8B5
:1043F0008DF80430FFF74AFF05B05DF804FB86290D
:104400000CBF0A230923F2E730B508490A680023E4
:10441000012505FA03F42242D8B202D122430A60F0
:1044200030BD0133182BF4D11846F9E7A4CA002097
:1044300010B50378182B044602D1FFF7E5FF207072
:1044400010BD000010B5024B197DFDF72FFA10BD0D
:10445000A4CA00202DE9F04F3D4D89B02878FFF720
:1044600087FC60B103A8FFF7EDFFDFF8E8A0DFF8F5
:10447000E8B00DF110090027039B9F4202D309B059
:10448000BDE8F08F39F8024B29782046FFF7ACFCE5
:10449000064678B39AF800102046FFF7A5FC804640
:1044A00040BBBBF800304FF6FF7219462046FBF7C1
:1044B0003BF943F20302904229D10133ABF80030BB
:1044C000EFE7052320468DF80030FFF743FDADF8F8
:1044D00002006846ADF80440FEF770FEB046324672
:1044E00029782046FFF750FC42469AF800102046F3
:1044F000FFF74AFC0137BFE72046FFF72BFDFEF729
:104500004BFE0026EBE72046FFF7B2FDE7E7082861
:10451000F2D012D80028D4D00628EDD0092302907A
:1045200020468DF80030ADF80440FFF713FDADF8DC
:1045300002006846FEF742FED1E743F202039842CA
:10454000CDD043F201439842DDD01128E6D1C6E731
:104550001FCD002020CD0020CCD200201FB5044666
:1045600040882378ADF80600012B10D05AB21AB15A
:10457000022B15D004B010BD01A88DF80420FEF761
:104580001DFE6088FBF7D8F8FFF772FDF2E78DF8A3
:10459000043001A8A388ADF80830FEF70FFEE9E764
:1045A0002379002BE6D0FBF7C7F84FF6FF7398424C
:1045B000E0D0044B01221978FFF7E6FBFFF74AFF32
:1045C000D8E700BF1FCD002038B5074C0146207D3D
:1045D000FDF7BEF830B1A07DFDF7BAF8002814BF92
:1045E0000220012038BD00BFA4CA00202DE9F047F9
:1045F0008CB0894616468046FFF7E6FF20228246A9
:10460000002104A8FAF78EFFBAF1000F46D0B9F1E5
:10461000000F17D099F8005015F001054FF6FF7400
:1046200015D04046FFF796FCA042074639D14048D6
:10463000FDF778FEB0F5807F01D0B84275D1002536
:10464000032470E04D4685264FF6FF775FE02E4647
:1046500027465CE04A4631464046FBF769F8044687
:10466000B9F1000F5DD000285DD199F8003013F04A
:10467000010F14BF012102214046FEF7DBFDB6F118
:10468000850218BF012200240095012339464046C7
:10469000FFF72AFC20460CB0BDE8F08743F2020485
:1046A000F8E7002502AB012207213846FDF76AFD35
:1046B0000446002837D1214650220398FAF732FFEA
:1046C000039B83F800A0039C079604F13403049332
:1046D00004F118030893631C09934046154B0B9390
:1046E000FFF796FBFF280CD0134A0C2101FB00209A
:1046F00050F8042FC4F811208288A4F8152082797C
:10470000E2753846FBF7C0F8044660B90646BAF1D0
:10471000020F04AB9ED1002231464046FBF708F859
:104720000446002CABD00022AEE707460125B9E7CE
:10473000B8D0002073D000208ECC0020F0B585B01A
:104740000446FFF741FF324F012806463D7831D13C
:104750002046FFF7FFFB4FF6FF7398422AD0204612
:1047600032462946FFF710FB0023CDE901330393BE
:1047700001A80C238DF80430ADF80640FFF786FD44
:10478000244B1B78E3B139782046FFF72DFBB8B9ED
:10479000214B22491A682046FFF728FF8628054644
:1047A00032D011280FD070B129462046FFF714FEF1
:1047B00005B0F0BD002229462046FFF7E5FADFE705
:1047C00000221146E7E7A5F111035E425E41002297
:1047D000134B20461978FFF7D7FA124B3246197857
:1047E0002046FFF7D1FA104B002219782046FFF738
:1047F000CBFA0E4B002219782046FFF7C5FA002DA0
:10480000D6D0112DD4D0CFE700260122E0E700BF9B
:10481000AE2C00209FD100205CD000209AD1002037
:10482000AD2C0020AC2C0020AB2C0020AA2C0020AA
:10483000F0B587B0074601A8FFF704FE02AD0024DB
:10484000019B9C4201D307B0F0BD35F8026B39469D
:104850003046FFF7C9FA10B13046FFF76FFF013459
:10486000EEE700002DE9F04F054687B090469946E7
:104870000F4639B9A14B1B78F3B90524204607B080
:10488000BDE8F08FFFF7A0FE0138C0B2012800F2AA
:104890002D8100212846FAF74DFF0446862C00F0B2
:1048A000B080112C00F09980002C00F09680B9F1B6
:1048B000000F00F0BF80B9E0FFF786FE012800F08E
:1048C0009E80022840F012818D490B78284613F013
:1048D00001048B4614BF4FF0010A4FF0020AFFF7A4
:1048E00039FB4FF6FF739842064659463AD03B468D
:1048F00002AA0721FEF7F4FC0446F0B9039B93F8E3
:104900004420D10740F1C780B8F1000F40F0D680B5
:1049100003F1340202F112012846FAF707FF4FF0C3
:10492000000A044600230093BAEB030318BF0123D7
:10493000B4FA84F25209314645E00528F2D1BDE0CF
:1049400004AB012207213046FDF71CFC0446002879
:1049500040F0C1803046FAF797FF0446002800F087
:10496000B280B8E0002C41D06648FDF7DBFCB0F522
:10497000807F834637D0B04236D004AB0122072176
:10498000FDF700FC044650B95846FAF77DFF04468F
:1049900028B95B492846FAF7CDFE044638B107210D
:1049A0005846FDF755FB10B1052818BF03244FF6F4
:1049B000FF73BBEB030318BF0123B4FA84F2009327
:1049C0005209012359462846FFF78EFA002C7FF43E
:1049D00065AF51462846FEF72DFCA4F111035E4257
:1049E0005E4100220FE0B3460324E0E72846FAF7D1
:1049F000A1FE009704460123B0FA80F29AE74049ED
:104A000048E700260122404B28461978FFF7BCF9F9
:104A10003E4B324619782846FFF7B6F9B9F1000F38
:104A200008D0002C3FF42AAF112C17D0214628467D
:104A3000FFF7D2FC0D2C3FF421AF06D8002C3FF439
:104A40001DAF082C18BF032418E7862C14D043F29E
:104A500002039C423FF412AF112C1AD12C4B3A4660
:104A600019782846FFF790F92A4B424619782846CC
:104A7000FFF78AF9002401E7254B3A4619782846C2
:104A8000FFF782F9234B424619782846FFF77CF955
:104A9000F4E60324F2E6B8F1000F0FD1598D03F1CB
:104AA000180200297FF436AF03F12C01343311F8DA
:104AB000010B00287FF42EAF8B42F8D19BF8003019
:104AC000DA073FF53DAF0E492846FAF733FE0446B4
:104AD00000283FF427AF07213046FDF7B9FA002838
:104AE0003FF420AF052818BF03241BE743F202045C
:104AF000B9F1000F3FF4C2AE98E700BF9FD100208C
:104B00009AD10020B8D00020AB2C0020AA2C002085
:104B1000A92C0020A82C00202DE9F04786B00746DC
:104B2000FFF726F958B101A8FFF78CFCDFF84880A1
:104B3000DFF8489002AE0025019B9D4202D306B0EB
:104B4000BDE8F08736F8024B39462046FFF74CF9AE
:104B500080B198F800102046FFF746F999F8001048
:104B600082462046FFF740F901230146524620467F
:104B7000FFF778FE0135DFE7A82C0020A92C0020E4
:104B800010B50378062B0ED9072B1BD10E4B1C78C2
:104B90002046FFF7EDF810B12046FFF749FE0B4B1A
:104BA0001878FFF7B9FF0A4B1C782046FFF7E0F8AA
:104BB00010B12046FFF73CFE064BBDE810401878C8
:104BC000FFF7AABF10BD00BFAD2C0020AB2C00200A
:104BD000AC2C0020AA2C00201FB503780446092B1A
:104BE00009D8DFE803F0050A20202020202020201B
:104BF0004088FFF7A3FD04B010BD144B197819B31A
:104C0000134B00791B7803F00102904206D86179BA
:104C1000C3F34003994294BF0021012101230022E4
:104C20006088FFF71FFE23788DF80430043434F8D1
:104C3000023CADF8063094E8030004AB03E903003E
:104C400001A8FFF723FBD6E70121E7E79FD100206A
:104C50009AD1002037B5174B174A5B881188174C3B
:104C6000174D994208D852889A4205D36369FBB917
:104C700000232B7003B030BD2B783BB16369002B50
:104C8000F6D000228DF8042001A80FE00D490E484F
:104C90000978D4E9012300290CBF11461946FDF714
:104CA00009FA0028E4D0A369002BE1D09847DFE798
:104CB0000122E7E7EECC0020F8D0002050CC002005
:104CC000E4CB0020C8D100206CCC00207BDF7047F3
:104CD0007ADF704776DF704775DF704737B5164B60
:104CE00018884FF6FF73984210D0144A144D137869
:104CF000297B0133DBB2994213702C4608D311494A
:104D0000FFF7EAFF10B1AB6903B1984703B030BDBC
:104D1000002313702B7C33B13B21FFF7DBFF10B175
:104D2000AB6903B198476369002BEFD000228DF87F
:104D3000042001A8E9E700BF4CCC0020C8D1002026
:104D400050CC0020F8D0002065DF70472DE9F74FE8
:104D50000C9CBDF834B02788002580468A469146D1
:104D60002E46B8F80020B2420BDC35B12288013A59
:104D7000D21B92B2FF2A39D8DA55002003B0BDE821
:104D8000F08FD8F8042052F82600019000220DF18F
:104D9000030101A8FFF7D8FF0028EFD19DF80320F9
:104DA0004A4521D12288002D14BF0020022002EBA9
:104DB00009010144594519DC3DB9013292B2228002
:104DC00003F802A022880132228022880DF103011B
:104DD0001A4401A8FFF7B8FF0028CFD121889DF819
:104DE00003200A44228001250136BAE70C20C5E7DA
:104DF0002DE9F341089CBDF824501746CDE9004544
:104E000002220646FFF7A2FF48B910223946304673
:104E1000CDE9084502B0BDE8F041FFF797BF02B009
:104E2000BDE8F0812DE9F04F00231688138090F83B
:104E30002D3085B007460D4614465BB3082E01D8C9
:104E40000C2008E102A8FAF7F5FC002840F00381E5
:104E500013880822CA54238801339BB21B22238063
:104E6000CA54238801339BB2CA18DDF80910238085
:104E7000E950BDF80D30938023889DF80820063353
:104E80009BB212F0FE0218BF01222380EA5423884D
:104E900001332380BB78FBB123880433B342CFD8DE
:104EA00002A8FAF7C5FC002840F0D5802388032229
:104EB000EA54238801339BB219222380EA542388C1
:104EC000BDF8082001339BB2E9182380EA54120A86
:104ED0004A70238802332380FA789AB12388D91C38
:104EE000B142ADD80221E954238801339BB201219C
:104EF0002380E95423880B449BB22380EA542388FF
:104F00000B4423807A68AAB12388D91CB14297D870
:104F1000022192F90020E954238801339BB20A212F
:104F20002380E954238801339BB22380EA542388E9
:104F3000013323803B89002B40F081803B8A53B1B1
:104F4000CDE900462B460722032107F11000FFF7A9
:104F50004FFF00287FD13B8B53B1CDE900462B4654
:104F60001522142107F11800FFF742FF002872D123
:104F70003A6A002A72D1D7F82480B8F1000F30D0F5
:104F8000B8F804302188981C8A1C0244B2423FF6CB
:104F900057AFFE283FF654AF03336B5423880133D9
:104FA0009BB2FF222380EA54238801339BB22380E3
:104FB000B8F80020EA54E918120A4A702088023032
:104FC00080B22080B8F804205AB1D8F8081000291F
:104FD0004ED0284436F0D6FE2388B8F80420134477
:104FE000238097F82C30002B7DD1387898B33B88FC
:104FF000012B3DD0228802F1020CB4453FF620AFD0
:10500000012805D17B78023313449E42FFF418AF88
:10501000023EB61AB6B202A905EB0C00ADF8086064
:10502000FAF704FCB8B93B78022B40F09F80BDF83A
:105030000830B34240F2B580ADF808609FE0CDE99A
:1050400000462B460622022107F10800FFF7D0FE9A
:1050500000283FF473AF05B0BDE8F08FB4F800C08E
:105060000CF10603B3423FF6EBAE1188052901D8D7
:105070000720F0E76FF4486E01EB0E039BB24FF28E
:105080007D3E7345F4D95388052BF1D96FF4486000
:10509000181880B27045EBD94FF6FF70814203D0EB
:1050A000834201D09942E3D8052305F80C302388C8
:1050B00001339BB212212380E954238801339BB230
:1050C00023801188E954E818090A417023880233C3
:1050D0009BB223805288EA54E918120A4A70238846
:1050E0000233238047E7BB6A002BC1D04FF0000991
:1050F0004FF00C0A4FF0160B97F82C305FFA89F23C
:1051000093427FF672AFB96A0AFB02F201EB020822
:10511000B8F80430981CFE283FF692AE208803337E
:105120002B54238801339BB2238005F803B02388D6
:1051300001339BB223808A5AEA54E918120A4A7052
:105140002088023080B22080B8F804205AB1D8F804
:10515000081000298CD0284436F014FE2388B8F8B3
:1051600004201344238009F10109C5E7012B7FF4D2
:1051700063AF7B789E42FFF45FAFADF80830082143
:10518000BDF80830FE2B3FF65BAE22880133AB54EE
:105190002288013292B22280A954228813442380AB
:1051A00059E70921ECE700002DE9F0430646B2F883
:1051B000009007460D4690460FCE9FB06C460FC438
:1051C0000FCE0FC40FCE0FC496E8070084E8070087
:1051D0003C2200210DEB0200CDE90C118DF82E10C0
:1051E0008DF82D1000910E91FAF79CF93C2269463A
:1051F0000DEB020036F0B8FD002840F0C9807C6B52
:10520000002C34D1BB6B23B104F12400002D3ED11E
:1052100084B23B6B23B104F11201002D62D18CB238
:1052200097F82E30002B00F0A980E11C002D7CD1D6
:105230008CB297F82D300BB10934A4B2BB780BB106
:105240000434A4B2FB780BB10334A4B2387800283C
:1052500000F08F80012840F094807B78ADF83C30DE
:105260000020BDF83C3002331C44A4B281E065B19B
:10527000B9F1020F03D80C201FB0BDE8F083022261
:1052800023782A7011226A70AB700324BAE748456C
:10529000F1D811222A55621C92B22221A954A21CD3
:1052A00003F1170115FA82F203F1270C0E4651F8AB
:1052B00004EB42F804EB6145F9D104F1120292B219
:1052C0001121A95404F1130292B223211434A954D8
:1052D000073315FA84F453F8042B44F8042BB34233
:1052E000F9D195E74945C6D811222A55621C92B2D8
:1052F0001020A854274A1668023415FA84F456B1CF
:10530000107992F805C0844540D900F1010C82F86B
:1053100004C046F820405A1E013C0F3312F8010F1A
:1053200004F8010F9342F9D179E74945A3D8601CED
:10533000022280B22A551C261444013B2E54A4B2EA
:10534000032B25D8DFE803F00205071800232B55AF
:1053500002E00123FBE72A558CB2A9EB04092919C5
:105360000FAA3846ADF83C90FFF75CFDBDF83C3025
:105370001C44A8F800407FE70323E8E7002DECD1A8
:1053800057E70FA90020FAF751FA6AE7042073E7FC
:10539000072071E7C0D10020F0B590F82D3085B01E
:1053A0000C461546002B44D190F82E30002B40D1EE
:1053B000436B002B3DD0C3780BB15B0739D584B369
:1053C0002B68072B33D9083BB3F5803F28BF4FF636
:1053D000FF7304F10806ADF806300DF10602314600
:1053E000FFF7E2FE0346F8B9BDF80620083292B294
:1053F000ACB1110AA71C6170F11B89B2052902909A
:105400002270CDF80B0012D902A8FAF713FA50B99E
:10541000DDF80910C4F80210BDF80D10E1802A6013
:1054200002E02646D9E70346184605B0F0BD04233E
:10543000FAE70723F8E713B590F82D301446CBB1FF
:1054400090F82E30B3B1436BA3B9C3780BB15B07AF
:1054500010D52368B3F5803F28BF4FF6FF730DF1D9
:105460000602ADF80630FFF79FFEBDF80630236058
:1054700002B010BD0720FBE707B5144B1A686AB1EC
:10548000002018601B6800934FF08042009B0123AE
:10549000C2F808330E4A5370FAF75CFA0D4B1A68DB
:1054A0008AB100221A601B680193019B4FF0804370
:1054B0000222C3F80823064B0120987003B05DF860
:1054C00004EBFAF747BA03B05DF804FB00010040B3
:1054D00030CC0020040100400E4BD3F8183182B0CC
:1054E000B3B10D4B0D4800221A601B680193019B5C
:1054F0000B4B997EFF291FBF01228A404FF0A0412C
:10550000C1F8082500225A761A711B6802B01847A4
:1055100002B070470030004018310040A8CB002096
:10552000A4CB002070B52D4C86B094F821300193A7
:1055300094F820300093E36904F1260204F123017A
:105540004FF04020FAF724FA2346E0B994F823609C
:10555000A56906BB217B8A1E012A1CD8E069226945
:10556000904218D16269E37BE261C5F340150329DB
:1055700084F8203084F8215007D100954FF0402165
:105580002046FAF7DCFA06B070BD4FF04021204605
:10559000FAF778FAF7E7124A07CA06AC04E90700F7
:1055A000C6B14FF04021D1F8C424C1F8C4249007FB
:1055B0000CD501228DF80820002283F824206A07E8
:1055C000E1D4D3E9002102A89047DCE75107F3D5E5
:1055D0000222EFE78DF80860EEE700BF7CCB0020E9
:1055E00088CB0020F7B515464FF0FF32C1F80823ED
:1055F00090F8242004460F4602F0FF0E2AB183687B
:10560000C1F80433112003B0F0BD012680F82460F6
:10561000836100F10C0C95E807008CE80700AA787C
:1056200084F820206A68E2616A78C7F888252A78B9
:10563000B24212D012B91E1C18BF012684F8216094
:105640000096AB786A6839462046FAF778FA2368FC
:10565000002BD8D184F82430D5E784F821E0AB784A
:105660006A6839462046FAF70DFAF0E730B54A4A3B
:10567000D2F8043313F4007F85B015464AD0D2F82F
:105680002431002B46D04FF492711046FAF7C2FA3B
:105690004FF40173C2F80833404B997E09B90121D8
:1056A00051603D4902228DF80020D1F88024C1F8D4
:1056B00080240392DA7D8DF80820DA6801920022B6
:1056C000DA751A766846D3E9001290473248D0F866
:1056D0001C313BB1314A938A917D994247D9114699
:1056E000FAF7C7FA2C4AD2F844318BB14FF4A271C1
:1056F0001046FAF78FFA294B997E09B10121116002
:10570000DA7D2AB10022DA75587ED968F9F732FFBE
:1057100005B030BDD5F804335B07D7D5D5F80831CF
:10572000002BD3D01D4C1C482146FAF78BFA637E20
:10573000E27D9A422346C9D1227E52B12369E168B3
:10574000E3600023607EE27523766376F9F712FF4B
:10575000BCE7A27E0AB901226A600F4A4FF40171C8
:10576000C2F808130022DA75587ED968EEE74FF4C4
:105770008E71FAF74FFA917D0029B3D000238DF88E
:10578000081091688DF80030019193756846D2E950
:1057900000139847A6E700BF0020004060CB002020
:1057A000800000F1A040D0F8003723F44033C0F867
:1057B0000037D0F8003743EA0141C0F800177047BE
:1057C0000E4B034493F94020072A02DD0021FFF726
:1057D000E7BFD3B2072B10D8930003F1804303F542
:1057E000C043D3F8101521F00101C3F810150123AF
:1057F00003FA02F2024BC3F808237047F4CA0020F0
:105800000060004000F1804000F5C040002382B0FD
:10581000036003680193019B02B070472DE9F04FCC
:1058200085B00024594D01944FF48072012102F19A
:10583000804303F5C04390B21B68012B06D1D5F815
:1058400004330B4202D0FFF7DDFF0C430432B2F504
:10585000907F4FEA4101EAD14D4B1B68012B0AD1E1
:105860004FF4BE70FFF7CEFF4FF0A04344F000446A
:10587000D3F81035019314F0FF0F1AD0454F0126CD
:105880000025344210D0AB0003F1804303F5C04340
:10589000D3F81005D3F8101557F8253023B1C1F30C
:1058A0000141C0F3042098470135082D4FEA460610
:1058B000E7D1002C63DA4FF0FF330022CDE902324A
:1058C000344D354E0024A24601274FF0A04816F96A
:1058D000012B531C46D0D2B222F0C0094FEAD901A5
:1058E00004A8084402F0070310F808CC07FA03F3F1
:1058F0001CEA030F36D005EB090C92099CF940C055
:1059000055F82CB0BBF1000F0AD1032A2AD10DF1B2
:105910000C0E1EF801C04CEA030C0EF801C001E0A9
:10592000032AF4D009F5E07110F80C0C58F8211096
:105930001842C1F3014105D0022913D1032A0BD12A
:10594000114604E003290DD1032A05D1022148465E
:10595000FFF726FF0134E4B2BBF1000F02D011467D
:105960004846D8470AF1010ABAF1080FAFD134B15D
:105970004FF0A043019AD3F81035934202D105B0FD
:10598000BDE8F08F0193039B02939AE7006000400B
:105990007C610040F4CA002054CB00200028C3B230
:1059A000A8BF00F160424FEA501010B5BABF0D4ACF
:1059B00003F00F0402F561424FEA41114FEA800003
:1059C000C9B200F16040B4BF115582F8001300F570
:1059D000614003F01F0201239340C0F8803103604F
:1059E00010BD00BF14ED00E02DE9F8430568EB178A
:1059F0005906674B41EAD51104464FF0FF3268065D
:105A00008B4208BF82420AD3624A002335F0EEFF80
:105A100000F5006020F47F6727F00F072FB92946B3
:105A20005D48BDE8F84329F01DB9207924F022FD36
:105A300040B9607924F01EFD20B95848BDE8F8430C
:105A400029F010B9E279E17A0D2024F0A3FD237B3F
:105A5000534A002B00F08A80537843F01003514ED4
:105A60005370F3781BB10023F370FAF7FBFD25792F
:105A700000232846F37024F0FDFC20B14FF4407160
:105A800028461BF0CFFE6579284624F0F3FC20B1B0
:105A90004FF4985128461BF0C5FE637A2579002BF8
:105AA000284614BF4FF00E094FF0000924F0E2FC25
:105AB00000285FD03C4B05EB85051D4495F801801F
:105AC0006479204624F0D6FC002856D0364B04EBEF
:105AD00084041C446378354CE27E002A50D15A1C61
:105AE0000AD04FF0A04101229A40C1F8082503F5E1
:105AF000E072032041F82200B8F1FF3F2C4D1FBF98
:105B00004FF0A04108F5E072002041F82200C5F8EE
:105B10002475C5F86C950027C5F81485C5F80C35B3
:105B2000244B636028464FF48E712760FAF772F8B1
:105B30004FF4A271FAF76EF81F4BC5F80433022137
:105B40000846FFF72BFF0423C5F80035B8F1FF3FE7
:105B50004FF48073E7822776638315D01748FAF7EE
:105B600061F80123A376FBF781FA0DE0537803F087
:105B7000EF0374E74FF0FF38A2E74FF0FF33AAE7D7
:105B800008210F4829F04EF80123F370BDE8F8838F
:105B900047E8010048E80100A6BF0500BBBF0500BB
:105BA0009CCA0020D9D2002040C0050060CB002054
:105BB0000020004045A103008000020080BE0500D7
:105BC000D1BF050010B50D4C00226260A2602261B9
:105BD000E2600B4A106810F0010002D10621FFF7C5
:105BE000DDFE084B1B7823B94FF080430122C3F838
:105BF000182501232370002010BD00BF30CC0020E9
:105C000000E100E0A1D10020F8B50E46D11C48BF4C
:105C1000911D144641F387010546671EFAF7E8F81F
:105C200000214AB2A24201F1010100DBF8BDBB1A1A
:105C300023F00300B25C03F00303DB0002FA03F37A
:105C40002A581A432A50ECE7F0B500254F1E6CB2D3
:105C50008C4205F1010500DBF0BD3B1B23F0030680
:105C600003F003039659DB0026FA03F30355EEE72E
:105C70002DE9F041B3F9024014F11F0548BF04F1CA
:105C80003E050F4603F1240645F3471590460146AD
:105C90002B4632463846FAF7EBF8B8B9B4EB451F55
:105CA00016DA6211012304F01F0403FA04F457F812
:105CB00022301C4214BF012400242B4632463946B0
:105CC0004046FAF7D5F82046BDE8F0810124F4E714
:105CD0000446F2E710B500231A465CB2A14203DC89
:105CE000B2FA82F0400910BD50F82340013322433C
:105CF000F3E700002DE9F04F8A46234F8BB00646AC
:105D0000114650461446FAF753F83B68FBB1042598
:105D1000C0EB441014FB05FB00B205FB04654FF01B
:105D2000FF38043D28FA00F84FF040093B68594617
:105D30003046984758B12B6803EA08032B60214688
:105D40003046FFF7C7FF20B1B9F10109EED10020BD
:105D500017E023463246514602A8FAF759F8214681
:105D6000019002A8FFF7B6FF019B003318BF012383
:105D70005B00002814BF5842C3F10100C0B20128E3
:105D8000E2D10BB0BDE8F08F602E00202DE9F04F7E
:105D9000D1B0CDE905015B9D95F9004048A8914639
:105DA00022461F46F9F7F8FFA3000793069BA200BF
:105DB00013441946224638A80293F9F7EDFF95F9E6
:105DC0000060002F00F08C803246394628A8F9F791
:105DD000E3FF0DF5807A324630AF48A95046F9F717
:105DE000DBFF38A93846F9F7D7FF2B4628AA38A990
:105DF00048A8F9F790FF2B4628AA38A948A8D5F853
:105E0000A460B0472B4628AA39465046F9F783FFCD
:105E1000BDF968310497023B1BB2002B67DCD9F84F
:105E20000030009503F001084FEA481840AADB4310
:105E300002EB080A03F0010330AA90445B0140AA78
:105E40001A44039230AAD3184146039A0493504649
:105E500005F10409FAF703FA4B4640AA48A908A835
:105E60000094FAF76CF908A908462B464246F9F760
:105E700011FF08A908462B46069AF9F70BFF2146A1
:105E800008A8FFF727FF00285DD008A8F9F7B0FFA2
:105E900008A92B46029A0846F9F7FCFE08A92B46EA
:105EA00052460846F9F7F6FEDDE90301434652463D
:105EB0000095FAF756F92B4608AA30A940A8F9F739
:105EC0002AFF224640A90598F9F766FF059B079C23
:105ED000234430A91846F9F75FFF51B0BDE8F08FB1
:105EE000314628A8F9F784FF0123289371E71FFAA8
:105EF00083F85B1108F01F0259F823300095012147
:105F000001FA02F21A42049B13BF20270027202621
:105F100000260AEB070B1F440AEB06030393049BBE
:105F2000039A1E44334639465846FAF798F908F161
:105F3000FF383B4600955A4631460398FAF711F967
:105F40000FFA88F369E710AF224608A938460DF129
:105F5000600BF9F721FF20AE49465846F9F71CFFC0
:105F600030462146F9F744FF012328A82093F9F78A
:105F70003FFF224659463846F9F7F9FE28B922462E
:105F800020A908A8F9F708FF82E73B68DA0709D4D7
:105F900021463846F9F7DEFE224649463046FAF7F2
:105FA000B2F8E6E7189BDB0707D421465846F9F715
:105FB000D1FE2246494628A8F1E7002823461CDDE9
:105FC0005A4639463846F9F723FF21463846F9F74D
:105FD000C1FE224628A93046F9F7C9FE002805DA95
:105FE00023464A4631463046F9F742FF234628AA5F
:105FF00031463046F9F70CFFCEE73A465946584647
:10600000F9F706FF21465846F9F7A4FE2246314625
:1060100028A8F9F7ACFE002805DA28A923464A4645
:106020000846F9F725FF28A9234632460846F9F71E
:10603000EFFEBEE72DE9F04793F9006092B0044609
:1060400089461046314615469846FFF743FE00281C
:1060500040F09180424649460AA8F9F758FE434667
:106060000AAA214602A8F9F715FE0AA908464246DF
:10607000F9F74DFE43462A4649464846F9F70AFED7
:1060800008F10407424629462846F9F740FE3B46F8
:106090002A46214620460096FAF7C8F83B462A468B
:1060A000294628460096FAF7C1F83B462A4621467B
:1060B00028460096FAF743F843462A4621462046EA
:1060C000F9F7E8FD3B462246214628460096FAF7B6
:1060D000ADF83B4600962A4621462046FAF7A6F838
:1060E0002368DB074AD533463A4621462046F9F76E
:1060F000BFFE314682462046F9F72CFE06F180436A
:10610000013B54F8230040EACA7044F82300424699
:1061100021462846F9F7FBFD3B4602AA29462846B8
:106120000096FAF70CF83B4602AA29462846009644
:10613000FAF705F802A908463B462A460096F9F701
:10614000FEFF434602AA21462046F9F7A3FD0AAA0C
:106150003B46104621460096F9F7F1FF32462946A4
:106160002046F9F719FE49462846F9F715FE0AA90F
:106170004846F9F711FE12B0BDE8F08731462046D7
:10618000F9F7E8FDC3E7000073B500230DF1020045
:106190008DF80230FBF71EF8264B1B7803F0FF0446
:1061A000002B41D1244B1A68002A3DD0234AD2F853
:1061B0000813C90738D51C601B68214D01930DF1E8
:1061C0000300019BD2F808658DF80340FBF702F845
:1061D0006A6829681F2A98BF541CA142F6B26C60F5
:1061E00004D1202C14BF611C0021296015499DF8A1
:1061F00003008E542A6894423ABFC2F12102131957
:10620000A31AAA689A4238BFAB60FBF7B9FE6B6865
:106210002A681F2B94BF013300239A4201BF074A0B
:106220000123C2F8083353609DF80200FBF7A8FE73
:1062300002B070BDA1D1002000D1004000D00040CC
:106240008CD1002068D1002030DF70472DE9F74F56
:106250003B4F06468846B8F1000F03D1012003B03A
:10626000BDE8F08F4546202D28BF20255FFA85FB2D
:10627000002400230DF102008DF80230FAF7AAFF86
:10628000304B1B7803F0FF0993BB0DF103008DF831
:106290000390FAF79FFFD7E900148C4204D3641AE5
:1062A000A54207D9052414E02134641AA542F9D87F
:1062B000C1F12104244BA542194431D82A46304665
:1062C00035F060FD3B682B44212B28BF00233B6049
:1062D00000249DF80300FBF753FE1C4B00221A60BC
:1062E0001B680193019B1A4B0122C3F804231A6017
:1062F0009DF80200FBF744FEB9F1000F08D05946A3
:106300003046FFF7A1FF42F2070398420446ADD0A2
:10631000022CAED0002CA9D1A8EB05082E449AE798
:106320002246304635F02EFD074BA5EB040A5246B7
:106330001946301935F026FDC7F800A0C8E700BFA0
:106340008CD10020A1D1002068D1002000D10040D4
:1063500000D0004017B4314A314B116889B900218F
:10636000304A106820BB00205A79D40740D408B9BD
:10637000002949D01C68DA88234603B05DF8044B35
:106380001847002111601268D9680092009A00290C
:10639000E5D0254AD2F84005814204BFD88801EBF8
:1063A0008001C2F840155A7942F004025A71D7E7C9
:1063B00000201060126898680192019A0028D2D0DB
:1063C000194AD2F83845A04204BFDC8800EB8400AB
:1063D000C2F838055A7942F0020214075A71C3D53F
:1063E00012F0010402BF64F3C3025A712046BBE7F6
:1063F00002F00601062907D122F0060211075A71A0
:1064000006D56FF3C3025A7103B05DF8044B7047B1
:10641000054AD2F83805D2F84015ABE714510240CE
:10642000E4CA00200451024000500240A5DF70473A
:10643000A4DF7047A3DF70472DE9F0470E4690B008
:1064400016F01005814692469846189C0CD01123F0
:106450008DF8083023788DF8093001224FF00003C1
:1064600062F342038DF80A301C22002109A8F9F7D3
:1064700059F88DF8246005B102AD42F64D23ADF810
:106480000C3063789DF864108DF804300022A378F6
:106490008DF80530134661F3C303DBB243F0030309
:1064A000CDE906220E95012701AD8DF80630089240
:1064B00003AE1A9BB9F800008DF80E7004AA09A962
:1064C000CDE90465ADF81CA0FDF708FC58BB42F609
:1064D0000813ADF80C3063788DF80430A3788DF88C
:1064E0000530034667F342038DF806301A9A98F890
:1064F00000308DF8003098F80130CDF81A00ADF872
:106500001E008DF8013032F8080B8DF80E70022352
:1065100004A9CDE90465ADF81830ADF81C30CDF80C
:1065200020D0FFF787FF10B0BDE8F087A1DF7047EC
:10653000BFF34F8F0549064BCA6802F4E06213436C
:10654000CB60BFF34F8F00BFFDE700BF00ED00E061
:106550000400FA0508B5F9F75BFF10B1664B674A0E
:106560001A60F9F735FF28B1654B664A1B68C3F31B
:1065700042331360F9F74CFF20B1634AD36823F02C
:106580008073D360F9F724FF40B14FF080430022BD
:10659000C3F80C21C3F81021C3F83825F9F738FFE8
:1065A00010B15A4B03221A60F9F732FF40B1584B31
:1065B00005221A6001229A6700229A603F225A60DF
:1065C000544B1B78062B50D1534B1B681B074CD1E7
:1065D000524B1B6803F0F003502B46D14FF0805212
:1065E0004F4BD2F80414C3F82015D2F80814C3F89E
:1065F0002415D2F80C14C3F82815D2F81014C3F8D7
:106600002C15D2F81414C3F83015D2F81814C3F8A6
:106610003415D2F81C14C3F84015D2F82014C3F86E
:106620004415D2F82414C3F84815D2F82814C3F836
:106630004C15D2F82C14C3F85015D2F83014C3F806
:106640005415D2F83414C3F86015D2F83814C3F8CE
:106650006415D2F83C14C3F86815D2F84014C3F896
:106660006C15D2F84424C3F87025F9F7B1FE28B1AF
:106670002C4B2D4A1B6803F04F0313602B4AD2F8B2
:10668000883043F47003C2F88830BFF34F8FBFF3F4
:106690006F8F4FF01023D3F80022002A03DBD3F8CA
:1066A0000432002B24DA224B0122C3F80425D3F84C
:1066B0000024002AFBD04FF010221521C2F800124E
:1066C000D3F80024002AFBD04FF010231522C3F882
:1066D0000422174B1A46D3F800140029FBD00021DE
:1066E000C3F80415D2F80034002BFBD0FFF720FFCD
:1066F000104B114A1A6008BD74C007400DF0ADBAC6
:10670000440200103C050040F0ED00E0A005004010
:1067100010560040E00F00F0E40F00F0E80F00F02A
:1067200000C0004058020010E40E004000ED00E000
:1067300000E00140A42C00200090D003002382B090
:10674000036003680193019B02B070472DE9F34198
:10675000844BD3F8042162B3D3F800339F0728D5C4
:10676000814D8248FFF7EAFF2B7803F0FF08F3B969
:106770007F4F804E7B783C4603F0FF02002B00F0F9
:10678000AF8073684046984701A88DF80480FAF7F7
:1067900021FD7B689DF8040001337B60FBF7F0FB73
:1067A000754B0122DA601A60744B00221A600123D3
:1067B0002B706C4BD3F81821D2B1D3F800235606B6
:1067C00016D5D3F824356E48DB08C3F3080113F45B
:1067D000FF7F18BF0239FFF7B1FF624B4FF48052C1
:1067E000C3F808254A1EFE2A40F2A4800122DA617D
:1067F0005C4AD2F81031D3B1D2F80033DD0616D599
:106800006048FFF79BFF1023C2F808335E4BC2F8C5
:106810001035FF23C2F814350123D3615B4B1C688C
:106820002CB15B4800231A4603210068A0474D4A5B
:10683000D2F84C3133B3D2F800331C0322D555487B
:10684000FFF77CFF4E48FFF779FF5348FFF776FFCD
:106850004D4BC2F81035FF23C2F814350123D36124
:106860004FF48863C2F804330D23C2F80C34C2F825
:106870000434464B1C682CB1454800231A4619467F
:106880000068A047374AD2F828315BB1D2F800330C
:10689000580507D54048D2F80C34FFF74FFF0D23B9
:1068A000C2F80C342F4AD2F81C31B3B1D2F80033FD
:1068B000190612D53948D2F80414FFF73FFFCB0769
:1068C00007D5374B197821B10121C2F804140022F1
:1068D0001A70244B0D22C3F8042402B0BDE8F081E5
:1068E0000DF103008DF80320FAF774FCBA68134623
:1068F00083B93260A660636833B92A4B1B7803F012
:10690000FF025BB1F9F73AF863689DF803000133C1
:10691000636043E7B342EED01B68E9E7224B1A609D
:106920001B680193019B4FF080430122C3F80423AD
:106930001A60E9E7144A1078502803D11849012257
:106940000A7054E711480468002C3FF451AF4FF629
:10695000FF70C3F808050E480B4600680221A047E7
:1069600046E700BF005000401CCD0020045100400D
:1069700030CC002044CC002000B001405C2E002030
:106980001851004010510040C0CE0020CCCF002054
:10699000D0CF00204C510040285100401C510040F5
:1069A000A0D10020A1D100200001004013B5284B48
:1069B0002849D3F83C3413F0030345D10A68013267
:1069C000072A0A602CD9244A012414610DF107001A
:1069D0008DF80730FAF7FEFB204B5A68013A5A60EF
:1069E0005A6822B91E4A127802B3F8F7C5FF9DF81B
:1069F0000700FBF7C5FABFF35F8F1A4A0023136045
:106A0000BFF35F8F01211160174A14681CB117484A
:106A10001A460068A047164B00221A70FAF75AFB74
:106A20000D4B0022C3F8402102B010BD114A4FF0B7
:106A300080411460D1F80C2402F00112B2F1011F60
:106A4000F8D000225A70D2E700230B60E8E700BFBD
:106A5000005000405C2E002000B0014030CC0020EF
:106A6000A1D10020FC5F0040CCCF0020D0CF00207F
:106A70001CCD002004000040D0E9012393423FBF19
:106A8000026842F82310836801333ABF8360002014
:106A9000042070472DE9F04F87B00D4693460190D2
:106AA000C8B1C2B103680393ABB14FF00009C84647
:106AB000019B9B68434503D8CBF80090002022E05F
:106AC000B8F1000F09D1012B0CBFC0238023039A1A
:106AD00052F8284044B90E2015E008F10102934213
:106AE0000CBF40230023F2E76178227A571869B976
:106AF000971D002D44D0DBF80020A2EB0902BA421A
:106B0000029205D2042007B0BDE8F08F0737F0E706
:106B10002B702278AA4613430AF8023B227A6A7045
:106B200062783ABBAE1D227AE168304635F02AF928
:106B3000237A62781E442AB13046616835F022F922
:106B400063781E44029BDB1B05932369002BC2D094
:106B500005AA3146606998470028D4D1059B16B133
:106B60001ABACAF800201F44B94405B13D4408F1DF
:106B700001089DE743F00803EE1DAA712B70D2E7D0
:106B8000AA462E46E1E710B5144661B113689BB1E1
:106B90004378027803F00F0343EA021301F8013B44
:106BA0002368013B236022464068FFF773FF10B95A
:106BB00023680133236010BD0420FCE770478DDF9C
:106BC000704777DF7047D0E91F32816F1A44D0F8E1
:106BD0008430C0F880200B4490F82110C0F8843035
:106BE000C9B1016F002ABCBF5218C0F88020D0F88C
:106BF00080208A42A4BF521AC0F88020426F002B26
:106C0000BCBF9B18C0F88430D0F884309342A4BF36
:106C10009B1AC0F884307047D0F88030C0F88830B4
:106C2000D0F88430C0F88C3070470368C91A4368C4
:106C300070B5D21AD0E91E6302FB03F4724301FB64
:106C4000064501FB1322D0F88040D0F884302C4454
:106C50001A44C0F88040C0F8842070BD2DE9F04F80
:106C600089B00E4600AF0023044607F114013046F8
:106C70007B612DF0E5FD05465EB318BB30462BF079
:106C80000DFE8046786126F037FE08F5807383425A
:106C90000CD9A949012028F005F93246A74901205D
:106CA00028F000F92437BD46BDE8F08F08F107034E
:106CB00023F00703ADEB030D6D46424629463046EF
:106CC0002BF010FF7E693EB99D49012028F0EAF8BB
:106CD000E8E70028F6D1E0E74FF00308B6FBF8F349
:106CE00003EB43039E4201D09649EEE7204623F092
:106CF000C1FB08B99449E8E7944BC7F808D004EB06
:106D000084041C446378924C2179002940F00B8163
:106D1000904A0120C2F80415FF2BC2F82415C2F8CE
:106D20002015C2F81C05C2F82815C2F818154FF036
:106D3000C051C2F81415C2F810054FF0A04118BF99
:106D400003F5E070C1F85C87C1F8FC8A18BF41F810
:106D500020804FF01701C2F864154FF0FF01C2F810
:106D6000681508BF4FF0FF334FF0FF31C2F86015D0
:106D70002520C2F87035C2F86C15774B23600221CC
:106D8000FEF70CFE012323710323B6FBF3F39BB242
:106D900003EB430808F1010828F001029100ADEB74
:106DA000010D6846FA606D4A3A6041184FF0000CD8
:106DB000796082F800C0E91C4FF0EE09851C4FF0A5
:106DC000880A4FF08E0B63455FDC0C2202FB030345
:106DD00000227968994200F29E802679012E40F0C7
:106DE000A28000F06043B3F1005F40F0A280FB6836
:106DF000C3F34E02574B0021C3F85025C3F8381592
:106E0000C3F80815C3F84005C3F80C656579E2803E
:106E100025F0090545F008056571C4E90210C3F8BD
:106E20000065022323710D46002977D04FF6FE72CC
:106E300008EA0202F8F776FB494B00221A601B6849
:106E4000FB61FB69474B1A601B68BB61BB69414B27
:106E50002222C3F8042301221A603A681278042A15
:106E6000FBD94149002222250120C3F808530860BC
:106E7000C3F80025C3F808530860C3F800253B4B4E
:106E80002021C3F88410227150E011F8026C11F82F
:106E9000032C360246EA024611F8012C05F10C0ECD
:106EA000164306F44012B2F5001F1ED0B2F5401F83
:106EB00020D0B2F5801F20D105F802BC06F44002B4
:106EC000B2F5000F1CD0B2F5400F1ED0B2F5800F06
:106ED0001ED105F801BC0235AE454FEA0616E0D1D9
:106EE0000CF1010C033175466DE76FF0170205F8E0
:106EF000022CE3E705F8029CE0E705F802ACDDE7C9
:106F00006FF0170205F8012CE5E705F8019CE2E7B0
:106F100005F801ACDFE703F8012B5AE701462368C7
:106F20002846984788E70820FAF7C8FFD7F808D01E
:106F3000B8E61020F8E700BF69D6050090D6050036
:106F4000BCD60500DCD6050007D7050040C005000B
:106F5000E4CA002000500240B18B030038D3002067
:106F600004510240145102400450024000E100E08C
:106F700070B50022104905462EF01EFB2EF064FE6F
:106F80000E4B0F490646032258682EF015FB0446A7
:106F900030B10022B1B22EF052FA20462CF086FF1A
:106FA000084B18682BF0AEFD00210446284614F06B
:106FB000CFF8204670BD00BF06CD0500482E00204A
:106FC00013CD0500F8D2002010B5838AC3F30C045A
:106FD00013F4604301D1204610BDB3F5005F02D128
:106FE00006206043F8E71B0407D500220449006827
:106FF0002EF0E2FA2EF028FEF3E70020ECE700BFC7
:1070000095D4050008B540B2FFF7DBFD40F2EA7108
:10701000BDE8084013F0FEBC38B5054608460C46EE
:107020002CF010F8002808BF002422460F492846FB
:107030002EF07EFA0E4B4FF6FF72198884B18A4209
:1070400006D1002040F63551BDE8384013F0E2BCCF
:1070500000221888114614F0F1F80828F2D1F0E760
:107060008A42EED0188814F0E7F8F6E7EFCC050076
:10707000682D0020014B188813F0E0BC682D00201B
:10708000014B188813F0DABC6A2D002008B5084BB4
:107090001A884FF6FF71914209D018881321FDF725
:1070A00019FE4FF4F171BDE8084013F0B3BC08BD00
:1070B0006A2D002007B50023084607226946009381
:1070C000CDF80330F9F74CFC0A4B1A884FF6FF71E4
:1070D00091420BD018886A46012114F0DBF840F683
:1070E000DF3113F097FC03B05DF804FB43F20200BC
:1070F000F5E700BF682D002038B500220E4905468F
:107100002EF05AFA0446A8B90C4925F0C9FF0A49DD
:107110000446024628462EF00BFA2A460849204625
:107120002EF006FA00202CF0A5FD06490246204666
:107130002EF015FA204638BDA6CC0500ABCC0500D4
:10714000C5CC0500E5CC0500F8B5044628B9244AAD
:10715000136823F480431360F8BD22492DF03CF9F5
:107160000028F4D120462BF093FF0546A0B11C4A1D
:107170001368204643F4804313602FF0EBF853EC80
:10718000102B10EE100A194616F0FEFB40F6E12116
:10719000BDE8F84013F03EBC20462BF038FF002835
:1071A000DAD00F4A1049136843F480431360204635
:1071B0002A462EF001FA2FF0BBFB2A4606460F4660
:1071C00020460A492EF0F8F92FF0B2FB02460B4692
:1071D0003046394616F0D8FB40F6E721D8E700BF25
:1071E000FCD2002083D0050088D0050094D0050093
:1071F000084B1A6818B142F400521A60704722F422
:1072000000521A60044B1860044B01221A7013F0EC
:1072100077B900BFFCD200203CD300203AD3002035
:10722000F0B583B0044600AF28B9014613F0A4F9C5
:107230000C37BD46F0BD2CF0E1F828B120462DF00A
:1072400061FF0421C0B2F1E77860391D20462DF0BE
:10725000F7FA0546F0B920462BF020FB0646786089
:1072600026F04AFB06F58073834208D90D490120B8
:1072700027F018FE0C49012027F014FED8E7F31D73
:1072800023F00703ADEB030D6D4632462946204639
:107290002BF028FC79680029ECD0284613F09EF9E1
:1072A000C6E700BF69D60500ADD8050008B5044B98
:1072B000044958682EF082FDBDE8084013F0C6B9B5
:1072C000482E0020EDD80500F0B583B0044600AF8D
:1072D00013F0BCF9002C60D00023391D20467B60E0
:1072E0002DF0AEFA054610BB20462BF0D7FA064625
:1072F000786026F001FB06F5807383420CD9314992
:10730000012027F0CFFD3049012027F0CBFD0024DC
:1073100020460C37BD46F0BDF31D23F00703ADEB4F
:10732000030D6D463246294620462BF0DBFB78687C
:107330000028E8D02CF06EFB044608B92349E3E7A7
:10734000234B2449024658682EF0F2F820462CF0D0
:10735000ADFD20462BF0C2FE7A68294634F012FDBE
:1073600020462BF0BBFE054620462DF040FA014694
:10737000284613F07BF90023391D0A207B60F9F7BA
:1073800021FD7B680446002BC2D0134A11681960A6
:107390005168596012891A81BAE720462CF03AFBED
:1073A000044620B90949012027F07CFDB0E7084BCD
:1073B0000849024658682EF0BBF820462CF076FDAE
:1073C000CEE700BF69D60500ADD80500C4D80500DA
:1073D000482E0020EDD80500BFCF0020F0B583B0C7
:1073E000054600AF48B9384B384958682EF0E6FCDE
:1073F000FFF75CFF0C37BD46F0BD0023391D7B60F5
:107400002DF01EFA0646F0B928462BF047FA04463E
:10741000786026F071FA04F58073834208D92C490C
:10742000012027F03FFD2B49012027F03BFDE1E73C
:10743000E31D23F00703ADEB030D6E4622463146F4
:1074400028462BF04FFB78680028ECD013302CF046
:10745000E1FA054608B92049E6E71B4B1B490246FD
:1074600058682EF065F828462BF038FE044628466A
:107470002CF01CFD194B224603F1100153F8040BAC
:1074800042F8040B8B42F9D11B8813807D6831468A
:107490002A4604F1120034F075FC65742544FE237D
:1074A000AB740020FFF710FF394605462DF0C8F9F0
:1074B00028B10368236043686360038923812846F9
:1074C0002CF0F4FC96E700BF482E0020A5D805005C
:1074D00069D60500ADD80500C4D80500BECB0500AF
:1074E000F0B5ADF5037D064600AF50B9334B3449D6
:1074F00058682EF063FCFFF7D9FE07F50377BD4609
:10750000F0BD0023391D7B602DF09AF90446F0B9D7
:1075100030462BF0C3F90546786026F0EDF905F505
:107520008073834208D92749012027F0BBFC2649F4
:10753000012027F0B7FCE0E7EB1D23F00703ADEBDC
:10754000030D6C462A46214630462BF0CBFA7B6869
:10755000002BECD04FF400721C4D3A600022AA6060
:107560001B4A1C491460DBB228465360FFF784FABB
:1075700038B9AB6893B13A4607F108012846FFF7DE
:1075800089FA40F6CC0113F045FA0028B5D13868E5
:107590002CF040FA044618B90F49C9E70720F0E774
:1075A0002BF09CFD3A6807F1080134F0EBFB204614
:1075B000FFF714FF20462CF079FC9EE7482E0020B0
:1075C000A5D8050069D605002FD80500842D002018
:1075D000F0D20020142D002046D805002DE9F043FC
:1075E000E1B0054600AF58B95E4B5F4958682EF0D0
:1075F000E5FBFFF75BFE07F5C277BD46BDE8F0830C
:107600000023391D7B602DF01BF90646F0B9284692
:107610002BF044F90446786026F06EF904F5807387
:10762000834208D95149012027F03CFC50490120F0
:1076300027F038FCDFE7E31D23F00703ADEB030D74
:107640006E462246314628462BF04CFA7B68102BBA
:10765000ECD107F108044FF480733C22002120464E
:1076600007F144054FF001083B604FF00209F7F7BE
:1076700059FF40F201433C2200212846BE637B8132
:1076800087F8089087F8358087F83680F7F74AFF43
:107690007E67384E384BBB67736938495B6887F83B
:1076A000468000229A60736987F844905868FFF713
:1076B000E3F900283AD1736931495868FFF7DCF9DA
:1076C000002833D12F4B304A1B781370DFF8D0805D
:1076D0002E4AC8F81440003318BF012388F801303F
:1076E0002B4B2C4C1B78DFF8BC901370003318BF69
:1076F0000123A06031462046C9F8145089F80130B2
:10770000FFF7BAF990B941462046FFF7B5F968B9D5
:1077100049462046FFF7B0F940B91F4B3A4618607A
:10772000988007F180012046FFF7B4F940F69101F7
:1077300013F070F900287FF45EAF38682CF06AF916
:10774000044608B9154972E72BF0C8FC3A6807F1FE
:10775000800134F017FB2046FFF740FE20462CF056
:10776000A5FB48E7482E0020A5D8050069D60500EE
:1077700073D805003C2D00205FD90500E82C0020BF
:10778000BC2C00202F2D00204CD300204DD30020F6
:107790002E2D0020302D0020C0D1002046D805001D
:1077A000902D00206C2D00202DE9F04182B005467F
:1077B00000AF50B94E4B4F4958682EF0FFFAFFF713
:1077C00075FD0837BD46BDE8F0812BF042FD28B9B4
:1077D0002A464949032027F065FBF2E70023391DBB
:1077E00028467B602DF02CF80446F0B928462BF093
:1077F00055F80646786026F07FF806F580738342D8
:1078000008D93E49012027F04DFB3D49012027F0D2
:1078100049FBD6E7F31D23F00703ADEB030D6C46E0
:107820003246214628462BF05DF97D68002DECD0CC
:1078300007223449204634F097FA60B9073D0734EF
:107840007D604FF0030878681B302CF0E3F80646A3
:1078500080B92D49DAE708222C49204634F084FA11
:1078600028B9083D08347D604FF00408EBE74FF07D
:107870000008E8E71E4B1F49024658682DF058FEE5
:1078800030462BF02BFC054630462CF00FFB204BEE
:107890002A4603F1180153F8040B42F8040B8B42FB
:1078A000F9D11B8813807E6885F8198021463246FD
:1078B00005F11A0034F066FAF3B203F108022E441F
:1078C0000133EB75FE236A740020B376FFF7FCFCEE
:1078D000394604462CF0B4FF28B103682B60436896
:1078E0006B6003892B8120462CF0E0FA69E700BF2A
:1078F000482E0020A5D80500C3D7050069D605008D
:10790000DED70500F5D7050006D80500FDD7050030
:10791000BECB050010B504462BF094FB094B0A4979
:10792000002808BF0024224618682DF001FE201C04
:1079300018BF012013F084FC40F2CC71BDE8104068
:1079400013F068B8482E0020EFCC05002DE9F74F62
:10795000464B47490746032258682DF02DFE064640
:1079600000283CD000224349DFF8088138462DF03A
:1079700023FE31468146684626F026FB009CF4B182
:1079800020462DF0A1FB0022414605462DF014FEB5
:107990000123002249468246F8F7B6FE10BBB5F82F
:1079A0000B3003F50073A5F80B302C4650462946E2
:1079B0002DF0EFFA684626F0F6FA002CDED000989B
:1079C0002CF074FA3946002C4CD001A826F0FCFAB1
:1079D000019D4DB93246494620462DF0CDFA03B0FF
:1079E000BDE8F08F0024E1E7B5F80B3003F5007334
:1079F000A5F80B3028462DF067FB012229460746E3
:107A000020462DF06CFF1C49804628462CF0E4FCF3
:107A10001A49824628462CF0DFFCBAF1000F00D14B
:107A200070B140462DF050FB8346B0B1BAF1000F63
:107A30000FD00122394630F0F6F958462CF036FACC
:107A400040463A4629462DF097FA01A826F0ABFAAF
:107A5000BEE739462DF08CFFEFE7394640462DF062
:107A6000D9F9EDE730462DF0A1FCB3E7482E002010
:107A700037CE050091CF05003ECE050047CE05006C
:107A8000F8B5054608460C462BF0C1FA0646D8B1B3
:107A900000222B4920462DF08FFD2EF00EFA0022F9
:107AA0000646284920462DF087FD044698B12BF064
:107AB000A5FA80B920462CF0F9F922462249032084
:107AC000BDE8F84027F0EEB92CB122461F4903204B
:107AD00027F0E8F9344628462BF0B4FA40B33DB31A
:107AE00048F248011A482CF0ABF8074688B1224604
:107AF00000212EF000F82A46164938462DF018FDD0
:107B0000154B164918683A462DF012FD38462CF0F0
:107B1000CDF9281C314618BF012012F027FE40F293
:107B2000DC6112F077FF2046BDE8F8402CF0BEB9CA
:107B3000094B0A4918682EF041F90025E9E700BF12
:107B4000AAD0050053CF0500B1D00500E5D005004F
:107B5000A9800200FED00500482E002003D10500B8
:107B60002DE9F84380460C462BF06CFA30B92F49CA
:107B700042460120BDE8F84327F094B920462BF097
:107B800087FA05462046C5B12EF0E4FB57EC106B92
:107B9000002432463B463046394633F079FE30B950
:107BA0000022234B3046394633F04AFEC8B1214902
:107BB0000120BDE8F84327F075B92BF028FA50B141
:107BC0002A461D4920462DF0F7FC40B12EF0B0FEAC
:107BD00006460F46DDE714B122461849C9E7184F9B
:107BE0000026184DD5F804902CF034F816490246BA
:107BF00048462DF0B4FC4246144968682DF098FCC4
:107C0000082113482CF01CF8054628B12146FFF73F
:107C100037FF28462CF04AF932463B460D4822F001
:107C200067FABDE8F8432CF041B900BFCDCD05009F
:107C3000000024401ECE050026CE0500FBCD050029
:107C400000409F40482E002037CE05002ECE050074
:107C50004D790200597C020037B5144C00210846CA
:107C6000FFF70EFF0322124960682DF0A5FC0022E9
:107C70000190104960682DF09FFC0D490546606831
:107C80002EF09CF80B4960682EF098F8019B33B1F8
:107C90002DB1012301AA2946002022F041FA2946EC
:107CA00001982DF076F903B030BD00BF482E0020BA
:107CB00037CE05002ECE05001FB54FF08052D2F80A
:107CC000A430D2F8A820D8B20290C3F307200190C4
:107CD000C2F30721C3F3074000901B0ED2B241F05C
:107CE000C00103482CF098FC05B05DF804FB00BF10
:107CF00053CE050038B52BF0B0FF1E4D0446286862
:107D00002BF0C0FF1C49024620462DF028FC686875
:107D10002BF0B8FF1949024620462DF020FCA86838
:107D20002BF0B0FF1649024620462DF018FCE868FB
:107D30002BF0A8FF1349024620462DF010FC2869BD
:107D40002BF0A0FF1049024620462DF008FC686980
:107D50002BF098FF0D49024620462DF000FC287EAE
:107D60002BF088FF0A49024620462DF0F8FB2046FA
:107D700038BD00BF08D300207CD50500D3DC05004A
:107D80007FD5050083D5050087D505008BD5050077
:107D90008FD505002DE9F04786B00D46014601A8B4
:107DA00026F012F9019838B9044601982CF07EF8B3
:107DB000204606B0BDE8F0872DF086F900229949EB
:107DC00006462DF0F9FB0746002800F0E18000226E
:107DD000944928462DF0F0FB3946804602A826F04B
:107DE000F3F801240298002840F0A180414638466B
:107DF0002DF0CFF800228C4930462DF0DDFB0746F0
:107E0000E0B10022884928462DF0D6FB804638464E
:107E10002BF068FA002800F0BD8040462BF062FA93
:107E2000002800F0B780414638462CF0D5FD0028E8
:107E30004146384608BF00242DF0ABF800227B49AC
:107E400030462DF0B9FB074610B30022764928468C
:107E50002DF0B2FB804638462BF0FBF998B1404636
:107E60002BF0F7F978B138462CF09FFC814640465C
:107E70002CF09BFC814506D8012300224146384660
:107E8000F8F742FC00B10024414638462DF081F855
:107E90000022674930462DF08FFB074680B1002253
:107EA000634928462DF088FB0146804638462CF071
:107EB00093FD41460028384608BF00242DF069F89C
:107EC00000225C4930462DF077FB804670B12BF0E4
:107ED0009EF840B1414605A826F076F8DFF85491A7
:107EE000059F002F62D140462BF0E0FF002252494F
:107EF00030462DF061FB804670B12BF088F840B120
:107F0000414605A826F060F8DFF830A1059F002F54
:107F10006CD140462BF0CAFF30462BF0C7FF01A8BA
:107F200026F041F8002C3FF43DAF01243DE7B8F1C5
:107F3000000F10D02DF0C8F8014603A81AF0D6FAA9
:107F4000414604A826F040F84FF00009049838B9DB
:107F5000B9F1000F00D1002402A826F024F841E76F
:107F60002DF0B2F8014605A81AF0C0FA9DF81620C7
:107F70009DF80E309A4207D1BDF81420BDF80C30A0
:107F80009A4208BF4FF0010904A826F00CF8DDE77B
:107F900001242FE738462AF0D5FE814640462AF0D4
:107FA000D1FEA9EB00035842584140E7B7F80B3027
:107FB00003F50073A7F80B300022494628462DF040
:107FC000FBFA824680B1002239462DF088FC002859
:107FD00008BF00242BF06AFF384651462CF0D9FF29
:107FE00005A825F0E0FF7BE70446F5E7B7F80B307E
:107FF00003F50073A7F80B300022514628462DF0F8
:10800000DBFA8146014638462CF0E6FC494600285A
:10801000384608BF00242CF0BCFF05A825F0C3FF9C
:1080200074E700BF3ECE050041D80500A4CD050091
:1080300091CF050047CE0500AFCD0500C0CD0500AE
:1080400073B505460E462AF0D9FF38B91549032005
:1080500026F028FF0024204602B070BD30462AF0EA
:10806000CDFF0028F2D02BF0F5FD04460028F2D019
:10807000294601A825F0A8FF01980028EBD02DF093
:1080800023F8054601463046FFF784FE18B129461D
:1080900020462DF08BF928462BF008FF01A825F08B
:1080A00082FFE9E77ECD05002DE9F04F87B000AFF4
:1080B000C7E902011446002A6CD09149002024F03F
:1080C000EFFF0022054638618E4920462DF074FAF4
:1080D0008C49024628462DF042FA00228A493D6921
:1080E00020462DF069FA8849024628462DF037FAD5
:1080F0002BF0B0FD80462BF0B0FD00228246834974
:1081000020462DF059FA8146E8B102467F49386988
:108110002DF00EFA002307F1140148467B612CF084
:108120008FFB0446002844D148462AF0B7FB054699
:10813000786125F0E1FB05F5807383422ED97449FF
:10814000012026F0AFFEB8F1000F07D0D8F80030BC
:1081500023B142466F4938692DF0EAF950462CF0B8
:1081600046FB20B152466C4938692DF0E1F9524680
:10817000414648462CF000FFFB68002B40F0B780DA
:1081800007F1100301220021B86823F015FC3869BB
:108190002BF08CFE1C37BD46BDE8F08FEB1D23F0A5
:1081A0000703ADEB030D6C462A46214648462AF0EC
:1081B00099FC7B69002BC6D0B8F1000FCED0BAF184
:1081C000000FC0D0002514E0092A09D1A91C2144C0
:1081D000701ED7F810B02CF07BFD5049024619E014
:1081E000911E012927D89B4602239E4216DA0136AA
:1081F00035447B69AB42A6D96319665D5A78082A73
:10820000E2D1A91C2144701ED7F810B02CF060FDFB
:108210004349024658462DF0A2F9E8E73BF8021F11
:1082200040487B602CF0F8F9014640462DF0D7F825
:108230007B680233D9E7911F012908D8A81C204484
:108240001AF024FA014640462DF0C9F8CFE7162A65
:108250002BD0212A32D1A81C20441AF017FA12235D
:1082600083463B60BBF1000F1BD0012259465046AC
:108270002DF035FB3B6878605919701CC01A2144F9
:108280002BF023FE7A6803463AB130B101463860DC
:1082900010462CF0BFFDD7E90032194610462CF0ED
:1082A00078FE58462BF002FEA1E759881D482CF0B5
:1082B000B3F92EF043FD04238346D2E7FF2A96D17B
:1082C000D8789B78D7F810B043EA00202BF0DAFC7E
:1082D0001549024658462DF042F9291D2144F01E49
:1082E000D7F810B02BF0F1FD1049024692E7D7E91C
:1082F0000301FFF74FFD00287FF442AF47E700BFBF
:1083000074D1050091CF0500F5CC0500BFD805005C
:1083100069D605003ECE050047CE050041D80500D0
:1083200084D105005A060600C0CD0500AFCD05007A
:108330002DE9F04186B000AF00238846391D044680
:108340007B602CF07DFA0546002C38D0E0B9204641
:108350002AF0A4FA0646786025F0CEFA06F5807376
:10836000834206D94149012026F09CFD224640491E
:108370003BE0F31D23F00703ADEB030D6D463246E2
:10838000294620462AF0AEFB7B68002BEED0404603
:108390002AF058FE28B1374B3749186842462DF06D
:1083A000C7F8364B1A6812F0400F1E460AD13449FE
:1083B000012026F077FD1837BD46BDE8F081002882
:1083C000E2D1D3E72F4A12884FF6FF71914201D1D3
:1083D0002D49EDE71A6812F0800201D02B49E7E73A
:1083E0007C68102C05DD2A491022012026F05AFD58
:1083F000E1E7284B93F800C0274BA4B2BCF1000F73
:1084000025D19A7C72B3B3F8760188422CD09B8A2E
:108410007C80C7F80AC0A7F80EC03B810123BB725D
:1084200007F10801BB1CC7E90435FBF755FC18B977
:108430007B88A34218BF0C2040F6BB3112F0EAFA49
:108440000028B8D1336843F080033360B3E7B3F852
:108450007601884208D07C80C7F80A20FA81B3F8F8
:108460004E31DAE70720E7E70820E5E769D605009F
:10847000FACF0500482E00208ACF0500FCD200204C
:1084800094CF05006A2D0020A8CF0500B7CF0500C6
:10849000CFCF050039D3002030CD00202DE9F04F9B
:1084A0009D4B91B01B681B0700AF044607D59B4945
:1084B000012026F0F7FC4437BD46BDE8F08F15F0EB
:1084C000DDFA20462AF0A3FD0546002800F01A81B7
:1084D000214607F1140025F077FDDFF864A27969E1
:1084E00089B10023BB61B1F80B3003F50073A1F82B
:1084F0000B3007F1180019F0F9FF024638B188492E
:10850000012026F0CFFC78692BF0D0FCD3E7D7F818
:108510001480B8F1000F03D040462CF0D5FD804602
:10852000414607F11C0025F04FFDF96985B179B18D
:10853000B1F80B3003F50073A1F80B3007F1200000
:1085400019F0D4FF024670B17649012026F0AAFC4A
:10855000F8692BF0ABFC40462BF0A8FC07F11400A7
:1085600025F021FDBBE707F128003C8C97F822603D
:108570001AF0CCF808B1F9F7A1FC4FF0000900227D
:1085800007F13001388DC7F830901AF0BDF8052892
:1085900010D043F2030290420CD0A8B93B8EA34204
:1085A00014D197F83230B34210D1B7F82890B9F10E
:1085B000000F0FD1386A1AF07FF85B490446024673
:1085C000012026F06FFC3EE0F9F778FC3B8D01338B
:1085D0003B85D4E7FC691CB120462CF075FD0446B0
:1085E0000022524920462CF0E7FF0022504906465F
:1085F00020462CF0E1FF2DF060FC0022B8604D49D0
:1086000020462CF0D9FF2DF058FCF860C6B10023AD
:1086100007F1240130467B622CF012F9834620BB1F
:1086200030462AF03BF97862786025F065F97A687F
:1086300002F5807383420ED93F49012026F032FCB7
:1086400030462BF033FC20462BF030FC07F11C00A9
:1086500025F0A9FC69E7D31D23F00703ADEB030D5B
:10866000EB46594630462AF03DFA7A6A002AE7D0AE
:10867000002179853A85494607F12802BAF80000B9
:10868000C7F82CB0FDF7D4FE40F2915112F0C2F9B8
:10869000BB6880F00100C5B213B9FB68002BCFD0D6
:1086A000BAF800204FF6FF719142C9D0FB68BAF8C2
:1086B0000000A7F830900022002BC7F83220FA867D
:1086C0007A6A7A8214BF0222012287F8322007F1E7
:1086D000300107F11202C7E90E2BFBF7FDFA30F06B
:1086E0000802ADD043F204029042A9D043F2014205
:1086F0009042A5D040F2A65112F08CF9002818BF84
:1087000000259DE7002C3FF4D6AE22460B490320FE
:1087100026F0C8FBCFE600BFFCD2002024D2050023
:108720004CD2050065D2050095D2050038E305005E
:1087300085D205008CD2050069D60500B9D20500A6
:108740006A2D00202DE9F04F9BB000AF0D46044686
:108750003C22002107F12C00F6F7E4FE022387F803
:108760002C302846062387F82F302AF050FC0028AA
:1087700079D00022844928462CF01EFF38B12DF014
:108780009CFB002814BF0223002387F82C30002212
:108790007E4928462CF010FF38B12DF08EFB0028C2
:1087A00014BF0623052387F82F3000227849284676
:1087B0002CF002FF8146D0B1002307F10C01FB60D1
:1087C0002CF03EF8064600283CD148462AF066F8D0
:1087D0008046F86025F090F808F58073834225D92B
:1087E0006C49012026F05EFB48462BF05FFB2846D3
:1087F000002269492CF0E0FE054640B13B6D6BB3A9
:108800002CF080FC3B6D188028462BF04FFB204657
:108810002AF0F4FB80B3B4F80B3003F50073A4F82E
:108820000B3020466C37BD46BDE8F08F08F10703DA
:1088300023F00703ADEB030D6E4642463146484632
:108840002AF050F9FA68002ACED084B06B464FF671
:10885000FF713B6519809A809E60C5E74F490320F0
:1088600026F020FBD0E7002DD1D04D492A46032029
:1088700026F018FB0024D4E720462AF0A2FB054688
:108880000028C8D120462AF0C2FB002876D0204616
:108890002BF0F2FC0C235843073020F00700ADEB1F
:1088A000000D214607F1080025F08EFBE846DFF8B1
:1088B000E4A04446A946B868F8B987F85850C7F804
:1088C00054801F2307F1080207F10C0107F12C0067
:1088D0003B81FCF7A7FA18B1324B5B68002BC9D07B
:1088E00040F2F63112F096F80028C3D107F10C01DE
:1088F00038892BF0EAFA044693E72CF0E5FB07F100
:108900000C018346C7F80C902BF09AFF0646BBF18A
:10891000000F10D078B9584629F0C0FFF860786091
:1089200024F0EAFF7A6802F5807383421BD951462E
:10893000012026F0B7FA58462BF0B8FAB86828B1EB
:10894000B0F80B3003F50073A0F80B302DF07CF974
:10895000FB682080A380A66007F1080025F023FBB8
:1089600001350C34A7E7D31D23F00703ADEB030D4E
:108970006E46314658462AF0B5F8DCE7002CA0D008
:108980002246094973E700BF71CE05007ACE050083
:10899000AFCD050069D60500C0CD050087CE050026
:1089A000BBCE0500482E0020F1CE050008B5064AD2
:1089B000136823F40073136012F0BAF840F20B212D
:1089C000BDE8084012F026B8FCD2002008B5054AE0
:1089D000136843F40073136011F0F4FEBDE808401F
:1089E000FEF754BBFCD2002008B513F095FB41EC18
:1089F000100B08BD10B50F4B1B884FF6FF729BB2D2
:108A00009342044603D10C4A1288934208D00B4883
:108A100021F0F4FB0A4A136843F00803136010BD09
:108A20002AF010FB002814BF20460020BDE81040AB
:108A300014F0B2BD682D00206A2D00205BCF050028
:108A4000FCD2002010B504462AF0E1FA224630B9E3
:108A50002CB10B490320BDE8104026F023BA094B86
:108A6000094958682DF0BBF912F052FA074B1B6800
:108A70001B0704D50020BDE81040FFF7BBBF10BDA9
:108A80008ED10500482E0020B7D10500FCD2002071
:108A900038B5104C10490022054660682CF08CFD5A
:108AA0002DF0D2F8C3B285B143F0010098420FD047
:108AB00064682BF0E7F80849024620462CF04FFD89
:108AC0000020BDE83840FFF795BF03F0FE00EDE75A
:108AD00038BD00BF482E0020A0D005002DE9F04190
:108AE0008CB0064688462AF092FA40B93EB132462A
:108AF0004749032026F0D6F90CB0BDE8F0810023E9
:108B000002930193434B039302AB0593424B0693AD
:108B100003270B23ADF81C300DEB0703012208934C
:108B20003E4B8DF8032009933A4601AB03A940461A
:108B3000ADF81070ADF828700B932DF07DFC002877
:108B4000DAD00298364D374C2AF0B0FB48B1029A81
:108B5000354968682CF0ECFC236843F00803236077
:108B600009E0029B002B37D12F4968682DF026F9C8
:108B700023685906F0D402982BF098F99DF8033039
:108B8000002B2ED02368294968689A065EBF2368A7
:108B900043F0080323602DF011F932462449686838
:108BA0002DF01DF94246234968682DF018F9019A05
:108BB0001AB1236843F0080323601F4968682DF049
:108BC0000EF901982BF072F9236813F0180F1BD0DF
:108BD0000020FFF70FFF8FE71849384626F062F9AB
:108BE000C9E723686F689B0648BF23684FF0000001
:108BF00044BF43F0080323602BF03CF80B490246C6
:108C000038462CF0ACFCC8E7304614F011FD73E791
:108C1000B9D2050090CF0500BFD10500C4D1050031
:108C2000482E0020FCD20020CED10500FDD1050049
:108C300006D2050010D205001AD20500D8D10500D1
:108C400013B56946044619F095FC28B90749012077
:108C500026F028F902B010BD054B06495868224697
:108C60002CF066FC0020FFF7C5FEF3E712D00500EC
:108C7000482E002048D0050038B50A4C05462DB9CD
:108C8000094B002C08BF1C46204638BD3CB120468D
:108C900033F0B2F8013D01300444EDB2EFE7024C8D
:108CA000F2E700BFD9CB05002C4B060070B50D4C88
:108CB000064620780D4640B1FFF7DEFF0A4902461E
:108CC000012026F0EFF8002070BD09F0E3FB074B10
:108CD00026701860284629F015FF054B1860012002
:108CE000F2E700BF00D3002063CC0500F8D20020DB
:108CF00004D3002037B50546002105208DF8061065
:108D0000FFF7D4FF58B1074B186829F0FBFE019913
:108D10000446284611F0F2FD204603B030BD04465B
:108D2000FAE700BFF8D2002037B505460C4605200B
:108D30000021FFF7BBFFB8B1214601A819F040FBA5
:108D4000024638B10949012026F0ACF8002420463B
:108D500003B030BD064B186829F0D4FE01990446D3
:108D6000284611F0CBFDF2E70446F0E703DB0500EF
:108D7000F8D2002013B5002104208DF80610FFF76B
:108D800095FF50B1064B186829F0BCFE04460198C7
:108D900011F0FAFD204602B010BD0446FAE700BF0C
:108DA000F8D2002013B50C4604200021FFF77EFF07
:108DB000B0B1214601A819F003FB024638B10949B8
:108DC000012026F06FF80024204602B010BD064BAB
:108DD000186829F097FE0446019811F0D5FDF3E7D5
:108DE0000446F1E703DB0500F8D200202DE9FF413E
:108DF00000228846264906462CF0DEFB0022254943
:108E000007462CF0D9FB6946054619F0B3FB04462A
:108E100058B9294638462CF0BCF81F49032026F0E3
:108E200041F8204604B0BDE8F08138462BF03EF80A
:108E300000221A4930462CF0BFFB2DF03EF80746C1
:108E400020B1304609F086FB0446EAE731460220AD
:108E5000FFF72CFF20B9002428462BF027F8E0E785
:108E600048210F482AF0ECFE04460028F3D00146C2
:108E7000022302AA3846CDE9025821F051F92046D2
:108E80002BF014F8074B186829F03CFE0446E3E782
:108E9000C5CC050091CF05003ACD0500E5CC050015
:108EA00021C00200F8D2002070B504460E46002012
:108EB0000E4924F0F5F8054610B90025284670BD86
:108EC00022460B492CF034FB2846FEF715F90446E0
:108ED00028462AF0EBFF002CEFD031462046FFF762
:108EE00085FF054620462AF0E1FFE7E774D105003B
:108EF00091CF050070B5064650B12AF088F80446B7
:108F000030B928493246032025F0CCFF204670BDF9
:108F10000022254930462CF04FFB05462AF06EF81A
:108F20000446284624B92AF0C1FF2A461F49EAE729
:108F30002AF0BCFF00221E4930462CF03DFB2DF0EC
:108F4000F7FC02460B4604460D4632F0A1FC30B950
:108F5000002200232046294632F07CFC08B1154D42
:108F600000242B462246144821F0C2F8054601464B
:108F70000120FFF79BFE78B1082110482AF060FE1F
:108F8000044628B13146FEF77BFD20462AF08EFFCD
:108F90000B4B186829F0B6FD044628462AF086FFD8
:108FA000B4E700BF1ECF050053CF0500B1D00500C8
:108FB00026CE050000409F40C5BC020075C10200DE
:108FC000F8D2002030B500218FB0044609202BF0E4
:108FD0007FFE164D0190024680B115496868FF2357
:108FE000CDE90213002313498DF810302CF0B7FAA5
:108FF00001A81AF07AFA01A81AF07EFA01A81AF06C
:1090000074FA01A81AF06EFA22460B4968682CF02F
:109010008FFA0A4B02221A70B4F80B30204603F57F
:109020000073A4F80B300FB030BD00BF482E0020F5
:109030000300FFFF3E0B0600BFD7050040D3002012
:1090400019F022BC19F064BB38B5054609B119F016
:10905000CFFB00220D4928462CF0AEFA2CF02DFF54
:1090600010B10B482BF08CFE01460446284619F03F
:10907000BFFB20462AF01AFF01202AF0FBFD05491C
:1090800002462846BDE838402CF069BA0DC00500FC
:10909000411806002BD6050008B519F0A9FB0020E1
:1090A00008BD000070B58EB0044601A80E461546F6
:1090B0001AF07CFA90B12046002209492CF07CFA83
:1090C000044658B1324607492CF032FA2A4606497E
:1090D00020462CF02DFA20462AF0E8FE0EB070BD96
:1090E00004D3050008D3050017D3050010B58EB0D2
:1090F000044601A81AF05AFA30B101A8214619F025
:1091000079FD01A81AF0EEF90EB010BD70B5064653
:109110002BF0DAFF054629F095FF044640B90E48CA
:10912000294625F09FFD28462AF0C0FE204670BD46
:1091300028462AF0BBFE0949002023F0B1FF04466F
:109140000028F3D0012119F0DBFD32460449204606
:109150002CF0EEF9EAE700BF2FD6050056D6050041
:109160005ED6050070B506462BF0AEFF054629F029
:1091700069FF044640B90E48294625F073FD28468C
:109180002AF094FE204670BD28462AF08FFE094939
:10919000002023F085FF04460028F3D0002119F0B9
:1091A000AFFD3246044920462CF0C2F9EAE700BF81
:1091B0002FD60500BECC05005ED6050030B591B0B7
:1091C000044603A80D461AF0F1F948B1002303A89C
:1091D00000932A46214619F0EFFB03A81AF082F902
:1091E000002011B030BD30B58FB0044601A80D4647
:1091F0001AF0DCF958B11DB129462046FFF7DEFF11
:1092000001A8214619F0F6FC01A81AF06BF90FB07D
:1092100030BD000030B58FB0054601A81AF0C6F980
:10922000E8B10021114819F079FD0446A0B12946A2
:1092300001A819F02DFD2946012220462EF0DAFD65
:10924000054670B1014620462CF008FD28462AF05C
:109250002DFE20462AF02AFE01A81AF043F90FB08D
:1092600030BD034825F0DEFCF3E700BF7BD70500E7
:1092700081D705002DE9F04391B0804603A80F4641
:1092800014461E461AF092F9B8B1002118982BF036
:1092900029FF054629F0FCFE78B320462BF032FF6B
:1092A000814630462BF02EFF06461B202AF05AFC42
:1092B000044628B903A81AF015F911B0BDE8F083E7
:1092C00033464A4639462BF069F9012118982BF0AC
:1092D00009FF064628462BF015FF80B20090334662
:1092E0002246414603A819F067FBBC42E2D0324651
:1092F000294620462BF040FEDCE728462AF0D6FD22
:1093000025463C46E6E700002DE9F04F8BB082464B
:10931000019129F09EFF20B9002630460BB0BDE830
:10932000F08F2AF09AFC06460028F5D04FF000098D
:109330004FF0FF350022514605A825F032FACB4602
:109340002C46A8462F464A464B46DDE90501814298
:1093500000F2B680B4F1FF3F08BF5C4608982AF0DF
:10936000A5FDB8F1FF3F08BFA046002F09DD7A1E1A
:10937000002150462BF03FF9A349024630462CF01D
:10938000EEF8A2482BF0FCFCA149024630462CF036
:10939000E6F8791CA8EB010250462BF02CF99D4908
:1093A000024630462CF0DBF86FF000422146504672
:1093B0002BF021F907462BF0F8F918B996493846F1
:1093C0002BF085F93A46954930462CF0C8F8691CCF
:1093D00014BF2A1B6FF00042214650462BF00BF9B8
:1093E00004462BF0E2F918B98B4920462BF06FF9AF
:1093F00022468B4930462CF0B2F86A1C00F09E8061
:109400006FF00042294650462BF0F5F80246854998
:1094100030462CF0A4F809F1FF324FF6FE739A4261
:1094200040F2908002202AF09DFB02467E493046A1
:109430002CF095F86B1C00F089806FF00042691CDD
:1094400050462BF0D8F8019B80469BB329F0A0FD35
:10945000044678BB0246414605A825F0A2F92AF049
:10946000FCFB81461B202AF07DFB05461B202AF0D1
:1094700079FB0746DDE905239A426BD308982AF069
:1094800015FD40462AF012FD28462BF08EF90028E3
:1094900000F08D8028462DF051FC394605462BF012
:1094A0000DFB294648462BF0A3FE394628462BF0F3
:1094B00070FDC84642465D4930462CF050F82CE716
:1094C00005A8CDE9022325F065F82F28DDE9022360
:1094D00012D1B4F1FF3F08BF5C46012A03F101033A
:1094E00006D1022B04D1791C02D13D463C465F4691
:1094F000B8F1FF3F0DD118E03A2807D1791C02F1ED
:109500000102F5D0611CF3D1D8460EE0B8F1FF3F5F
:109510000ED0D8450CDA611C73D12F2805D9392813
:1095200003D830380A2101FB09090BF1010B0CE7C4
:109530003F28FAD1601CF8D05D46F6E702202AF0F9
:1095400011FB63E748462AF09DFB6EE702202AF0F4
:1095500009FB78E705A825F01DF8262822D1284622
:109560002BF023F9C0B128462DF0E8FB394604461C
:109570002BF0A4FA214648462BF03AFE3946204605
:109580002BF007FD1B202AF0EDFA05461B202AF0E0
:10959000E9FA074600246DE738462BF006F9002863
:1095A000E1D167E754B93D2820D1019C62E73846F4
:1095B0002BF0FBF800287FF46DAF76E725280CD15F
:1095C00005A824F0E7FF824605A824F0E3FF014642
:1095D000504624F0C6FBC0B254B18DF813000122EE
:1095E0000DF1130138462BF059F8DEE72528E7D0B6
:1095F0008DF8130001220DF1130128462BF04EF8CF
:10960000C8E73F2898D090E7F8D8050001D90500B1
:1096100005D90500470B0600FBD705000CD905004E
:1096200011D905001AD9050021D9050026D9050050
:109630002DE9F04F2DED028BA3B08B4615462AF095
:1096400009FB8246002800F0C080584629F02EFE13
:10965000002800F0BA80284629F0D9FC002800F044
:10966000908008AA1892804A199206AA1B927F4AF3
:109670007F4B1C9204AADFF8049216931E920A23D1
:109680007C4AADF85C30002600274FF00008ADF8AA
:109690006830ADF874301F92ADF88030042202AB10
:1096A00016A92846CDE90867CDE90667CDE9048902
:1096B000CDE9026721932CF0BFFE002800F08580E1
:1096C0009DED028B32463B4651EC180B32F0AEF862
:1096D000002851D1B0EE480AF0EE680A2FF0B4FC31
:1096E00053EC102BB0EE480AF0EE680ACDE90023E7
:1096F0002FF09AFDDDE9002355EC104BDDE90467FE
:109700003046394631F02AFE3246804689463B468D
:10971000204605F10041CDE90A8931F01FFEDDE95F
:109720000823CDE90E01CDE91223304622462B460F
:10973000394631F013FEDDE90623CDE90C01CDE910
:109740001089CDE914230122594616A825F0D5FD2C
:1097500016A824F0F1FB58B116A824F07DFD0646AA
:1097600016A80F4624F003FD16A824F0E5FB90BBD5
:1097700016A824F0B5FB28E034463D4642464B4649
:10978000BCE7284629F092FDC8B128462BF02FF8F7
:109790000628044613D12946012216A825F0ADFD5E
:1097A0000AAD16A824F058FDE5E8020116A824F039
:1097B000DEFC013CF5D116A824F092FBC3E72E494C
:1097C000032025F06FFB4FF0000A504623B0BDEC9C
:1097D000028BBDE8F08F16A824F03EFD044616A8C3
:1097E0000D4624F0C4FCDDE90A233046394631F049
:1097F000B5FDDDE90E23804689462046294631F035
:10980000ADFD02460B464046494631F0F1FBDDE92D
:10981000122331F0EDFB41EC100B2AF021FA014646
:1098200050462BF0DCFDDDE90C233046394631F0A3
:1098300095FDDDE9102306460F462046294631F006
:109840008DFD02460B463046394631F0D1FBDDE94D
:10985000142331F0CDFB41EC100B2AF001FA014644
:1098600050462BF0BCFD73E7DDFB0500D5D50500A8
:109870001DFB0500DBD50500E2D505000000F03F2B
:109880002DE9F04F93B00C4616462AF0E3F9054651
:10989000002800F08480002C00F081802368062BD3
:1098A0007DD12146012207A825F027FD01AF002424
:1098B00007A824F026FD013447F8040B07A824F07C
:1098C00056FC062CF4D107A824F00AFB304629F0F8
:1098D0009EFB30B10022354930462BF06DFE2CF056
:1098E000B3F9DDF80480059EDDF80890069FB8EB1B
:1098F000060448BFA6EB0804B9EB070348BFA7EB73
:1099000009039C42A8BF1C46002C08BF01244FF449
:10991000A04393FBF4F4B4F5805F44DA40F299136A
:109920009C42B8BF1C460028C8BF4FF480544A462A
:10993000C8BF94FBF0F4414628462BF05AFDC4F50D
:10994000805BA2460BFB0BFC0AFB0BF04FEA2C3CA6
:10995000049A40F3D3200CFB09F302FB0032039B73
:109960000AFB0AF10CFB08FC03FB00C3091301FB13
:10997000072201FB063102F5006201F500611213B6
:1099800009132846A2442BF034FDBAF5805FABEBF7
:10999000040BD7DD3A46314628462BF02AFD2846EF
:1099A00013B0BDE8F08F40F25554BCE7CBD40500AE
:1099B0002DE9F04F9BB0014609A81AF0C1F828B96B
:1099C0000023039303981BB0BDE8F08FBDF8293046
:1099D0009DF82F40DB06A4F1020347BFBDF82D70B0
:1099E000BDF82B60BDF82B70BDF82D60012B70D930
:1099F000082CB8BF082407FB04F31F33082C4FEAD8
:109A00006313D8BF4FF001094FEA83030093D4BF1B
:109A100009FA04F94FF00009009B09EB490505F12B
:109A20001A0803FB068A504629F0F4FF0390002829
:109A3000C6D029F053FB422303704D2343700C23FF
:109A400083733B1280F802A0C3744FEA2A2A3312B0
:109A50004FF0010E082C80F803A080F80A8087746C
:109A60000675437580F816E0047634DD0123A340C3
:109A7000013B0693009A0823B3FBF4F30193E31030
:109A80000593731E02FB0355431902934FF0000820
:109A9000B04597DA08F101030493029B072C03F108
:109AA0001A0547DD4FF00009B94549DA42464946F3
:109AB00009A819F0F6FF2A46002308339C4202F851
:109AC000010B4FEA1020F8DC059B09F101091D4448
:109AD000EAE704248FE79DF82F30032B00F11A03E7
:109AE00015D000219DF82F200EFA02FC8C4503F1C1
:109AF0000303BBDDC1EB012292FBFCF2D2B203F8FF
:109B0000032C03F8022C03F8012C0131EAE70022B0
:109B10004A4503F10303A9D042F3000103F8031CF3
:109B200042F3400103F8021C42F3800103F8011CD8
:109B30000132EDE7DDF804B04FF0000ABA451CDB56
:109B4000029B009ADDF810809B1A0293A0E74B1C41
:109B5000424609A8079319F0A4FF069B1840079BEB
:109B600009FA04F940EA090919465945EFD1019B60
:109B700005F8019B9A449B44E0E751464FF00009E9
:109B8000F3E7000038B5FFF713FF054610B90025CD
:109B9000284638BD0CF0CAF8044628462AF086F953
:109BA000002CF4D0214604482AF036FD0546204614
:109BB0002AF07CF9ECE700BF39D3050010B5FFF7B8
:109BC000E1FF044608B121F06FFE20462AF06EF94D
:109BD0000248BDE8104021F09FB900BF40180600C0
:109BE00000B593B0014601A819F0AAFF10B101A871
:109BF000FDF7EAF913B05DF804FB000000B593B07F
:109C0000014601A819F09CFFD8B1BDF8180010F466
:109C100060430AD0B3F5005F0D4918BF00211B0453
:109C200005D429B92AF02EF80BE00A49F7E70A49CA
:109C300041F6FE73184207D0C0F30C0207482AF021
:109C4000EBFC13B05DF804FB08462BF099F8F8E73D
:109C50008BD4050084D40500C4D405008FD405003E
:109C600030B593B00C46014601A8154619F068FFBF
:109C700020B12A46214601A819F013FF13B030BDC8
:109C800000B593B0014601A819F05AFF08B19DF83C
:109C90000F0013B05DF804FB2DE9F041B2B00546AA
:109CA000884601460CA819F04BFF002800F0D4802C
:109CB0000BAA1F92694A20920AAA2292684A694B0B
:109CC000239209AA1D9325920923674AADF878309B
:109CD000ADF88430ADF890302692ADF89C3008AAEB
:109CE000ADF8A830ADF8B43006AB28922E935F4A99
:109CF0005F4B29922F9307AA0B2300242B92ADF8D8
:109D0000C0305C4ABDF83770BDF839608DF8174037
:109D10000DF117034046CDE90A44CDE90844CDE9E9
:109D200006442C92319329F072F940B9524901202E
:109D300025F0B8F80025284632B0BDE8F0810722AA
:109D40001DA940462CF078FB0028EFD00B99099A0A
:109D500000290A4404DA079B09925B1A07930B94C3
:109D60000A98089B0028034405DA06990893091A03
:109D7000069100210A91D21B002AC8BF09990B98AD
:109D8000C8BF8A1AA3EB0603C8BF0992002BC8BF3D
:109D9000089A0A99C4BFD31A0893079B099A002B03
:109DA0001A4404DAC31A0B93002309920793069806
:109DB000089B0028034404DA091A0A910021089339
:109DC0000691D71B002FC8BF099A07990698C8BFEC
:109DD000D71BA3EB0603C8BF0997002BC2BF089A85
:109DE000D31A0893DDE90823002B01DC002A2CDDBF
:109DF000CDE901100092DDF86B40DDE90A210CA8E5
:109E0000A0479DF8173003B3DDE90610BDF95340B4
:109E1000099A089BA0420244B8BFADF85300BDF9AF
:109E200057008242C8BFADF85720BDF95520914276
:109E3000BDF95920B8BFADF855100B4493420CA89A
:109E4000C8BFADF8593019F057FEB5F80B3003F51F
:109E50000073A5F80B306EE705466CE755D3050097
:109E6000B1FE050052D30500A1FC050058D3050042
:109E70005ED305005BD305006AD3050030B593B00F
:109E80000D46014601A819F05BFE00284CD0BDF933
:109E90002720BDF92B309A4244DC29F0DEFE04462F
:109EA00018B3BDF9270029F0EDFE204902462046EF
:109EB0002BF055FBBDF9290029F0E4FE1C490246B0
:109EC00020462BF04CFBBDF92B0029F0DBFE194995
:109ED000024620462BF043FBBDF92D0029F0D2FEAF
:109EE0001549024620462BF03AFBC5B100226FF01F
:109EF0007F038DF82B208DF82C308DF82D208DF8D8
:109F00002E304FF0FF327F2301A88DF827208DF8E7
:109F100028308DF829208DF82A3019F0EDFD2046E3
:109F200013B030BD0024E0E70446F8E752D3050043
:109F300055D3050058D305005BD3050070B592B02A
:109F400004460D46014601A8164619F0F9FD58B31E
:109F5000BDF80930022D23F070039BB21ED0032DF3
:109F60001FD0012D08BF43F03003ADF809304EB1CA
:109F7000BDF80930DA064CBF83F0400383F02003BC
:109F8000ADF8093001A819F0B7FDB4F80B3003F5AE
:109F90000073A4F80B30204612B070BD43F060038C
:109FA000E3E743F05003E0E70446F4E770B592B00E
:109FB00004460E46014601A8154619F0C1FD78B1C8
:109FC00001A8ADF81A60ADF81C5019F095FDB4F871
:109FD0000B3003F50073A4F80B30204612B070BDAF
:109FE0000446FAE7F0B593B004460E46014601A8D0
:109FF00015461F4619F0A4FD08B3012E9DF81E104A
:10A00000A8BF0126012DA8BF012546EAE67666F322
:10A01000010145EAE57565F3830187F3020767F3FC
:10A02000051101A88DF81E1019F066FDB4F80B306B
:10A0300003F50073A4F80B30204613B0F0BD0446BE
:10A04000FAE700002DE9F04792B004468A4601463F
:10A0500001A8914698461A9F19F072FD002859D020
:10A06000504629F0F6F840B92B49012024F01AFF98
:10A070000024204612B0BDE8F087B9F1FF0F01D9E6
:10A080002649F2E7404629F0E4F828B9404629F08D
:10A09000B5F908B92249E8E7C7F30726002E4FEAC9
:10A0A000274308BF0126012B05DD022B2CD0042BF2
:10A0B0002DD01C49D9E74FF4004552461A49204695
:10A0C0002BF036FA4246194920462BF031FAF8B205
:10A0D00029F0D8FD1649024620462BF040FA4846A2
:10A0E00029F0D0FD1349024620462BF038FA3544BA
:10A0F00001A8ADF8185019F0FFFCB4F80B3003F5C7
:10A100000073A4F80B30B4E74FF42045D5E74FF4C3
:10A110004045D2E70446ACE7EBD4050008D505007E
:10A1200025D505004FD505006DD5050072D5050074
:10A1300095D4050077D50500F0B593B004460F46D9
:10A14000014601A816461D4619F0FAFCA0B1189B5D
:10A15000ADF8253001A8ADF81F70ADF82160ADF85D
:10A16000235019F0C9FCB4F80B3003F50073A4F8C0
:10A170000B30204613B0F0BD0446FAE72DE9F0415C
:10A180009AB007460D46014609A8144619F0D8FCB6
:10A190004FF000080646002800F09D8006AA05A999
:10A1A00009A8CDE90754CDE9058819F0E7FB08AA0D
:10A1B00007A909A819F0E2FB059B079D089CBDF8BB
:10A1C0004120BDF84310BDF845000791ED1A069BEC
:10A1D0000890E41ABDF82B3006929D42C8BF1D4678
:10A1E000C3F10003C8BF4646AB42C8BF1D46BDF819
:10A1F0002D30C8BF00269C42C8BF1C46C3F10003D7
:10A20000C8BF0026A342C4BF1C460026BDF83F308D
:10A21000059346B1CDE901100092DDF86360224656
:10A22000294609A8B047DDE90512BDF94760DDE917
:10A230000730B142BDF94B60B8BFADF84710B3422B
:10A24000BDF94960C8BFADF84B30B242BDF94D60B1
:10A25000B8BFADF84920B042C8BFADF84D00002DE1
:10A2600023DD6B180D9DDDF85760CDE90005013B3E
:10A2700009A8B047002C23DD069A0D9B01931444D6
:10A28000013CDDF85750079B0094059909A8A847A1
:10A2900009A819F031FCB7F80B3003F50073A7F8E3
:10A2A0000B3038461AB0BDE8F081E3D00D99DDF8E7
:10A2B000576003F1010CCDE900010CEB0501D7E774
:10A2C000E6D0089B0D99DDF857505A1CCDE90031B6
:10A2D0002244079BD9E70746E3E70000000000009F
:10A2E0002DE9F04FCDB005460E46014617A817469A
:10A2F0000293569C19F024FC002800F06783382252
:10A30000002109A8F5F70EF9304628F080FE002854
:10A3100054D0B04930462BF06DF900284ED031466C
:10A3200028A819F00DFC002800F0A8809DF8A48052
:10A33000B8F1000F40F0A280BDF8A7300993BDF836
:10A34000A930A5490A9342469DF8AB300B9330469D
:10A350002BF032F906462AF05FF80E90304629F0CD
:10A36000A5FDCDF83C809DF8303013B94FF0FF3398
:10A370000D93109B5BB90B9B012B08D11B9AADF879
:10A3800054201A9AADF8562015AACDE910230E983C
:10A3900028F05FFF064648B10999002906DD0A9BAF
:10A3A000002B03DD0B9B202B40F32C818B490120DC
:10A3B00024F078FD0E9829F079FD5FE0304628F012
:10A3C00026FE002872D00022854930462BF0F4F892
:10A3D0002BF03AFC00228349099030462BF0ECF830
:10A3E0002BF032FC002280490A9030462BF0E4F832
:10A3F0002BF02AFC0028CCBF0B9001234FF0000269
:10A400007A49D8BF0B9330462BF0D6F8031C18BFFF
:10A4100001238DF830302BF017FC00220D90744989
:10A4200030462BF0C9F8804688B328F0CAFD50B3F7
:10A43000B8F80430022B26D1002328A940462893DF
:10A440002AF0FEF91090404629F030FD289B102B91
:10A4500005D9B3F5807F06D00023109305E0654A47
:10A46000DA40D107F8D5013B1193DDF84080B8F10F
:10A47000000F0CD16049012024F014FD002528466E
:10A480004DB0BDE8F08F404629F010FDEDE7002209
:10A49000514930462BF090F8064629F0BDFF0E904A
:10A4A000304629F003FD00230F935CE7304628F087
:10A4B000D0FE58B1304628F084FD70B9B6F80B30A4
:10A4C0000E9603F50073A6F80B300AE0304628F02C
:10A4D00078FD0028EED14949CDE7304629F09CFFB0
:10A4E0000E9000210E982AF042F8012109900E9852
:10A4F0002AF03DF802210A900E982AF038F8020658
:10A500000B902CD500F07F0001230B9003210E98B7
:10A510008DF830302AF02BF804230D900B9E0F930A
:10A5200073067FF520AF06F03F064FF0010808FAEA
:10A5300006F808F1FF39022E0B96CDF8449028DC7E
:10A54000DDF83C9015AB4FF0000AD04509DC15ABA7
:10A550001093022303FA06F60F9B3344A4E7032368
:10A56000DCE749460E9803932AF001F809F102024C
:10A57000834609F101010E98009229F0F8FF039B30
:10A58000009A4BEA002023F8020B0AF1010A9146D7
:10A59000DBE7082E16DC002328A90E982893DDF8A7
:10A5A0003C802AF04DF90B9B082B0BDC50B10223A9
:10A5B000B340289A434493423FBF0F9BCDF8449049
:10A5C000C0181090DDF84080B8F1000FC1D10C49DF
:10A5D00051E700BF7AD30500B0E605005AD4050064
:10A5E00083D3050089D3050090D3050094D30500DB
:10A5F000A0D3050014010100A8D3050025D405004F
:10A60000F3D3050001229A40013A072B1292DCBFD6
:10A61000082292FBF3F203FB01F3D4BF02F1FF32F5
:10A62000002207331392DB10DDE90E1204A8149305
:10A6300024F0B7F8002C40F08C80BDF8613013F0A6
:10A64000700F1AD0DFF89CA3029E4FF0000844461A
:10A650000A9B029A1344B34279DC079829F026FC3E
:10A660000E9829F023FC17A819F046FAB5F80B301C
:10A6700003F50073A5F80B3001E7BDF87700BDF8CE
:10A680007910029B099ABDF87DC08742B4BF344659
:10A6900038463A448B42BDF87B30A8BF029902F19C
:10A6A000FF3EB8BF34469E45C8BF9E460A9A029BED
:10A6B000134403F1FF33C8BF34466345C8BF634644
:10A6C000BDF97FC0BDF98120C8BF34468445C8BFED
:10A6D000ADF87F00BDF98300C8BF34467045BCBFEC
:10A6E0003446ADF883E08A42BDF98520C4BFADF899
:10A6F000811034469A4202DAADF88530A2E7002C88
:10A70000A0D1DDF88BA09FE704A823F043FF083415
:10A7100040EA08280B9BA342F6DC129AE41A28FAB6
:10A7200004F313400D9A9A4209D0109A1AB1119964
:10A730000B4032F813303246494617A8D04709F18A
:10A740000109099B3B444B45E4DC013680E7B946EF
:10A75000F7E7204628F05BFC00283FF47EAF00229C
:10A760009D4920462AF028FF2CF0E2F8824621F08D
:10A7700000498B464FF0FF32984B5046494631F026
:10A7800087F870B94FF0FF32944B5046494631F08C
:10A7900075F830B9002200235046594631F05AF876
:10A7A00018B1DFF844B24FF0000A00228C4920466D
:10A7B0002AF002FF2CF0BCF8CDE90001DDE90083AE
:10A7C00023F000494FF0FF32844B404649464FF09A
:10A7D000010431F05DF840B94FF0FF327F4B404645
:10A7E000494631F04BF800B9044684F001044FF0BB
:10A7F000FF327A4B40464946E4B231F049F838B965
:10A800004FF0FF32754B4046494631F037F818B1EA
:10A810009FED6F7B8DED007B029B299309AE0FCEE0
:10A82000289731AF0FC70FCE0FC70FCE0FC796E8CF
:10A83000030004AE87E803000FCE3FAF0FC79DEDC6
:10A84000007B33683B6028A80023CDE92EAB8DED5B
:10A850002C7B8DF8C0408DF8C130F7F76FF8BDF84C
:10A860007780289BBDF879402A9F2B9E9845B8BFDA
:10A870009846299B9C42B8BF1C46BDF87B30013FDF
:10A880009F42A8BF1F46BDF87D30013E9E42A8BF33
:10A890001E46BDF97F309845BDF98330B8BFADF88D
:10A8A0007F809F42BDF98130C8BFADF88370A3425D
:10A8B000BDF98530C8BFADF881402246B34241465C
:10A8C00028A8B8BFADF88560FCF7AFF9BDF86130D6
:10A8D00013F0700F0CBFDDF88BA0DFF808A1B442B5
:10A8E00006DD3FAE0FCE04AC0FC433682360B4E680
:10A8F00028A8FCF791F9C146B94504DD28A8FCF762
:10A9000062F90134EBE74A9A7F322BD44B9B13F167
:10A910007F0B27D4449B9A4224DA459B9B4521DA3E
:10A920004FEA222C339A082A4FEA2B2BDDE9361006
:10A9300023D13C9A0CEB000302FB0B323FA827F01B
:10A940009BFE439B0BB13F9A9B5C359A9A4209D080
:10A95000389A1AB139990B4032F8133022464946D9
:10A9600017A8D0474A9B469A13444A93479A4B9B51
:10A970009B1A4B9309F10109BEE7319B03FB0BCBFB
:10A980000BFB02F200EBE2023FA827F075FE439BAF
:10A990000BB13F9A9B5C08213398814207DB3B9ABD
:10A9A00022EA0B0250433A9AC3401340CDE73FA836
:10A9B0000091029323F09BFB029B439A00991B0298
:10A9C0000AB13F98125C13430831E5E7054656E5A6
:10A9D0000000000000000000D5D50500FFFFEF7F5C
:10A9E000DBD50500DB3A04000000F03F70B594B001
:10A9F00004460E46014603A8154619F0A1F8C0B159
:10AA00003346BDF92420BDF92210009503A818F0A3
:10AA1000D3FF03A8ADF82260ADF8245019F06CF80C
:10AA2000B4F80B3003F50073A4F80B30204614B0D3
:10AA300070BD0446FAE7F0B595B004460D460146F0
:10AA400003A816461F4619F07BF898B11A9B00938D
:10AA500032463B46294603A818F0AEFF03A819F07A
:10AA60004BF8B4F80B3003F50073A4F80B30204614
:10AA700015B0F0BD0446FAE72DE9F04F99B006464F
:10AA80008946014607A819F05BF8B0B3BDF830401D
:10AA900004F460480FFA88FABAF1000FC4F30C040A
:10AAA0002EDA0022304930462AF086FD00222F4956
:10AAB000054630462AF080FD2BF0C6F8074648468A
:10AAC0002BF054FA00220146814602A823F069FEC9
:10AAD0000026A3000093B346DDE902218A4212D387
:10AAE000059829F0E3F9284629F0E0F9484629F0CD
:10AAF000DDF9B3455846B8BF304619B0BDE8F08F10
:10AB000000273D46DBE7069939B1895C0A2904D163
:10AB10005E45B8BF5E464FF0000BB8F1000F07D19D
:10AB20002046F6F7BFFD834402A823F0E0FAD3E7FE
:10AB3000B8F5005F02D1009B9B44F5E7BAF1000F26
:10AB4000F2DA2846019128F084FB48B10199B94214
:10AB5000EADBC91B284629F00AFD00FB04BBE3E73A
:10AB600028462AF0CFFAF8E772D5050077D5050018
:10AB7000F0B595B004460D46014603A816461F469B
:10AB800018F0DEFFA8B1079B01931A9B0093324691
:10AB90003B46294603A818F06CFF03A818F0ACFF49
:10ABA000B4F80B3003F50073A4F80B30204615B051
:10ABB000F0BD0446FAE7F0B595B004460D460146EF
:10ABC00003A816461F4618F0BBFFA8B1069B0193C9
:10ABD0001A9B009332463B46294603A818F049FFCA
:10ABE00003A818F089FFB4F80B3003F50073A4F83C
:10ABF0000B30204615B0F0BD0446FAE72DE9F04FC2
:10AC0000E1B00D4602901C4601469DF8A83115930F
:10AC100024A8924618F094FF002800F0A582BDF801
:10AC2000A43024A803F46042C3F30C090592FCF796
:10AC3000CBF9BDF914300C90002B119380F2938066
:10AC4000059BB3F5204F00F08C80B3F5404F14BF47
:10AC5000012304230022B049029803932AF0ACFC9C
:10AC600000220E90AD4902982AF0A6FC0022069020
:10AC7000AB4902982AF0A0FC2AF0E6FF04909DF868
:10AC8000AA20BDF89530ADF8583002F03002102AF5
:10AC90009BB270D183F03003BDF89720ADF89530AA
:10ACA0000AF10103A246D41A9DF8AA3003F0030367
:10ACB000012B0DD829460298FFF7DEFE9DF8AA3039
:10ACC00003F0030303FB000000EBD070AAEB600A63
:10ACD0009DF8AA30C3F38103012B9FBF0C9A03FB9D
:10ACE000022303EBD373A4EB6304BDF8AB300A93E8
:10ACF000BDF8AD300993BDF8AF300893BDF8B13061
:10AD00000793BDF89530DB0642BFDDE90923CDE9A5
:10AD10000932DDE90732284648BFCDE907232BF089
:10AD200025F90022129001461FA823F03AFD039A4C
:10AD300001239340013B18934FEA89031793C2F113
:10AD4000080356461D93DDE91F239A4245D21FA8EA
:10AD500023F020FC0A2805462BD10C9B56461C44A8
:10AD6000F1E7022376E701230022CDE90332002335
:10AD700006930E9383E7202A0ED183F06003BDF87B
:10AD80009720ADF895300AF10103A2EB030ABDF854
:10AD9000993001341C1B87E7302A85D183F050039A
:10ADA000BDF89920ADF89530631C5446A2EB030A18
:10ADB0007AE7059B002B40F092800146BDF8A40085
:10ADC000F6F770FC0A9B0B901B1AB34222DB0B9B1D
:10ADD0001E4422F089FD0028B5D0229829F066F89B
:10ADE000129829F063F806990E982AF0D2F8BDF867
:10ADF0005830ADF8953024A818F07EFE029B029AD8
:10AE0000B3F80B3003F50073A2F80B30029861B071
:10AE1000BDE8F08F089B9E42D9DABDF8A480099B5B
:10AE2000A3EB0803A342D2DA079B9C42CFDA202D82
:10AE3000CDD93C49059AA5F121033B4DDBB208462B
:10AE4000D7B29F422AD3C75C002DC0D03301083B44
:10AE50000D932301083B0F932F444FF00D0BBD4280
:10AE6000B5D015F8012BC82A22D8304B30499B5C4D
:10AE700014932E4B00205FFA80FE964513D3149B4B
:10AE80000DF1D40C01EB030E8E450CF1040C11D125
:10AE900035AA149924A818F0F3FBE0E711F8017B18
:10AEA00001323D44CCE713F801EB01307144E2E795
:10AEB0000021E4E711F8012BB2FBFBF00BFB1022A1
:10AEC0000D9BD2B212FB08F21A4402380F9B2CF8E9
:10AED000042C10FB08F018442CF8020CD4E7059B56
:10AEE000B3F5005F26D10A9B033BB34212DC089BFB
:10AEF0009E420FDA099B053BA3420BDC079B9C4259
:10AF000008DA159B2246CDE900933146034624A872
:10AF100018F0F2FE179B5BE76DD5050072D50500B2
:10AF200077D505004FC105002EC2050089C3050075
:10AF300052C40500119B002BBFF64BAF069828F0BA
:10AF400088F900285ED0049BAB4200F30A810DF122
:10AF5000D40800220699404623F023FC049B0027D6
:10AF6000ED1ADDE935239A4203D2379B1344AB42F5
:10AF700041DB399B002B43D013F80280389828F02E
:10AF800095FF0A9BA3EB0803B34245DA089B9E4258
:10AF900042DA099B0C9A9B1AA3423DDA079B9C421A
:10AFA0003ADA92FBF9F3039A139353435F43FA108F
:10AFB0000E9935A823F0F5FB399D07F007070DB171
:10AFC000359BED5C039B7B439D4006EB09030D9392
:10AFD00000230F930F9B434580F2BF800D9BA3EB93
:10AFE00009031B930D9B013B1C9304EB09030B937B
:10AFF0000023109377E0404623F0CCFA0744B0E7F3
:10B000009846BBE706982AF07DF8049BEF1AAB42FE
:10B01000804600FB07F7B4DD08FB0966D9E61D9BF7
:10B02000E8B21841159B0BB9002851D00B9B9DF835
:10B030009BC0A3EB09031A930B9B013B19930002DE
:10B04000189BB0FBF3F0B0F5807F0146A8BF4FF42A
:10B050008071BCF1080FDDE9273223D9BCF1100F54
:10B060004CD1C3F34510C1F5807EC2F3451C484363
:10B07000C3F3C42B0EFB0C0C01FB0BFBC2F3C4206F
:10B080000EFB00B0000A03F01F034B434FEA1C2CD9
:10B09000C00202F01F0240EA4C1C0EFB02324CEAD6
:10B0A00012230CE04FF48A7E2EFA0CFC1CF0010FE8
:10B0B00046D0C1F580704B4302FB00331B0A01935D
:10B0C000199B0093DDE91A211C9B24A818F0D1FCE0
:10B0D000039B1F44072F37DC9D40109B01331093C7
:10B0E0000B9B4B440B93109B139A934297DB0F9B44
:10B0F00001330F930D9B4B440D936BE7BCF1180F7D
:10B100001ED1C3F30720C1F5807EC2F3072C48434C
:10B110005FFA83FBC3F307430EFB0C0C01FB0BFB35
:10B12000D0B24B43C2F307422CF0FF0C0EFB00B031
:10B130000EFB02334CEA10201B0A40EA0343BEE731
:10B140007F28D8BF1346BAE735A822F0D0FF399D33
:10B150000DB1359BED5C0027BFE7389828F0A6FEBF
:10B160005AE74FF0000857E702904FE630B595B028
:10B170000546014603A818F0E3FCA0B128F06AFDDB
:10B18000044668B1094829F0FBFD014620462AF033
:10B1900026F901220094064B114628460CF02AF9A4
:10B1A000204615B030BD0446FAE700BF8BD4050039
:10B1B000B5B1020038B5054608460C4629F0F5FA47
:10B1C000072824D901221249204629F0FDF8F0B1C0
:10B1D0001049204629F000F9C8B90F49204629F046
:10B1E000FBF8A0B90D49204629F0F6F878B96FF0C0
:10B1F00000420721204629F0FEF904460146284670
:10B200002AF0D4F82046BDE8384028F04FBE38BDBB
:10B210009AD40500A2D40500B0D40500BDD4050021
:10B220002DE9F04F97B090460191014605A81F46C1
:10B2300018F086FC002856D0019828F00AF800285B
:10B2400079D00023092202A901988DF81030CDE9A8
:10B2500002332BF00BF89DF80C609DF809009DF867
:10B260000A909DF80B70002E40D122F065FD30F061
:10B270000BF80022904B30F09BF9044648460D46EF
:10B2800022F05AFD30F000F800228B4B30F090F99C
:10B29000824638468B4622F04FFD2FF0F5FF864B55
:10B2A000002230F085F9002206460F460023204692
:10B2B000294630F0C5FA88B9002200235046594685
:10B2C00030F0BEFA50B9002200233046394630F043
:10B2D000B7FA18B99DF80F30002B3BD00120774901
:10B2E00023F0E0FD002017B0BDE8F08F494622F0C2
:10B2F00038FD2FF0C9FF6EA3D3E9002330F058F9D1
:10B3000004460D463846314622F02BFD2FF0BCFF97
:10B3100067A3D3E9002330F04BF982468B469DF8B2
:10B320000D009DF80E1022F01CFD2FF0ADFF60A364
:10B33000D3E90023B5E701982BF00CF8404655EC13
:10B34000104B2BF007F838465BEC10AB2BF002F8F3
:10B3500057EC106B25F000494FF0FF32584B204658
:10B36000494630F095FA002840F09E804FF0FF32B9
:10B37000534B2046494630F081FA002840F0948033
:10B380002BF000494FF0FF324D4B5046494630F00C
:10B390007FFA002840F088804FF0FF32484B50463B
:10B3A000494630F06BFA00287ED127F000494FF073
:10B3B000FF32434B3046494630F06AFA002873D1D9
:10B3C0004FF0FF323E4B3046494630F057FA0028E6
:10B3D0006AD100223B4B204629462FF0BFFF30F0B8
:10B3E0006DFA0022374B0446594650462FF0B6FFFF
:10B3F00030F064FA0022334B0546394630462FF0D0
:10B40000ADFF30F05BFABDF8191011F4607184F3F0
:10B41000080385F3080280F3080008D0B1F5C07F67
:10B4200019D010D880291AD0B1F5807F1CD09DF892
:10B430001F1010291FD19110DA10D20242EA4112D6
:10B4400042EAE0004FE7B1F5007F11D0B1F5207F6F
:10B45000EDD1114601E019461346024606E01946B1
:10B46000034610460A46E2E7194603460846DEE769
:10B4700019461346F6E7202906D11B0443EA0223A6
:10B48000034343F07F402EE7182904D11B0443EA0D
:10B490000223184327E713440344B3F5C07F4FF05A
:10B4A000FF30B8BF00201EE7019829F02BFE1AE7F5
:10B4B0000000000000E06F4000002E4094D5050021
:10B4C000FFFFEF7F0000704070B5044608460D4650
:10B4D00027F09DFD002875D000223E4928462AF01D
:10B4E0006BF8064650B100231A4601462046FFF786
:10B4F00097FE394B1860304628F0D8FC00223749B7
:10B5000028462AF059F8064650B100231A4601464B
:10B510002046FFF785FE304B5860304628F0C6FCC9
:10B5200000222F4928462AF047F8064650B100234A
:10B530001A4601462046FFF773FE274B98603046B7
:10B5400028F0B4FC0022274928462AF035F80646A0
:10B5500050B100231A4601462046FFF761FE1E4BFC
:10B56000D860304628F0A2FC00221F4928462AF065
:10B5700023F8064650B100231A4601462046FFF73D
:10B580004FFE154B1861304628F090FC00221749F9
:10B5900028462AF011F8064650B100231A46014603
:10B5A0002046FFF73DFE0C4B5861304628F07EFCEC
:10B5B00000220F49284629F0FFFF18B12AF07DFC30
:10B5C000054B1876B4F80B3003F50073A4F80B3074
:10B5D000204670BD7CD5050008D30020D3DC0500D3
:10B5E0007FD5050083D5050087D505008BD50500DF
:10B5F0008FD50500F0B593B004460E46014601A86C
:10B6000015461F4618F09CFAF0B1AFB9049B2A46C4
:10B61000314601A818F061FA01A8ADF81A60ADF83A
:10B620001C5018F069FAB4F80B3003F50073A4F855
:10B630000B30204613B0F0BD00231A463946204691
:10B64000FFF7EEFD0346E2E70446F2E72DE9F04F8F
:10B650009DB00BAD80460F460146284616461C4657
:10B6600018F06EFA0290002800F09B80269B0A9347
:10B6700008AA07A92846CDE90776099418F07EF9AB
:10B680000AAA09A9284618F079F90798099B089988
:10B690000A9CC21802EBD27252101B1A009203EBE2
:10B6A000D3730A19641A5B1004EBD4746410059305
:10B6B0005B43039302EBD27204FB04F35210049336
:10B6C0000192DDE903326600013E03FB16260027E6
:10B6D000009B03EB070B019B03EB040A52460E9BF6
:10B6E0005946284618F0B8F8009BA3EB07095246C4
:10B6F0000E9B4946284618F0AFF8019BA3EB040ABD
:10B7000052460E9B5946284618F0A6F828460E9B2E
:10B710005246494618F0A0F8049A7B0003FB022227
:10B7200071009142BFBF049A0298033302FB036683
:10B730004FEA440C039BCCF1010203FB02F2B4BFBD
:10B7400001370020914208DD039AACF10303013C6C
:10B7500002FB1366002CBBDA01E00028FAD1059B3E
:10B76000BB4207F101040CDC284618F0C5F9B8F813
:10B770000B3003F50073A8F80B3040461DB0BDE850
:10B78000F08FDDE900120E9B2144284618F064F882
:10B79000DDE900120E9B091B284618F05DF82746CC
:10B7A000DDE7DDF80880E8E713B51C461344009395
:10B7B000121B0B19091BFFF749FF02B010BD2DE941
:10B7C000F04F9FB00DF1340A80460E4601465046B8
:10B7D00015461C4618F0B4F90390002800F0898043
:10B7E000289B0C930AAA09A95046CDE909650B9438
:10B7F00018F0C4F80CAA0BA9504618F0BFF8099924
:10B800000B9B0C9CCDF818A0CA1802EBD2725210F8
:10B8100002920A9A1519A41A5B1A04EBD4746410E4
:10B8200003EBD3735B10660005EBD575059304FB42
:10B8300004F95B43013E6D10049303FB1696002749
:10B840007B0003FB099271009142BCBF033309FBEB
:10B8500003660498B8BF039A4FEA44030793C3F101
:10B86000010300FB03F3B4BF0137002299421FDD3F
:10B87000029B069803EB070AA3EB070B109B2A1900
:10B88000CDE9002351465B4617F0AAFE109B0698AF
:10B890002A1BCDE9002351465B4617F0A1FE079B0A
:10B8A000049A033B013C02FB1366002CC8DA01E05A
:10B8B000002AFAD1059BBB4207F101040CDC0DA85C
:10B8C00018F01AF9B8F80B3003F50073A8F80B302C
:10B8D00040461FB0BDE8F08F109B0299CDE90053A0
:10B8E000029B2A461B1B21440DA817F079FE274610
:10B8F000E0E7DDF80C80EBE713B51C46134400933A
:10B90000121B0B19091BFFF75AFF02B010BDF0B54F
:10B9100099B004460F46014607A816461D4618F082
:10B920000FF9002840D01E9B069304AA03A907A87C
:10B93000CDE90376059518F021F806AA05A907A810
:10B9400018F01CF8049A0A9B0399CDE9002307A874
:10B95000059B17F045FE0A9B0193069B0093DDE9CA
:10B96000042307A8194617F03BFE069A0A9B039981
:10B97000CDE9002307A8059B17F032FE0A9B01932F
:10B98000049B0093039B069A194607A817F028FE0C
:10B9900007A818F0B1F8B4F80B3003F50073A4F859
:10B9A0000B30204619B0F0BD0446FAE72DE9F0430C
:10B9B000ADB000AF0023884607F108010646BB6022
:10B9C00028F03EFF0546AEB3F8B9304626F066FFD4
:10B9D0000446B86021F090FF04F58073834209D9D2
:10B9E0006D49012023F05EFA2E463046B437BD463D
:10B9F000BDE8F083E31D23F00703ADEB030D6D46B7
:10BA000022462946304627F06DF8B8F1010F14BFE1
:10BA10004FEAE80014204FF00009391DC7F80490E0
:10BA2000F5F7D0F97C6806463CB95C4823F01AF972
:10BA30002646DAE70028E8D1D7E7B8F1010F40F051
:10BA40008C805C22494607F15400D7F80880F3F750
:10BA500069FD534BFB6503F188333B6603F12943D2
:10BA6000A3F59613A3F68B637B66A3F18833BB66BD
:10BA70004C4BFB66B8F1000F05D04246294607F152
:10BA8000540016F021FC7A6DB96D530F43EAC103DF
:10BA90001BBAFB60D30002F03F02372A94BFC2F109
:10BAA0003805C2F178051BBA4022002107F11400C5
:10BAB0003B61F3F737FD80232A4607F1140107F1B4
:10BAC00054003B7516F000FC07F10C01082207F149
:10BAD000540016F0F9FB97F85F302370B7F85E302A
:10BAE0006370FB6D1B0AA370FB6DE37097F8633006
:10BAF0002371B7F8623063713B6E1B0AA3713B6E12
:10BB0000E37197F867302372B7F8663063727B6E23
:10BB10001B0AA3727B6EE37297F86B302373B7F83E
:10BB20006A306373BB6E1B0AA373BB6EE37397F833
:10BB30006F302374B7F86E306374FB6E1B0AA37406
:10BB4000FB6EE3740023194607F154021A440133D3
:10BB50005D2B3FF44AAF1170F6E7B8F1E00F06D164
:10BB600001232246B968284616F0E4FA3DE7B8F505
:10BB7000807F01D14B46F4E7B8F5C07F06D10123A1
:10BB80002246B968284616F043F92EE7B8F5007F3B
:10BB90007FF42BAF4B46F3E769D60500DFD20500F3
:10BBA00001234567F0E1D2C3024B034958680022E4
:10BBB00029F002BD482E002059CC050070B5174B66
:10BBC0001C7884420DD0FDF757F805462046FDF756
:10BBD00053F82A46034612490420BDE8704023F07A
:10BBE00061B9104C00201870206840B189B111462D
:10BBF00004F056F8206828F059F9002323600A4C15
:10BC0000206828F053F900232360084B01221A70A2
:10BC100070BD114604F08CF9ECE700BF00D30020A2
:10BC200028CC0500F8D2002004D3002021D3002026
:10BC300010B50A460C460021FFF7C0FF2046BDE8BC
:10BC4000104028F033B9000038B5194D2A884FF656
:10BC5000FF719142044613D001460320FDF726F8F8
:10BC600018B1144B186826F04DFF0446132128889C
:10BC7000F9F730F840F66B410EF0CCFE204638BDA7
:10BC80000D4B1D78022D0DD10C4829F079F8014695
:10BC90002846FFF7CDFFFAF792FF2046BDE838406F
:10BCA00006F058BC0649012023F0FCF8F5E700BF78
:10BCB000682D0020F8D2002000D30020CCCC050055
:10BCC000E1CC050010B5094B1C78012C0CD10021EA
:10BCD0000846FBF7D5FE064829F052F801462046F3
:10BCE000BDE81040FFF7A4BF10BD00BF00D3002087
:10BCF0003ACF05000A460021FFF760BFF7B50022E2
:10BD00003449044629F058FC29F09EFF324B334950
:10BD100006460322586829F04FFC054630B12246FA
:10BD2000B1B229F08CFB284628F0C0F800222C493B
:10BD3000204629F041FC0746002839D12146082039
:10BD4000FCF7B4FF18B90025284603B0F0BD254B19
:10BD5000254E186826F0D6FE33884FF6FF729A42B9
:10BD6000054607D1214829F00BF801460820FFF7C6
:10BD70005FFFE9E73A461749204629F01DFC29F004
:10BD800063FF013080B2ADF80400ADF8060001A9F0
:10BD900030880FF04DFA0EF04DFD04460028D3D048
:10BDA00001460820FFF7A6FF204628F07FF8CBE7E2
:10BDB00028F07CF800210920FCF778FF0028C2D089
:10BDC000084B186826F09EFE0121054620460FF01C
:10BDD000BFF9B9E706CD0500482E002013CD0500B8
:10BDE000FACC0500F8D20020682D0020E1CC050037
:10BDF00070B5014606460720FCF758FF68B3184B9C
:10BE0000184D186826F07EFE2B884FF6FF729A4276
:10BE1000044608D1144828F0B3FF01460720FFF775
:10BE200007FF204670BD00221049304629F0C4FBB0
:10BE300029F00AFF2B8881B2002218460FF0F6F98C
:10BE40000EF0F8FC05460028EBD001460720FFF76E
:10BE500051FF284628F02AF8E3E70446E1E700BF4F
:10BE6000F8D20020682D0020E1CC050006CD0500A9
:10BE70002DE9F04F85B00D4600AF002380463946CE
:10BE800028463B6028F0DCFC0446002D39D0F8B988
:10BE9000284626F003FD0646386021F02DFD06F504
:10BEA0008073834209D93749012022F0FBFF002625
:10BEB00030461437BD46BDE8F08FF31D23F007036D
:10BEC000ADEB030D6C4632462146284626F00AFEAD
:10BED00000210620FCF7EAFE0028E8D02A4B2B4D73
:10BEE000186826F00FFE2B884FF6FF729A4206461E
:10BEF0000AD1274828F044FF01460620FFF798FEA4
:10BF0000D6E70028E4D1D2E700222249D7F80090F2
:10BF1000404629F051FB29F097FE00221FFA80FAD3
:10BF20001D49404629F048FB834640B300221B4987
:10BF300029F042FB29F0C1FF8046584627F0B6FFA2
:10BF4000002398453B8114BF022301233B71391D17
:10BF5000012328887B71FC60A7F806A0A7F80A9047
:10BF60000FF0F4F80EF066FC04460028A0D001465D
:10BF70000620FFF7BFFE204627F098FF98E780468F
:10BF8000DEE700BF69D60500F8D20020682D00204A
:10BF9000E1CC050006CD05001ACD050025CD050034
:10BFA00038B50D4601460A20FCF780FE60B3174BFA
:10BFB000186826F0A7FD164B1A884FF6FF719142BC
:10BFC000044608D1134828F0DBFE01460A20FFF79B
:10BFD0002FFE204638BD18880F4B1B7880B28BB1DE
:10BFE00000232A461946F8F73DFC0EF023FC0546CF
:10BFF0000028EED001460A20FFF77CFE284627F0F5
:10C0000055FFE6E70820F0E70446E2E7F8D2002013
:10C01000682D0020E1CC0500B0CE0020000000001B
:10C02000F0B58BB06D460C46294616F0A3FA0028F1
:10C0300000F084800022012395E80300ADF8182069
:10C040008DF81830A023ADF81A303F4BADF80C1026
:10C05000CDE907323D4B0290090C58688DF80E105F
:10C060003B49099229F0A8FA29F0EEFDC3074CBF1D
:10C07000384B394B089320464FF0C873099326F08C
:10C08000C6FF002841D000223449204629F094FA06
:10C090002AF04EFC02460B4606460F462FF0F8FBF0
:10C0A00090B900222E4B304639462FF057F924A381
:10C0B000D3E900232FF07CFA00222A4B2EF098FFC0
:10C0C0002FF024FCADF8200000222749204629F05B
:10C0D00073FA2AF02DFC02460B4604460D462FF05B
:10C0E000D7FB90B900221E4B204629462FF036F987
:10C0F00013A3D3E900232FF05BFA0022194B2EF093
:10C1000077FF2FF003FCADF8220002AB93E80300A9
:10C11000ADF81410090C04908DF8161008AA06A9A1
:10C1200004A80FF087F80EF085FB044630B10146F5
:10C130000220FFF7DFFD204627F0B8FE0BB0F0BD70
:10C14000000000000088934090000400482E00206A
:10C15000A0D00500900120031000A00088D00500A9
:10C1600000408F400000E03F94D005000A460121C6
:10C17000FFF724BD70B50D4B1C78012C054613D17B
:10C1800000210846FBF77CFC2146094829F044F9C8
:10C19000064609F0BDFA304627F088FE29462046BB
:10C1A000BDE87040FFF7E2BF70BD00BF00D30020C4
:10C1B00004D300207CDF70472DE9F04F964C85B00A
:10C1C000236800AF054603F0040308460E463B60B3
:10C1D00026F01DFF002800F0AB8000228F4930467A
:10C1E00029F0EAF9B0B129F02FFD4FF47A735843E2
:10C1F00040F2712390FBF3F080B2B0F5804F884B92
:10C2000028BF4FF4804020281A8838BF202082425F
:10C2100018BF188000228349304629F0CDF938B183
:10C2200029F04BFE2368002862D023F400632360CA
:10C2300000227D49304629F0BFF938B129F03DFE92
:10C240002368002857D023F48053236000227749C5
:10C25000304629F0B1F98146002873D0002307F158
:10C260000C01FB6028F0ECFA8046002852D14846C9
:10C2700026F014FB8246F86021F03EFB0AF580733D
:10C2800083423BD96A49012022F00CFE484627F040
:10C290000DFE284626F0BBFE814608B9002D54D17C
:10C2A00031462846FCF74EFA002D40F0B2800025BA
:10C2B000604C614960682A4629F091FD32465F4929
:10C2C000606829F08CFD284627F0F0FD3B680BB133
:10C2D0000EF078FA4FF45B7140460EF09BFB3B6822
:10C2E00063B30EF025FC40F26E310EF093FB25E0B7
:10C2F00043F400639BE743F48053A6E70AF1070386
:10C3000023F00703ADEB030DE8465246414648468D
:10C3100026F0E8FB11234146BA893B7207F1080079
:10C32000FFF748FF40F22D3180460EF073FBADE77A
:10C3300046B132464249032022F0B4FD1437BD46CF
:10C34000BDE8F08F4FF00008A3E7284626F056FE20
:10C35000786000284BD0B5F80B3003F50073A5F8D2
:10C360000B30236823F07F7323F40033294607F151
:10C370000C00236021F028FECB46F86850B9B9F1D3
:10C38000000F95D0BBF1010F92DD236843F4003319
:10C3900023608DE728F098FE824626F038FE10B91B
:10C3A000BAF1000F0FD131465046FCF7CBF9814668
:10C3B000F86810B1494628F02DFD484627F076FD73
:10C3C000D7F8049009E0504626F018FE0028F7D16F
:10C3D000504626F0F6FD0028F2D1504627F066FDC3
:10C3E00007F10C000BF1010B21F0DDFDC5E728463C
:10C3F00026F0E7FD00283FF45AAFB5F80B3003F5FF
:10C400000073A5F80B30236823F07F7323F4003307
:10C41000BEE705464CE700BFFCD2002050D0050027
:10C420002C2D002059D0050065D0050041D805000D
:10C4300069D60500482E00206FD0050079D0050090
:10C44000BBCE050072DF7047F0B5284B284983B09A
:10C45000044600AF0246586829F0C1FC204626F089
:10C46000CDFD48B10023391D20467B6028F0E8F956
:10C4700005466CB970BB1BE0204626F0A2FD0028E3
:10C48000F0D1CCB122461B49032022F00BFD13E072
:10C4900000BB204626F002FA0646786021F02CFA0E
:10C4A00006F5807383420AD91349012022F0FAFC71
:10C4B0001249032022F0F6FC0C37BD46F0BDF31DF7
:10C4C00023F00703ADEB030D6D46324629462046A7
:10C4D00026F008FB00213B792A460846FFF7B2FF09
:10C4E00040F225410EF096FAE6E700BF482E002004
:10C4F0000ED1050043D1050069D6050017D105000E
:10C5000070B5294C29492068002229F055F80546C4
:10C5100018B1002101200EF029F9284627F0C6FCA9
:10C5200000222349206829F047F8054610B1012070
:10C530000EF086FE284627F0B9FC00221D496068EF
:10C5400029F03AF8002205461B49606829F034F8C2
:10C55000014606462846FFF72FFE2846314628F0BA
:10C5600018FD00221549606829F026F8054611F0EB
:10C570005FF8284627F09AFC60681149002229F0EC
:10C580001BF8044608B1FFF75FFF204627F08EFC3A
:10C590000EF0BEFC0B4B1B689B0503D5BDE870403D
:10C5A000FCF704BA70BD00BF482E002003D105007F
:10C5B000EFCC05006FD0050079D0050006D205004C
:10C5C0000ED10500FCD200202DE9F043B0F80B306D
:10C5D00091B003F500730446A0F80B3003A8884619
:10C5E000174616F0E3FF90B30121294816F096FB99
:10C5F000054648B31FFA88F027F044FB2549024658
:10C60000204628F0ACFF00222349204628F0D4FF22
:10C61000DDF82690009006461FFA88F3002239467E
:10C6200003A8C847002816DA1C49042022F03AFC67
:10C63000012027F01FFB1A490246204628F08FFFF1
:10C640002946304628F0A5FC03A816F04BFF2046EB
:10C6500011B0BDE8F083013027F014FB1149024608
:10C66000204628F07CFF022F0DD101210E4816F044
:10C6700055FB07460028E3D0214628F097FE3846B0
:10C6800027F014FCDCE72146284628F08FFED7E788
:10C690007BD7050021D9050004D3050093D70500F9
:10C6A000ACD70500B3D70500B8D7050037B5019062
:10C6B000B0F80B300C4C03F50073A0F80B300D46AE
:10C6C000214628F035FF294602220198FFF77CFF1A
:10C6D00027F0ECFB0198012301AA21461DF058FD2B
:10C6E000019803B030BD00BFFCD205002DE9F04732
:10C6F0008EB005468846164626F0ABFD814620B131
:10C7000028460021FCF700FE0546284626F07FFC5F
:10C71000044638B94648294622F0A4FA20460EB00D
:10C72000BDE8F087B8F1000F07D0404626F08AFC3C
:10C73000044610B941463F48EEE7022E16D101A843
:10C7400016F0DAFE90B100223B49284628F034FF6B
:10C7500029F07AFADDF80D30834204DACDF80D00C5
:10C7600001A816F0C2FE01A816F0BCFE0121334854
:10C7700016F0D4FA0746002858D0012E4BD1304984
:10C78000002020F08DFC044648B9384627F08EFB87
:10C79000B9F1000FC2D0284627F088FB2CE02949C8
:10C7A000002020F07DFCA2460446F4B1314620462C
:10C7B00016F0A6FAB8F1000F06D0234A41462046EB
:10C7C00028F04FFF27F072FB2146384628F0EEFD97
:10C7D000BAF1000F04D052461C49204628F0A8FEAA
:10C7E0002A461B49204628F0A3FE3946504628F029
:10C7F000D0FBB9F1000FCED1002E8FD101A816F0D9
:10C80000D5FE00288AD001A8214616F05FF801A8BD
:10C8100016F068FE82E7022E0CBF0E490E4900207A
:10C8200020F03EFC4FF0000A0446BEE70446E0E775
:10C8300019D705002FD6050049D7050058D70500A0
:10C840005FD7050067D705005ED60500BFE005008D
:10C8500004D305006FD7050074D70500F0B58FB07D
:10C86000054601A80F4616F0A1FEA0B3284626F003
:10C87000CEFB58B1194828F083FA194A01460446FC
:10C88000284628F0E1FE214628F083FB384628F0B0
:10C890001BFC064668B126F0D5FB044648B9114892
:10C8A000314622F0DFF9304627F000FB20460FB07A
:10C8B000F0BD304627F0FAFA012239462846FFF744
:10C8C00015FF044618B1014601A816F093F901A816
:10C8D00016F008FEEAE70446E8E700BF01D90500C4
:10C8E00005D905002FD6050070B592B004460D4657
:10C8F000014601A8164617F023F960B33EB140F295
:10C90000FF339D42A8BF1D46012DB8BF0125BDF9CB
:10C910001830002B11DA2B040FD41049204629F0CF
:10C920004DFA0F49204629F049FA0E49204629F0D0
:10C9300045FA0D49204629F041FA01A8ADF81850F2
:10C9400017F0DAF8B4F80B3003F50073A4F80B30E5
:10C95000204612B070BD0446FAE700BF6DD5050051
:10C9600072D5050095D4050077D505002DE9F8436B
:10C97000074608460D46144626F06BFC002800F0DA
:10C98000848001224249284627F01EFD0646C8B38E
:10C99000284627F00AFF062894BF4FF0FF384FF0D3
:10C9A00006083A21284627F0BFFD00282DDB00F1BC
:10C9B000010841466FF00042284627F01CFE29F08E
:10C9C00043F9B8F1010FB8BF4FF00108044608F170
:10C9D000FF322846002127F00EFE054641F6FF7380
:10C9E0009C42A8BF1C46012CB8BF0124BEB1A4B212
:10C9F000284627F05BFA324621463846BDE8F84320
:10CA0000FFF772BF4FF0FF38CBE7B8F1FF3FD0D14F
:10CA1000B5F80B3003F50073A5F80B30DEE715B958
:10CA200004F50054E3E7284627F0BFFE0028F7D0BE
:10CA30001849284627F0D0FC0028F1D1294616488D
:10CA400027F0EAFD324601468046384622F030FBA8
:10CA50008146B8B13346324639461EF0ADFF27F065
:10CA600025FAA4F50044A4B24146484628F091FABC
:10CA70004FF6FF739C42BBD12A460849012022F0A1
:10CA800011FAB5E74FF6FF74EEE7BDE8F88300BF93
:10CA900084D405008BD40500D1D40500DBD4050077
:10CAA00070B592B00546014601A817F049F868B381
:10CAB0009DF80830012B83BF154B1A6804924FF084
:10CAC000FF338EBF5B68049300230593BDF80B30E2
:10CAD000013BADF82330BDF80D30013BADF82530FA
:10CAE000079B03F44003002442F2010643F4702341
:10CAF00001A806960793ADF820408DF8224016F065
:10CB0000FBFF224631462846FFF7EEFE12B070BD0D
:10CB100008D3002010B5044694B019B1FFF7C0FF48
:10CB200027F0C4F9214603A817F00AF8C8B1079AFC
:10CB30000192BDF81520BDF81330013A0092002291
:10CB4000013B114603A816F04BFD03A816F0D4FFD5
:10CB5000B4F80B3003F50073A4F80B30204614B082
:10CB600010BD0446FAE710B592B00C46014601A884
:10CB700016F0E6FF60B1BDF8093003F010031CB1F8
:10CB800023B1BDF80B0003E0002BFAD0BDF80D0077
:10CB900012B010BD2DE9F04F99B006460D46014682
:10CBA00007A816F0CDFF044620B90024204619B08E
:10CBB000BDE8F08F8DB15C49284627F00DFC80461A
:10CBC00058B95A49284627F007FC044630B92A4686
:10CBD0005749012022F066F9E8E7A04600213046D7
:10CBE000FFF7C1FF012183463046FFF7BCFF9DF8E8
:10CBF000277000FB0BF47C4307340646E410B8F1C1
:10CC0000000F35D027F029F805460028CDD058462A
:10CC100027F038F847490246284628F0A0FC30465D
:10CC200027F030F844490246284628F098FC012FA6
:10CC300007D0384627F026F840490246284628F013
:10CC40008EFC9DF82030ABB9082F05D0BDF82130FF
:10CC500003F00F03042B0DD100223949079828F067
:10CC6000ABFC02463649284628F079FC2C469DE765
:10CC7000033445462046002128F02AF8044618B916
:10CC8000284627F013F991E70146002202A821F077
:10CC900088FDB8F1000F0CD15FFA8BF102A821F0EA
:10CCA000A8FBF1B202A821F0A4FB394602A821F0AA
:10CCB000A0FB0026B1463346B24627E01A4651464D
:10CCC00007A8009316F0EDFE0AF1010A09FA07F928
:10CCD000D34549EA000907EB0602009B02DC013359
:10CCE0004FF0000A16460AE0083E29FA06F1C9B2DA
:10CCF00002A8CDE9003221F07CFBDDE90032072EED
:10CD0000F2D8D6086FF0070101FB0626DDE9021212
:10CD10009142D3D3059827F0C9F8B8F1000F3FF43A
:10CD200045AF22469EE700BFE40B060065F3050011
:10CD300023D3050083D3050089D3050090D30500D4
:10CD4000B0E6050001381F289DBF034B23FA00F011
:10CD500000F00100002070478B80808030B551ECDE
:10CD6000100B85B053EC112B8DED000B55EC124BD5
:10CD70008DED021B2EF064FD9DED000B28B19DEDA5
:10CD8000021BB0EE410AF0EE610A53EC102B204674
:10CD900029468DED000B2EF053FD9DED000B08B1E3
:10CDA00045EC104B05B030BD38B555EC104B0022AA
:10CDB000002310EE100A29462EF042FD10B105F1B5
:10CDC00000431D4645EC104B38BD10B413460A46CF
:10CDD00053F8044B0021A4465DF8044B6047000063
:10CDE000024621B3012924D0022924D0032924D0CA
:10CDF000042924D0052924D0062924D0072924D0A9
:10CE0000082924D0092924D00A2924D00B2924D088
:10CE10000C2924D00D2924D00E2924D0134B1448DA
:10CE20000F2908BF03461349012022F03BB8124BDB
:10CE3000F9E7124BF7E7124BF5E7124BF3E7124B0A
:10CE4000F1E7124BEFE7124BEDE7124BEBE7124B1A
:10CE5000E9E7124BE7E7124BE5E7124BE3E7124B2A
:10CE6000E1E7124BDFE7124BDDE700BF5FDA0500B9
:10CE7000F6DA0500FEDA050067DA05006ADA050071
:10CE800073DA05007BDA050085DA05008DDA050026
:10CE900095DA0500A2DA0500A9DA0500AFDA050087
:10CEA000BEDA0500CEDA0500DCDA0500E8DA0500B6
:10CEB00052DA05002DE9F0478AB0804626F0C9F91C
:10CEC000044638B94849032021F0ECFF20460AB057
:10CED000BDE8F08700224146684621F062FC002749
:10CEE0003D463E463C464FF00009DDE900329A429D
:10CEF00025D8039826F0DAFF26F0AFFE0446002876
:10CF0000E4D0304626F0BEFE38490246204628F0DE
:10CF100026FB284626F0B6FE35490246204628F074
:10CF20001EFB05FB06F007300021C01027F0D0FEE5
:10CF30000546C0B9204626F0B9FF2C46C6E768462C
:10CF400021F028FB0A2805D159EA040308BF01276C
:10CF50000134C8E7AC4209F10109A8BF651C4E4580
:10CF6000B8BF4E46C1E73A464146684621F019FC33
:10CF70004FF0000847464FF08009DDE900239A4250
:10CF800008D3039826F092FF2A461A49204628F033
:10CF9000E6FA9BE7684621F0FDFA0A2803D108F17A
:10CFA00001080027E9E720281CD0284626F051F97F
:10CFB000C0B106FB087A29464FEADA0205A821F03B
:10CFC000F0FB099909B1059BC95C0AF0070A49FA07
:10CFD0000AFA41EA0A0105A8C9B221F03FFA089805
:10CFE00026F064FF0137C8E76ADD050083D305003A
:10CFF00089D30500B0E60500024B034958680022BA
:10D0000028F0DABA482E00200308060070B5002286
:10D0100086B00E46114928F0CFFA054626F019F9D8
:10D02000044660B10022294601A821F0BAFB002481
:10D03000DDE901239A4208D3049826F037FF2846F9
:10D0400026F034FF204606B070BD01A821F0A2FAF8
:10D05000B04208BF44F00104E4B2E9E713E105007F
:10D0600070B5044625F0D3FF30B90024254620468C
:10D0700026F01CFF284670BD00221449204628F0E7
:10D080009BFA054625F0C3FF044618B9284626F04A
:10D090000DFFEBE7002DE8D000220D49284628F0CF
:10D0A0008BFA044625F0CEFF50B1284626F0FEFE4E
:10D0B000002CDBD0074D2368EB1A5D425D41D6E7BB
:10D0C0002946204627F065FFCFE700BF97D9050026
:10D0D00075E70500B9240300014900201FF0E0BFF7
:10D0E00077BF0500014900201FF0DABFFBE1050012
:10D0F000014900201FF0D4BF49BF05002DE9F043CE
:10D1000090461D46421E47F6FE739A4293B006466D
:10D110000F4602D84A1E9A4208D93249012021F00E
:10D12000C1FE0024204613B0BDE8F0834046FFF75F
:10D1300009FE044620B92C49012021F0B3FEF1E795
:10D14000284625F064FFD8B100222849284628F057
:10D1500033FA002204462649284628F02DFA2546AF
:10D160008146284625F06EFF044688B92A462149A3
:10D17000012021F097FE4946284627F00AFFD1E713
:10D18000B5F80B3003F50073A5F80B308146E8E7DE
:10D19000B9F1000F06D0484625F054FF044608B9FF
:10D1A0004A46E4E7144900201FF07AFF04460028AD
:10D1B000B8D001238DF808303A464346314601A8DD
:10D1C00016F04AFD2A460D490194204628F0B0F990
:10D1D0004A460B49019828F0ABF901A816F08CFCDF
:10D1E000C9E700BFF7DC050004DD050010DD050020
:10D1F00019DD050022DD05007AD3050056DD0500A6
:10D2000060DD050070B506460D4626F022F804469E
:10D2100030B932461349032021F044FE204670BD48
:10D22000114900201FF03CFF32461049044628F007
:10D230007FF945B1284626F00CF868B9324609490D
:10D24000032021F02FFE002026F01CFD0849024695
:10D25000204628F084F9E1E72A460649204628F0CE
:10D2600067F9F0E7D0E00500FBE0050002E105000A
:10D2700009E1050013E1050038B50022084905461B
:10D2800028F09AF9044640B906491FF009FF0449FD
:10D2900004460246284628F04BF9204638BD00BF18
:10D2A000E2150600C3E005002DE9F04391461D4656
:10D2B000421E47F6FE739A4293B00746884602D84C
:10D2C0004A1E9A4205D96749012021F0EBFD00244E
:10D2D00008E04846FFF736FD044638B962490120A8
:10D2E00021F0E0FD204613B0BDE8F0835F49002047
:10D2F0001FF0D6FE04460028F4D0002601A84B46B5
:10D30000424639468DF8086016F0A6FC28468DF88E
:10D3100009608DF80A60019425F079FE00285CD040
:10D3200032465349284628F047F928F0C6FD28B16F
:10D33000BDF8093043F00103ADF8093000224D4932
:10D34000284628F039F928F0B8FD28B1BDF8093091
:10D3500043F00403ADF8093000224749284628F07D
:10D360002BF928F0AAFD28B1BDF8093043F00803D5
:10D37000ADF8093000224149284628F01DF928F06F
:10D380009CFD88B19DF80F0001280BD1BDF8093034
:10D3900043F00203ADF80930BDF80D305B0703D050
:10D3A000374992E737498FE728460022364928F067
:10D3B00003F9054688B1354927F00EF850B93449CC
:10D3C000284627F009F808BBBDF8093043F0800370
:10D3D000ADF80930284626F069FDBDF80D00BDF80E
:10D3E0000B3043439DF80F0058430730C0080BF043
:10D3F00075FD284A05460146019828F032F929466C
:10D4000027F0C7FD01A816F077FB6BE722492846F5
:10D4100026F0E2FF20B9BDF8093043F48073D7E766
:10D420001E49284626F0D8FF20B9BDF8093043F43C
:10D43000C073CDE71A49284626F0CEFF20B9BDF8C3
:10D44000093043F40073C3E71649284626F0C4FFA9
:10D4500020B9BDF8093043F42073B9E7124821F030
:10D46000E1FBB7E7F7DC050004DD05007AD3050032
:10D4700024DC05002BDC05002FDC05003BDC05006F
:10D4800079DC050049DC0500B2DC0500BEDC0500E6
:10D49000C2DC0500B0E60500C6DC0500CADC0500FC
:10D4A000CEDC0500D2DC0500D6DC05000000000063
:10D4B00008B500222DED028BB0EE408AF0EE608AB6
:10D4C000002351EC100B2EF0CFF998B1B0EE480AC2
:10D4D000F0EE680A2BF090FF0B4B51EC100B002282
:10D4E0002DF03CFFBDEC028B41EC100BBDE8084079
:10D4F0002BF0FEBEBDEC028B9FED010B08BD00BF03
:10D50000000000000000F87F0000E03F0000000085
:10D51000F8B555EC104B25F000474FF0FF32284B83
:10D52000204639462EF0B4F960B94FF0FF32244B53
:10D53000204639462EF0A2F920B9B5F1004F08BFB8
:10D54000002C05D145EC104BBDE8F84026F088BB17
:10D5500000220023204629462EF072F9C8B912A1F4
:10D56000D1E900012B4622462DF042FD06460F462A
:10D570002EF054FA04460D4654EA05030DD100225C
:10D580000023304639462EF05BF930B19FED080B91
:10D59000DAE709A1D1E90001E4E720462946BDE820
:10D5A000F84026F084BB00BF2083E4FFFFFFDF3F8D
:10D5B00000000000000000802083E4FFFFFFDFBFC9
:10D5C000FFFFEF7F2BF090BE2BF012BB38B555EC70
:10D5D000104B10EE102A2B4610EE100A29462DF0A3
:10D5E000BDFE02460B46002009492DF0FFFC41EC30
:10D5F000100BFFF75DFF204653EC102B29462DF052
:10D60000D7FFBDE8384041EC100B2BF0F1BA00BF5A
:10D610000000F03F2BF008BE08B50B464022014643
:10D62000184628F023FE402805D10120034921F0A7
:10D6300039FC002008BD0120FCE700BFF7D9050038
:10D6400070B50E46044600220D49304627F0B4FF5F
:10D65000054628B90024284626F028FC204670BD3F
:10D6600025F032FD0028F5D0284625F037FD26604C
:10D67000606090F82642631E5C425C41EBE700BFAD
:10D68000CBD9050030B591B0054625F00FFE044614
:10D6900038B92A461F49032021F004FC204611B066
:10D6A00030BD0122294605A821F027FE00231A4695
:10D6B00005A9194817F035FF044605A820F010FC0D
:10D6C0002046002127F004FB044618B9134821F036
:10D6D000C9FAE3E72946012205A821F00EFE2146FA
:10D6E0000022684621F05DF86B460D4A0A4805A9FC
:10D6F00017F017FF039826F0D9FB05A820F0F0FBE0
:10D700000021204627F0DBF80546204626F0CEFB18
:10D710002C46C3E77DDD0500A1770400DFD20500BC
:10D72000C377040030B591B0054625F0BFFD04462F
:10D7300038B92A461F49032021F0B4FB204611B016
:10D7400030BD0122294605A821F0D7FD00231A4645
:10D7500005A9194817F0D9FF044605A820F0C0FB19
:10D760002046002127F0B4FA044618B9134821F0E6
:10D7700079FAE3E72946012205A821F0BEFD2146FA
:10D780000022684621F00DF86B460D4A0A4805A9AB
:10D7900017F0BBFF039826F089FB05A820F0A0FB3B
:10D7A0000021204627F08BF80546204626F07EFB18
:10D7B0002C46C3E77DDD0500A1770400DFD205001C
:10D7C000C3770400F8B5051E0C4606DC2949012084
:10D7D00021F068FB00242046F8BD084625F017FC20
:10D7E0000646A8B100222449204627F0E5FE28F08D
:10D7F00064FB002221490646204627F0DDFE28F082
:10D8000023FA30F0080309D0102809D01C49DEE7BC
:10D8100024B122461B49012021F044FB012400E0F1
:10D8200002242946204626F067FB07469EB129467A
:10D83000204626F061FB0546134900201FF030FC0E
:10D84000044610B10FB146B13DB92A4639462046CB
:10D8500027F092FBBEE73546EEE73A460B492046F5
:10D8600027F07DFE002DB6D02A460949204627F034
:10D8700076FEB0E73EE305005DE305007CE30500CE
:10D880006AE3050081E30500B8E30500B0E60500A2
:10D89000C1E3050038B5044625F0B9FB88B1002284
:10D8A0000949204627F088FE054625F0D2FC10B134
:10D8B000284626F07AFF0446284626F0F7FA204646
:10D8C00038BD0446FBE700BFE9E20500F8B50646AF
:10D8D0000D460AB3104627F015FC002D044603DA66
:10D8E000304626F062FF0544002C03DA304626F06D
:10D8F0005CFF04441B2026F035F925EAE57524EA8F
:10D90000E474074630B1A54204DA631B2A46314667
:10D9100026F044FE3846F8BD00296FF00044E9DAED
:10D92000DEE7F8B505460C46C2B1104627F0EAFB23
:10D9300020EAE076002C05DA284626F036FF04447B
:10D9400024EAE4741B2026F00DF9074620B1334683
:10D950002246294626F022FE3846F8BD6FF00046E2
:10D96000E8E7F8B507460C46CAB1104627F0CAFBEF
:10D9700020EAE07524EAE474A542B8BF23464FF0DC
:10D980001B00BCBF2C461D4626F0ECF8064620B115
:10D990002B1B2246394626F001FE3046F8BD6FF0BB
:10D9A0000040E5E770B50D1E064606DA0B4901207A
:10D9B00021F078FA0024204670BD1B2026F0D2F812
:10D9C000044615F1FF35F6D31FF08EFF0028F2D183
:10D9D0003146204626F00AFEF3E700BF2AE30500A1
:10D9E000F8B506460F46154625F033FC044698B1B7
:10D9F000284625F04DFB88B1284627F083FB0446D6
:10DA0000384628F0B3FA054626F0CFFE241A09D589
:10DA10000024284626F04AFA2046F8BD304626F073
:10DA2000C4FEECE7284626F0C0FE0719304626F073
:10DA3000BCFE8742ECDC2246012329463046F2F741
:10DA400063FEB0FA80F46409E3E7F8B507460E46D2
:10DA5000154625F0FEFB044648B1304628F086FA0C
:10DA6000002D064605DA0024304626F01FFA20462F
:10DA7000F8BD26F09AFE4419384626F096FE8442F8
:10DA8000F1DC01232A4631463846F2F73DFEB0FA72
:10DA900080F46409E8E72DE9F04186B028F066FAE1
:10DAA0000546E0B10146002201A820F07AFE4FF0C1
:10DAB000FF340026DDE90183984514D3049826F04D
:10DAC000F5F9A642DABFA21B0132002231462846F0
:10DAD00026F091FD0446284626F0E8F9254628461A
:10DAE00006B0BDE8F08101A8039F20F053FD20F0AF
:10DAF00055F90028DED107EB080336EA240628BFD3
:10DB00001E461C46D6E708B508B1036823B91B209A
:10DB1000BDE8084026F026B8002127F0E3FABDE86A
:10DB2000084028F022BB08B526F021FD08BD70B5DD
:10DB3000054686B01B200E4626F014F80446E0B1D8
:10DB4000284625F086FBC0B1002E16DB324629465A
:10DB500001A820F026FEDDE901239A420AD2059BA6
:10DB600003B19B5C8DF8033001220DF103012046C7
:10DB700026F094FD049826F099F9204606B070BD71
:10DB800037B505461B2025F0EDFF044628B1294690
:10DB900001A820F019FA019810B9204603B030BD51
:10DBA00027F092FA28F050F801228DF803000DF1C9
:10DBB0000301204626F072FD01A820F0F4F9EAE7FF
:10DBC000F8B507460E4625F022FA88B30022194917
:10DBD000384627F0F1FC054625F03BFB18B32846F4
:10DBE00026F0E3FD002E01DD86420AD311493846B6
:10DBF00028F0E4F82C460025284626F057F9204660
:10DC0000F8BD32460021284626F0F5FC3146044690
:10DC10006FF00042284626F0EEFC064902463846E0
:10DC200027F09DFCE8E71B2025F09CFF0446E3E776
:10DC30000446E4E7E9E205002DE9F041CB1D23F0BD
:10DC4000070300AFADEB030D134614466E460D46B9
:10DC500053F8048B0A463146C047A3692B44A3619D
:10DC600063692B44636135441C34AE4202D1BD4626
:10DC7000BDE8F081204616F8011B20F0F6FB204697
:10DC800020F05BFAF1E700002DE9F04F93B000AF10
:10DC90000E46154681461CF0D7FA4FF0010A04469D
:10DCA00007F11701304687F817A0F3F723FE002D80
:10DCB000804606DC4FF0000840464C37BD46BDE8C4
:10DCC000F08F1FF019FE05F58073834204D9604977
:10DCD000504621F0E7F8EDE7EB1D23F00703ADEB2D
:10DCE000030D122C6E463BD15A4B1B78CBB100234F
:10DCF00007F120024FF040215748C7F82230C7F8FB
:10DD000026307B8587F820A087F8218087F822506D
:10DD10007E62F7F767FC024618B15049042021F0F3
:10DD2000C1F82946012026F0E7F880460028C1D036
:10DD30000146002207F1200021F0B0FA354416F820
:10DD4000011B07F1200020F090FB07F1200020F0DC
:10DD5000F4F9B542F3D107F1200020F0BBF8ABE7AE
:10DD6000002CA7D13E492246484627F025FC824692
:10DD7000014607F118001BF0CDFC00285CD02246BC
:10DD80003849484627F018FC28F097F83B7FB877C9
:10DD9000FF2B51D07A7FFF2A4ED087F8212087F8B9
:10DDA0002030BA69304B93FBF2F37B62FB7FF97D45
:10DDB00087F82200002B07F120002C4BF96008BFE8
:10DDC0000023BB621BF06CFC4FEA480101F4FF71B9
:10DDD00041F0010107F120001BF01AFC60B305F1CE
:10DDE000FF38A8EB04035942594108224FF0000BB9
:10DDF00007F12000C7E901121BF0AAFBBA68796895
:10DE00004FEA4B0B013A40EA0B0BF1D107F120002E
:10DE10001BF0CEFB97F821001BF08AFB06F804B03C
:10DE20000134A542DDD1FB681BB107F120001BF0D6
:10DE300001FC97F82230BB77B87F25F01BFF09491A
:10DE40000246484627F074FB514627F0A2F868E7DF
:10DE5000A2DD0500D8D200207CCB0020D7DD050054
:10DE6000EADD0500F3DD050090D00300A086010087
:10DE70002DE9F04F89B000AF0D46904606461CF0E4
:10DE8000E3F94FF0010AF91D0446284687F807A078
:10DE9000F3F730FD0023834607F108014046BB60DD
:10DEA00026F0CEFC0546B8F1000F43D0F0B940464D
:10DEB00024F0F4FC8146B8601FF01EFD09F5807364
:10DEC000834207D94949504620F0ECFF2437BD462C
:10DED000BDE8F08F09F1070323F00703ADEB030D55
:10DEE0006D464A462946404624F0FCFDBB68002B9F
:10DEF000ECD0122C21D13E4A1278002AE6D0F979D2
:10DF00003C48BD61002291427A61FA61BB754FF0D5
:10DF1000402114BF1346202307F1140287F815B0DF
:10DF2000F7F760FB02460028D0D03349042020F0E8
:10DF3000B9FFCBE70028C9D0D8E7002CC6D12F49BC
:10DF40002246304627F038FB8046014607F10C0098
:10DF50001BF0E0FB60B322462949304627F02CFB3A
:10DF600027F0ABFF3B7CB874FF2B21D07A7CFF2AD3
:10DF70001ED07A753B75FA68224B93FBF2F3BB61B6
:10DF8000FB7CB875002B07F114001F4BD7F808A0D5
:10DF900097F8079008BF0023FB611BF081FB4FEA55
:10DFA0004B0101F4FF7107F114001BF031FB88B93C
:10DFB000B87C25F05FFE12490246304627F0B8FAD9
:10DFC000414626F0E6FF81E7295D07F114001BF0CA
:10DFD0001FFB0134A245F7DCB9F1000F03D007F1B4
:10DFE00014001BF027FBBB7DBB74E1E769D605007D
:10DFF000D8D200207CCB002047DE0500EADD0500FA
:10E00000F3DD050090D00300A08601002DE9F74F55
:10E010000D4603210446CDE9002313F021FC4FF007
:10E02000000B4FF0010A4FF08008D94615F1FF357B
:10E0300002D203B0BDE8F08F009B0AEA0306019B01
:10E040000BEA030756EA070316D088F3118800216C
:10E05000204613F09BF90A20F3F7A6FD0121204684
:10E0600013F094F989F311883720F3F79DFD1AEB2B
:10E070000A0A4BEB0B0BD9E788F3118800212046E5
:10E0800013F084F94120F3F78FFD0121204613F0AE
:10E090007DF989F311880520E7E710B40C78024672
:10E0A0000023204608215DF8044BFFF7AFBF0000B6
:10E0B0002DE9F04F89B0894600901CF0C5F849461B
:10E0C000044602A81BF026FBF0B1122C40F0F880A9
:10E0D0009DF80C4020461CF0CDF99DF80D5018B16C
:10E0E00028461CF0C7F990B922462946854820F0F9
:10E0F000B9FDB9F1000F00F00081834A009849464C
:10E1000027F0A2FA25F0D2FE09B0BDE8F08F7F49D2
:10E11000029E7F4B04EB840405EB85050C440D4403
:10E120009E4294F801806F7858DD7A4B9E42D4BFAE
:10E130004FF080664FF0CD66774A784C13785BB32A
:10E1400023681BB1764B1021C3F880104FF0402399
:10E150004FF0FF31C3F80813D3F800120021C3F8C1
:10E160000012C3F80015012184F8221094F827103A
:10E1700079B9D3F808154FF0A04001F5E07140F2ED
:10E18000023540F82150D3F80C3503F5E07340F820
:10E190002350002384F8223094F822300125157092
:10E1A000FBB108225F49042020F07CFE9DF80C4062
:10E1B00020461CF05FF920B14FF42071204613F087
:10E1C00031FB9DF80D4020461CF054F9002890D0FA
:10E1D0004FF49451204613F025FB8AE74FF0CC769C
:10E1E000AAE79DF81E2084F827209DF81D20A36033
:10E1F000C4E9003384F8253084F8243072B34FEA40
:10E200008800B90000F1A04001F1A04140F20C6289
:10E210004FF0A04BC0F8002705FA08FAC1F8002714
:10E22000BD4040F20D620193CBF808A5CBF808552C
:10E23000C0F80027C1F800270420F3F771FC019B08
:10E24000DBF810150D422BD043B14FF0A04A04204B
:10E25000CAF80C55F3F764FCCAF808554FF0A04310
:10E2600008F5E07140F20C6243F8212007F5E071F7
:10E2700043F821204FF040231D46C3F80885C3F81A
:10E280000C75C3F8246522681AB106210420F7F73B
:10E2900085FB0523C5F80035022384F8223085E785
:10E2A00001930420CBF80CA5F3F73AFCCBF808A5B2
:10E2B0000420F3F735FC019B0133092BC0D1C4E7DF
:10E2C000002C7FF416AF9DF80C00FF2807D0012129
:10E2D00013F05CF803219DF80C0013F0C1FA9DF8CF
:10E2E0000D00FF283FF405AF012113F04FF8032183
:10E2F0009DF80D0013F0B4FAFBE60349009827F0EF
:10E300005DFD01E7FBDD0500EADD050040C005001D
:10E3100097AB020087F50400D8D200207CCB002008
:10E3200000E100E02ADE0500F0B58DB00D4616468E
:10E330001C461BF089FF11289DF8487005D02F4915
:10E34000012020F0AFFD0DB0F0BD16B90CB90F24BF
:10E3500003262B4B1B78F6B2E4B25BB92949ADF822
:10E3600010306FF0FF02CDE9011201A8264A039296
:10E370000DF00AFDFF2F03D0002138461CF01CFDD4
:10E38000284624F085FE80B1284626F0BBFE2246B2
:10E390003146C0B2F3F7D6F8F2F7FEFEFF2FD2D027
:10E3A000012138461CF008FDCDE7284624F07EFF09
:10E3B000E8B1802383F311880122294601A820F0C7
:10E3C0009CFF01A81FF0B8FD054601A825B91FF064
:10E3D00087FD85F31188DFE71FF093FF2246314662
:10E3E000C0B2F3F7AFF801A81FF0C1FEE9E72A4673
:10E3F0000649012020F056FDCEE700BFFFE10500F1
:10E40000BCD20020A08601000001080027E2050020
:10E41000F0B58DB00D4616461C461BF015FF1128B1
:10E420009DF8487005D03049012020F03BFD0DB02B
:10E43000F0BD16B90CB9032401262C4B1B7806F04D
:10E440000F0604F00F045BB92949ADF810306FF0E6
:10E45000FF02CDE9011201A8264A03920DF094FCB7
:10E46000FF2F03D0002138461CF0A6FC284624F0DC
:10E470000FFE80B1284626F045FE22463146C0B246
:10E48000F3F720F8F2F788FEFF2FD0D001213846AD
:10E490001CF092FCCBE7284624F008FFE8B180236B
:10E4A00083F311880122294601A820F026FF01A844
:10E4B0001FF042FD054601A825B91FF011FD85F3A7
:10E4C0001188DFE71FF01DFF22463146C0B2F2F788
:10E4D000F9FF01A81FF04BFEE9E72A460649012093
:10E4E00020F0E0FCCEE700BFD7E10500BCD2002061
:10E4F000A08601000001080027E20500F0B58BB0FE
:10E5000004460D461BF0A0FE01AE074632466946A2
:10E5100020461BF0A7FE98B3009B059396E80F00DA
:10E5200006AC07C423807DB3296800292CDD01399E
:10E53000284626F0D7FD064624F084FF10B3304667
:10E540001BF020FF0446284627F002FC25F0AEFC15
:10E55000304625F0ABFCFF2C03D0002120461CF0F8
:10E560002BFC05AA0949284624F09EF8112F01D159
:10E57000F2F712FEFF2C03D0012120461CF01CFCF8
:10E580000BB0F0BDFF24E3E7FF24EAE7CBCD0200A8
:10E590002DE9F041B8B00D46164607A908AA1BF0B0
:10E5A00061FE002877D0FF2E03D0002130461CF0FA
:10E5B00003FC284624F06CFD80462846B8F1000F85
:10E5C00018D026F09FFD18A98DF8600008AB08460A
:10E5D0000122079CA0479DF8600025F053FB0446EC
:10E5E000FF2E03D0012130461CF0E6FB204638B058
:10E5F000BDE8F08124F02DFE0746002831D01B2015
:10E6000025F0B0FA42460446294602A820F0C9F88F
:10E61000DDE902239A4203D3059825F047FCDFE7A2
:10E620001FF062F90028F7D101AA694602A81FF07D
:10E6300035FD019D002DEBD0802D28BF802508AB36
:10E640002A4618A90098079FB8472A4618A92046C5
:10E6500026F024F8019B5B1B0193009B1D44009551
:10E66000E7E7284624F01AF90146012025F044FC8A
:10E6700004460028B4D03A4601460EA8CDE90C77EE
:10E6800020F00CFE07AA0549284624F00DF80EA834
:10E690001FF020FCA4E70446A8E700BF39DC020015
:10E6A0007FB50C4605461BF0CFFD21460646684661
:10E6B0001AF026FD60B1112E0CD168460DF064FBF6
:10E6C00004B3134A2146284626F0BEFF25F0EEFB90
:10E6D00004B070BD002EFBD19DF80500FF2802D0CC
:10E6E000012113F0BDF89DF80600FF2802D0042197
:10E6F00013F0B6F89DF80700FF28E1D0012113F0D0
:10E70000AFF8DDE70249284627F058FBE0E700BFF5
:10E71000EADD05002DE9F04300228DB024490646CC
:10E7200026F04AFF05AD0146284628F08BFE1B2245
:10E73000541E295D09B1144602E02246002CF7D18F
:10E740000CAB4FF001081C440DF1240904F81C8C9B
:10E7500099E807008DE8070095E80F0028F0C3FC52
:10E7600008F1010807460028F0D1012025F08AFAB7
:10E7700010490246304626F0F2FE384625F082FA6D
:10E780000D490246304626F0EAFE384625F07AFA70
:10E790000A490246304626F0E2FE384625F072FA73
:10E7A0000749024630460DB0BDE8F04326F0D7BE1B
:10E7B00041D8050078E205007EE2050085E205000B
:10E7C000C4F005002DE9F04F0022A1B00E466E49BD
:10E7D000054626F0F1FE27F037FAC0B2722808D0BD
:10E7E0006A49012020F05EFB0027384621B0BDE8D1
:10E7F000F08F00226649284626F0DEFE27F024FA34
:10E800008046002800F0BD8000226249284626F09C
:10E81000D3FE27F019FA00225F498146284626F0E8
:10E82000CBFE27F011FA00225C498246284626F0EA
:10E83000C3FE27F009FA002259498346284626F0EC
:10E84000BBFE014609A828F0FDFD1B22531E09A9A5
:10E85000C95C09B1134602E01A46002BF6D120AA82
:10E86000D318069303F85CBCF30F059318BF20265A
:10E8700000273EBB7CE04FF0000846E012F8011B89
:10E88000FF291CD00598013300286CD00A296AD1D1
:10E8900000221C46059237B91B20079325F062F928
:10E8A000079B074630B1224610A93846079325F04A
:10E8B000F5FE079B059AA1441AB91E1BD9E71C4611
:10E8C00054E02026AAEB0904002C3DDCBBF1FF0F2D
:10E8D000D1D0069B0BF1010B03F85CBC18AB039382
:10E8E0000DAB93E807008DE8070009AB0FCB28F0CC
:10E8F00008FB189B23F07F4A8046504625F0C2F95A
:10E9000025490246284626F02AFE404625F0BAF957
:10E910001F490246284626F022FE002025F0B2F9C3
:10E920001C490246284626F01AFE584625F0AAF948
:10E930001A490246284626F012FEB8F1000F3FF4AD
:10E9400054AF54464FF00009202E3346A8BF202371
:10E950009C42A8BF1C46224609EB080110A82DF0D6
:10E9600011FA10AA0023A34288DB3346002C92D16F
:10E97000484625F087F907490246284626F0EFFD6C
:10E9800033E7074631E700BFC4F005008AE205001F
:10E9900085E205007EE20500A2E2050078E20500BE
:10E9A00041D805004FF0FF31FFF70CBF21EAE171BC
:10E9B000FFF708BF2DE9F04F00229BB00C469B49A2
:10E9C000054626F0F9FD27F03FF9C0B2772808D0B8
:10E9D000612806D09649012020F064FA1BB0BDE8FA
:10E9E000F08F204627F0C2FA07460028F6D025F01F
:10E9F000DCFE81460028F1D000228E49284626F010
:10EA0000DBFD27F021F900228B498246284626F0BB
:10EA1000D3FD27F019F9002288498346284626F0BD
:10EA2000CBFD27F011F9002285498046284626F0C3
:10EA3000C3FD0BAC0146204628F004FD1B22531EEB
:10EA4000E15C09B1134602E01A46002BF7D11AAA7D
:10EA50001A44CDE9082302F83C8C7A490022284662
:10EA600026F0AAFD27F0F0F80646002845D0099BBD
:10EA7000A0F120020DF1480E10685168F446ACE890
:10EA800003000832B242E646F6D15A1C214613A8CA
:10EA90002DF06AF9A8B112AB03930FAB93E807000E
:10EAA0008DE8070094E80F0028F02BFA064608B915
:10EAB000654990E725F0E6F862490246284626F0C7
:10EAC0004EFDABEB0A0BD94556444FDB5A460021AD
:10EAD000384625F090FD3146824607F0CFFB504680
:10EAE00025F0E4F9B8F1FF0F4BD15849012020F08F
:10EAF000D9F9384625F0DAF970E74FF47E63CDE9AD
:10EB000005034023CDE903730FAE96E807008DE8B7
:10EB1000070094E80F0028F027FB0028E9D012AB8B
:10EB2000039396E807008DE8070094E80F0028F0AB
:10EB3000E8F90646129820F07F44484625F0A2F8EE
:10EB40003C490246284626F00AFD204625F09AF860
:10EB500039490246284626F002FD304625F092F853
:10EB600038490246284626F0FAFCC2E738463146C4
:10EB700007F084FB09EB0A0025F084F82D490246D2
:10EB8000F0E7089B08F1010003F83C0C25F07AF847
:10EB90002A490246284626F0E2FC6FF00042594618
:10EBA000384625F028FD00234FF47E62CDE905327A
:10EBB0004023CDE903030FAE804696E807008DE8B9
:10EBC000070094E80F0028F0CFFA002891D012AB8C
:10EBD000039396E807008DE8070094E80F0028F0FB
:10EBE00090F90646129820F07F44484625F04AF8EE
:10EBF00010490246284626F0B2FC204625F042F88D
:10EC00000D490246284626F0AAFC304625F03AF87F
:10EC10000C490246284626F0A2FC404625F0C5FDD8
:10EC20000446404625F042F92046A5E7C4F0050019
:10EC3000A6E205007EE20500A2E2050078E20500FA
:10EC400041D8050085E20500BFE20500DBE20500D2
:10EC50002DE9F04F0022A5B03B4926F0ADFC05ACF4
:10EC600001460546204628F0D3FB284625F01EF92C
:10EC70001B235E1EA25D0AB11E4602E03346002E33
:10EC8000F7D124AB1E444FF001080CAF06F87C8C82
:10EC90000DF1240B03979BE807008DE8070094E82B
:10ECA0000F0028F02EF90546002847D00C9B23F0D2
:10ECB0007F4303444FF0000913F8013C0C9AFF2BEB
:10ECC00022F07F4A02D0B8F1FF0F1ED10024AAEB38
:10ECD0000406002E14DD412E28BF4026324661195D
:10ECE00014A82DF04FF814AA002312F8011BFF29D5
:10ECF00022D001339E42F8D100221C44002AE6D0E3
:10ED000004EB090025B0BDE8F08F08F1010806F812
:10ED10007C8C03979BE807008DE8070094E80F00C0
:10ED200028F0EFF8D144054658B10C9B23F07F43FF
:10ED3000034413F8013CC1E70122DEE781460446A3
:10ED4000DEE70446DCE700BF41D805002DE9F04FBF
:10ED50000C46A7B006466749204625F03DFB98B90A
:10ED60006549204625F038FB50BB6449204625F014
:10ED700033FB054638BB22466149012020F092F85A
:10ED8000284627B0BDE8F08F4FF0720A5D49002099
:10ED90001EF086F905460028F2D01C2200213046DC
:10EDA00025F029FC0DF11C0801460646404628F0D6
:10EDB0002FFB1B214B1E18F803203AB10B4608E02D
:10EDC0004FF0770AE2E74FF0610ADFE71946002BC0
:10EDD000F0D126AAD3184C4905933246284601247F
:10EDE0000EAE03F87C4C0DF12C0926F0B8FB03960F
:10EDF00099E807008DE8070098E80F0028F081F8EF
:10EE00000E9BBAF1770F074623F07F4B09D10028FC
:10EE10006ED02846FFF77EFC4FF0000B5F460026C1
:10EE200029E0BAF1610FFAD1002F61D007EB0B0393
:10EE300013F8013CFF2B01D0FF2C45D10026ABEB92
:10EE40000608B8F1000F16DDB8F1400FA8BF4FF06B
:10EE500040084246F11916A82CF094FF16AA002388
:10EE600012F8011BFF2941D001334345F8D100229C
:10EE70001E44002AE3D0204624F004FF2349024622
:10EE8000284626F06CFB304624F0FCFE2049024662
:10EE9000284626F064FB384624F0F4FE1D4902465D
:10EEA000284626F05CFB584624F0ECFE1A49024640
:10EEB000284626F054FB504624F0E4FE174902464B
:10EEC000284626F04CFB5BE7059B013403F87C4C9D
:10EED000039699E807008DE8070098E80F0028F0EE
:10EEE00010F80E9B074623F07F4B9DE70122BFE7FA
:10EEF0003E46C0E75F480600B1FE05002C10060044
:10EF00005CE205006CE2050041D8050078E20500EE
:10EF10007EE2050085E20500A2E20500C4F00500DE
:10EF200010B58CB005AC0146204628F071FA0CAB48
:10EF300013E907008DE8070094E80F0028F0D3F8E4
:10EF40000CB010BDF1F7A0BE27F058BF70B500227D
:10EF500090B006460846114608F0F0FF09AC054699
:10EF60003146204628F054FA0023CDE90533CDE997
:10EF7000035310AB13E907008DE8070094E80F0076
:10EF800028F0F2F80446284624F090FF204610B0FE
:10EF900070BD2DE9F041804690B008460C461746FA
:10EFA0001E4624F034F810B300221146204608F023
:10EFB000C5FF00260546374609AC4146204628F0E5
:10EFC00027FA0023CDE90353CDE9057610AB13E909
:10EFD00007008DE8070094E80F0028F0C5F8044604
:10EFE000284624F063FF204610B0BDE8F08120469B
:10EFF00023F088FD0546DFE730B58FB007AC01464A
:10F000000025204628F004FACDE903550EAB13E99C
:10F0100007008DE8070094E80F0027F0B9FF0446C9
:10F0200038B1294625F04BFC0546204624F03EFF2A
:10F030002C4620460FB030BD70B58EB007AC1646DA
:10F040000D460146204628F0E3F9CDE903560EAB04
:10F0500013E907008DE8070094E80F0027F098FFF8
:10F060000EB070BD70B58EB007AC0E46014620469E
:10F0700028F0CEF90023CDE903330EAB13E90700E6
:10F080008DE8070094E80F0027F082FF054668B17D
:10F0900005F042FA0446284624F008FF1EB11EF08F
:10F0A000BFFB24F003FF20460EB070BD0446FAE714
:10F0B0004FF4D82028F078B913B50C461BF0C4F8EB
:10F0C0008DF807000938042805D80DF10702034917
:10F0D000204623F0F1FB02B010BD00BFE1F00200BA
:10F0E0000B78C1B218461AF0EBBE00002DE9F043D0
:10F0F00089B0984605460E4617461BF0A5F8A0F1C4
:10F100000903DBB2042B04462ED80D280FD1274B60
:10F11000DB7863B94FF0FF324FF41651CDE904129A
:10F1200004A8234A06928DF81C30F6F75DFC8DF892
:10F130000040204C1FB1304626F018FF06466A46B4
:10F140002146304623F0B8FB17B1304624F0AEFE1E
:10F15000B8F1000F05D069460D20A04769460A2086
:10F16000A04709B0BDE8F0830028FAD10246124951
:10F17000284626F021FA224681461049284626F0E4
:10F180001BFA04AD02464946044628461AF0DCF84C
:10F19000204624F08BFE484624F088FE95E80F00B8
:10F1A0006C4607C42370064CC4E700BFD9D20020C8
:10F1B00008000100FDAE0400C1D90500EADD05002C
:10F1C00095A4040000231A46FFF790BF01231A46B6
:10F1D000FFF78CBF00230122FFF788BF2DE9FF470F
:10F1E00004461BF031F8002205464049204626F02F
:10F1F000E3F9002207463E49204626F0DDF9A5F155
:10F2000009068246002F4CD001463A4668461AF05D
:10F210009BF89DF80600FF2802D0002112F020FB89
:10F220009DF80700FF2802D0002112F019FB9DF87D
:10F230000400FF2802D0002112F012FB9DF8050007
:10F24000FF2802D0002112F00BFBF3B2042B28D9C7
:10F2500000222849204626F0AFF910B326F0F4FC2E
:10F260005FFA80F80021404611F0A8FE002019F056
:10F27000FFFF8146A8B1414624F0F7FE804618B151
:10F280000146484626F0EAFC484624F0F5FF20B93E
:10F29000194B1A49586826F091FD4946404625F019
:10F2A00078FE5146384625F074FE1149204626F076
:10F2B00085FDF6B20D49204626F080FD042E11D8BA
:10F2C0000D2D0AD10E4BDB780BB10CF0BFFEFF22E7
:10F2D000002128461BF05EF904E0A5F10C03DBB227
:10F2E000012BF4D904B0BDE8F08700BFEADD0500CA
:10F2F000C1D90500C9E10500482E0020CEE1050076
:10F30000D9D20020F0B585B005460F4614461AF054
:10F310009BFF064684B922465249284626F04CF9FE
:10F3200004462246394668461AF00EF858B9204677
:10F3300024F0BCFD05B0F0BDB4F80B3003F500734C
:10F34000A4F80B30EDE7009824F09CFC46490246F7
:10F35000284626F004F97CB122464249284626F088
:10F36000FEF8A6F10903DBB2042B0AD80D2EE1D179
:10F370006846F6F739FBDDE73A49284626F01EFDD8
:10F38000EFE7002ED6D19DF80500FF2807D0012118
:10F3900012F066FA01219DF805001BF00DFD9DF8A5
:10F3A0000400FF280BD0052112F05AFA602024F047
:10F3B00031FB044660B92D4901201FF073FD9DF813
:10F3C0000630FF2BB6D02A4901201FF06BFDB1E7B4
:10F3D00002462849284626F0C2F8204623F07EFE41
:10F3E000002680F84060044611F0EAFF009B9DF87B
:10F3F0000A2084F85860C4E914369DF80830134494
:10F400009DF80920B24218BF0133C4E9120184F803
:10F41000593001219DF8040011F0D0FD0446C8B117
:10F4200024F030FC14490246284626F098F80120C2
:10F4300019F01EFF06460028C1D02A46214625F0B5
:10F44000FEFF304624F032FD013C0C4B0C4A43F8E1
:10F450002420B4E79DF804200A4901201FF022FD72
:10F46000ADE700BFEADD0500C1D9050044E10500B4
:10F47000A1E105006AE10500C9E1050088D5002089
:10F480008D92040072E1050010B50C461AF0DCFE06
:10F49000A0F10903DBB2042B04D82146BDE81040DB
:10F4A0001BF01EBF02490120BDE810401FF0FABC4E
:10F4B00019E105002DE9F74F9846012313600D6906
:10F4C00007468A4616460DB10B68ED5C38782E2843
:10F4D00000F0FA805B2836D1012388F8093097F8CC
:10F4E00001B0BBF15E0F02D13368013333604FF0DE
:10F4F000000907E02E2C19D12E2D08BF49F0010973
:10F50000013333603368FC5CF818002C00F0DE80B7
:10F510005D2CEFD101333360002388F80930BBF153
:10F520005E0F14BF484689F0010019E0434601AA66
:10F530005146FFF7BFFF3368019A49EA00095FFAB5
:10F5400089F91344DDE75C286CD1022333607878B5
:10F55000642808D1A5F1300009288CBF00200120C3
:10F5600003B0BDE8F08F442806D1A5F1300009288A
:10F5700094BF00200120F3E766286ED062286ED089
:10F580006E286ED072286ED0732805D1284603B03D
:10F59000BDE8F04F1EF002BC532806D128461EF0ED
:10F5A000FDFB80F00100C0B2DAE774285DD0762858
:10F5B0005DD077280ED1A5F13003092B40F284806D
:10F5C00028461EF0DFFB00287ED15F2D14BF0020EF
:10F5D0000120C5E757280CD1A5F13003092B12D91A
:10F5E00028461EF0CFFB70B9B5F15F0018BF0120AF
:10F5F000B6E730283DD0A0F13103082B05D83649B5
:10F6000001201FF04FFC0020AAE778280AD1BB7820
:10F6100043B1FB7833B104233360F978B8781EF036
:10F62000A0FBC0B298F809302BB33368FA5C2D2ADE
:10F6300021D13B445B785D2B1DD0A8F80A003068CF
:10F6400001303060434601AA51463844FFF732FF8B
:10F650003368019A1344336082E70C20E2E7082004
:10F66000E0E70A20DEE70D20DCE70920DAE70B20DF
:10F67000D8E70020D6E798F8082062B1A5F1410349
:10F68000192B98BF2035A0F1410398BFEDB2192B7B
:10F690009CBF2030C0B2B8F90A30B3F5807F11D0DA
:10F6A000DBB22AB1A3F14102192A9CBF2033DBB29D
:10F6B0004FF480729D42A8F80A20A4D38542A2D8B4
:10F6C000984255E7854281E7012049E70120034937
:10F6D0001FF0E8FB204643E794E40500B1E4050091
:10F6E00082B02DE9F047ACB00C4634A9054681E85C
:10F6F0000C001EF0F9F830B1002630462CB0BDE801
:10F70000F04702B070472B780BB17C2B43D15822C5
:10F7100034A90DEB02002CF035FBDDE93457DDF8A0
:10F72000DC9024F097FA2368A2681A440646D21B9C
:10F730003946284624F05FFF002104460246304641
:10F7400025F07DFE204624F0B1FB0DF16808002471
:10F750004C450DDB384624F095FA70490246304698
:10F7600025F0FDFE2A466E49304625F0E1FEC4E74D
:10F7700058F8041BD8F820202846521A24F03BFFE2
:10F780000134824602462146304625F058FE504656
:10F7900024F08CFBDCE75E2B09D12368A268D342FE
:10F7A000AAD11FF041FD0028A6D0013507E0242B87
:10F7B0001DD1D4E900329A4205F101050CD850223E
:10F7C00036A968462CF0DEFA34AB0CCB214628462D
:10F7D000FFF786FF064690E74C2237A968462CF0D3
:10F7E000D1FA34AB0ECB284600F026FAF2E7282BEC
:10F7F0000FD1379B2168A26834A80A44191D082B31
:10F8000040F8212000EB83014A63CADC01333793BF
:10F81000C7E7292B0AD1379B002BC2DD34AA02EBA4
:10F8200083032168A2680A441A63BAE734AB15AAB5
:10F8300021462846FFF73EFE159FEB5DA3F12A0205
:10F84000012A804605EB07064ED801372F4450B9F0
:10F850002B2B08D14C2237A968462CF093FA34ABF5
:10F860000ECB3846C0E7214616A81EF0C6FE502231
:10F8700036A968462CF086FA34AB0CCB16A938466C
:10F88000FFF72EFF0646199824F010FBD4E9002359
:10F890009A42BFF432AFB8F1000F3FF42EAF2046CA
:10F8A0001EF025FC34AB15AA21462846FFF702FEC0
:10F8B0002146804616A81EF0A0FE502236A96846B2
:10F8C0002CF060FA34AB0CCB16A93846FFF708FFD2
:10F8D0008146199824F0EAFAB9F1000FD6D03046E3
:10F8E00024F0E4FA4E46D1E7D4E900239A420BD241
:10F8F00050B120461EF0FBFB1FF096FC00283FF4A1
:10F90000FBAE159B1D445AE74C2237A968462CF0E4
:10F9100039FA34AB0ECB304666E700BFD3E40500BE
:10F92000D9E405002DE9F047B4B00646084614AF07
:10F9300026F01CFB002254498046304625F03CFE50
:10F9400026F082F9002205465049304625F034FE63
:10F95000044623F07EFC48B92146404625F019FBB9
:10F96000002420468037BD46BDE8F087404624F09D
:10F970001CFFA842F0D3204624F017FF00F1080333
:10F9800023F00703ADEB030D0DF1500A421C514665
:10F99000204626F06BFC204624F088FA6921304688
:10F9A000FDF734FB4FF48072002387F830007A862D
:10F9B00041462A46384687F831307B63C7F82880AD
:10F9C0001EF0EFFE394607F114001EF016FE50221D
:10F9D00007F130016846FD622CF0D4F907F12809DF
:10F9E00099E80C0007F114015046FFF779FE044630
:10F9F000386A24F05BFA38461EF079FB2CB9D7E957
:10FA000000239A4205F1010514D3F86824F04EFA58
:10FA1000404624F04BFAD4B9022024F0A3F8002584
:10FA20000446284624F02EF917490246304625F0B0
:10FA300096FD96E7394607F114001EF0DEFD5022D0
:10FA400007F130016846FD622CF09CF9C8E7672198
:10FA50003046FDF7DBFAA0B10021204625F042FB3D
:10FA6000002280460A49204625F0A6FD26F0ECF843
:10FA70000546404624F099FE0544404624F016FA17
:10FA8000CFE70546CDE700BF09E1050002E105002B
:10FA9000D3E405002DE9F84F04460D4623F0D9FBC9
:10FAA00020B94FF000084046BDE8F88F24F0D2F8A6
:10FAB00080460028F5D01DB9214625F077FCF2E7F5
:10FAC0005149284625F096FD00285FD0002024F0FB
:10FAD000D9F84E490246284625F041FD21462846E0
:10FAE000FFF720FF0027064626B1304623F050FAE4
:10FAF0008146D0B1304624F0D9F9002024F0C2F874
:10FB000042490246284625F02AFD204624F04DFEB3
:10FB1000B842C8DB39466FF00042204624F06BFD46
:10FB20000146404625F05BFCBDE74946304625F0DE
:10FB3000D9FA4A4636498246304625F03DFD26F040
:10FB400083F88146504624F030FE8346504624F028
:10FB5000ADF9A9EB07023946204624F04CFD0146D9
:10FB6000404625F03CFC0BEB0907304624F09EF99B
:10FB7000384624F087F825490246284625F0EFFC50
:10FB800021462846FFF7CEFE0646ADE7284626F07A
:10FB9000EDF9814688B124F008FE0746204624F09E
:10FBA00004FE002600F1010BABEB070A3546554574
:10FBB00022DC7FB925BB0135F9E70746EEE75D4654
:10FBC00012E00146404625F0F1FB304624F06EF984
:10FBD000EE19F0E75545F2D001232A464946204662
:10FBE000F0F792FD0028E6D1AA1B3146204624F00A
:10FBF00002FD06460028E4D1484624F057F952E7B2
:10FC00005545F1D1F8E700BFFBE0050009E105002B
:10FC1000D3E4050038B5FFF785FE054650B123F063
:10FC2000B7F980F00100C4B2284624F03FF904F08F
:10FC3000010038BD0446F7E784B0F0B59BB021AEB3
:10FC4000054686E80E001FF0EFFA68B90446204624
:10FC50001BB0BDE8F04004B070475C2C03D16C7859
:10FC6000002CF4D03D4601352C78002CEFD07C2CB4
:10FC700005F10107F1D1DDE9211215A81EF091FD72
:10FC800023A9502268462CF07DF896E80C0015A9AF
:10FC90003846FFF725FD0446189824F007F9D6E703
:10FCA00037B5054601910B4848F2080123F0C8FF1B
:10FCB000044660B12A46084925F03AFC284601234B
:10FCC00001AA21461AF02CFA204624F0EFF803B0DE
:10FCD00030BD00BF87010300FED005002DE9F743CA
:10FCE000054608460F46904623F0ACF938B93A4627
:10FCF000254903201FF0D6F803B0BDE8F083B8F122
:10FD0000000F0BD000222149284625F0B7FB0446FE
:10FD1000E8B125F0DDF904461D4E01E01D4E4446D4
:10FD200000223146284625F047FC814688B93A46EC
:10FD30003146284625F0FCFBB8F1000FDCD0284600
:10FD40002146FFF7ADFF204624F0B0F8D4E7804607
:10FD5000E2E723F053F938B13946484625F026FB4F
:10FD6000484624F0A3F8E7E702216846CDE900976A
:10FD700025F052FB314607460246284625F0D8FBBF
:10FD8000384624F093F8EBE76AD905008ED90500D0
:10FD900060D9050065D9050010B500220446FFF7BB
:10FDA0009DFF2046BDE81040FDF766BA38B5154600
:10FDB00001220446FFF792FF25B100222946204682
:10FDC000FFF78CFF2046BDE83840FDF755BA00002C
:10FDD0002DE9F74F054623F069FA044640B92A4653
:10FDE000344903201FF05EF8204603B0BDE8F08FD1
:10FDF000314900201DF054F904460028F4D048F29F
:10FE000008012E4823F01CFF8146D8B122462C4918
:10FE100025F08EFB23F01EFF2946824601A81EF026
:10FE2000D3F800263546019880B9A81B23F02AFF95
:10FE300024490246204625F092FB5246224920469C
:10FE400025F08DFB484624F031F8CDE725F03CF94C
:10FE50008046FDF705F930B348F260011B4823F0F6
:10FE6000EFFE0746284623F00DFF00210246834699
:10FE7000384625F040FE584624F018F8224610492E
:10FE8000384625F055FB39464A464046FFF78EFF77
:10FE9000394625F07EF8404624F008F801A80135DF
:10FEA0001EF081F8BFE742462946504625F0C7FAC2
:10FEB0000136F0E77DDD0500C3E005006DFF0200BF
:10FEC000FED00500B8E00500BEE00500D1FE02004E
:10FED0002DE9F0410F46904613490022054625F0D2
:10FEE0006BFB25F0B1FE002204461049284625F0A0
:10FEF00063FB0646B0B142463946013C25F09FFA05
:10FF0000204623F0BFFE08490246284625F027FB7D
:10FF10001CB931462846FFF7C3FE3046BDE8F04124
:10FF200023F0C4BFBDE8F081B8E00500BEE00500E5
:10FF300037B5054601910B4848F2080123F080FED1
:10FF4000044660B12A46084925F0F2FA2846012302
:10FF500001AA21461AF0E4F8204623F0A7FF03B0D7
:10FF600030BD00BF81010300FED0050038B500227E
:10FF70000D460949044625F01FFB58B123F096FFB2
:10FF80002046054925F01AFF29462046BDE838409D
:10FF9000FFF7CEBF38BD00BFBEE005002DE9F0433E
:10FFA00085B0064601914149144625F007FF4049B6
:10FFB000304625F003FF00223E49304625F0FCFA8A
:10FFC0003C490546304625F0F9FE204623F016F858
:10FFD000074660B3214603A81DF0F6FF00240398EE
:10FFE00078B91DF01DFC804658B301462846FFF73E
:10FFF0009FFF2A462146404624F0BEFF05B0BDE8DB
:020000023000CC
:10000000F08325F061F801AB0122314681461BF0F7
:10001000D3FC804617B923F049FFA046484623F099
:1000200045FF03A81DF0BFFF00274446D7E7002C7B
:10003000D7D0204601AB012231461BF0BDFC04465F
:10004000CFE74DB32046FDF70BF850B348F2080157
:10005000194823F0F5FD48F208010646174823F039
:10006000EFFD0746A6B198B12A461549304625F05E
:100070005FFA2A461249384625F05AFA01223146DB
:100080002046FFF72BFE424639462046FFF726FE64
:100090003946304624F07DFF2946204624F079FF7A
:1000A000ACE721462846FFF7FBFDF5E760D90500E0
:1000B00065D90500E2150600A1FC020031FF02002F
:1000C000FED00500294B2DE9F047B2F10009284E7A
:1000D00008BF1E460D4600223146804625F06CFAC8
:1000E000044670BB02462349DFF888A0404625F04D
:1000F00063FA04464CB9B9F1000F25D12A461E49CE
:100100000120BDE8F0471EF0CDBE0022314620465A
:1001100025F052FA0746024648B129462046FFF725
:100120003DFF21463846BDE8F04724F032BF514636
:10013000204625F041FA0746204623F0B7FE3C460C
:10014000D8E7B9F1000F05D02A460C49404625F002
:10015000EFF94CB1404622462946FFF71FFF2046E3
:10016000BDE8F04723F0A2BEBDE8F08765D90500E1
:1001700060D90500E2150600A1D905008ED9050059
:100180000022FFF79FBF0122FFF79CBF2DE9F74F29
:1001900011F016F98946074623F0FEF9834611F05F
:1001A0000FF980468A4623F058FD0446002800F0E7
:1001B000A680564B56495868002225F0FDF90546A1
:1001C000002800F0A08024F033F80646284623F0EB
:1001D0006DFE002501230D214E485A1E01FB02022F
:1001E000B2F80B0080060FD010460193009222F067
:1001F0006BFF0135019B0D2130B1009A12680C3262
:10020000B2FBF1F213441544013340F60442934229
:10021000E2D9B018AB1B401B009323F033FD3E49DD
:100220000246204625F09BF9009B184623F02AFD44
:100230003A490246204625F092F940F6044023F060
:1002400021FD37490246204625F089F9304623F042
:1002500019FD2F490246204625F081F9584623F022
:1002600011FD30490246204625F079F9B8EB070028
:100270006AEB09012BF044F800222B4B2BF06EF8AF
:100280002A4B00222BF06AF841EC100B23F0E8FC1B
:1002900027490246204625F062F90D2023F0F2FCA2
:1002A00024490246204625F05AF9234823F0EAFC67
:1002B00022490246204625F052F9002023F0E2FCB4
:1002C0001F490246204625F04AF91E4823F0DAFC71
:1002D0001D490246204625F042F94FF4D82023F06C
:1002E000D1FC1A490246204625F039F94FF4002086
:1002F00023F0C8FC16490246204625F030F9204676
:1003000003B0BDE8F08F064663E700BF482E00202B
:1003100040E00500682E002048E005004DE00500A3
:1003200053E0050059E0050000408F400000B03E5A
:100330005CE0050063E00500B0E200206DE0050030
:100340007DE00500F450060089E005009AE0050014
:10035000ABE0050010B523F080FC0446294824F0EA
:100360000FFD29490246204625F0F9F8274824F0D8
:1003700007FD27490246204625F0F1F8254824F0DC
:10038000FFFC25490246204625F0E9F84FF40020FD
:1003900023F078FC21490246204625F0E0F84FF48E
:1003A000204023F06FFC1E490246204625F0D7F876
:1003B0004FF4803023F066FC1A490246204625F0AF
:1003C000CEF805F063FA18490246204625F0C7F832
:1003D00002F01EFE15490246204625F0C0F81448DA
:1003E00024F0CEFC13490246204625F0B8F8124806
:1003F00023F048FC11490246204625F0B0F820467B
:1004000010BD00BF9EDF0500A6DF0500AEDF0500C2
:10041000B7DF0500C2DF0500CADF0500D0DF050039
:10042000D6DF050004FB0500DEDF0500E5DF050083
:10043000EDDF050032E00500A82D00203AE00500C0
:1004400038B50849054600201CF02AFE044638B19C
:10045000284623F01FFC04490246204625F07FF879
:10046000204638BD5BDE050050DB05002DE9F84372
:100470000D460321074611F0F3F9002401264FF041
:100480008008A14615F1FF3502D22046BDE8F88369
:1004900088F311880021384610F078FF0320F1F727
:1004A00083FB0121384610F071FF0A20F1F77CFB35
:1004B000384610F057FF00B1344389F311883520D6
:1004C000F1F772FB7600DDE710B50321044611F069
:1004D000C7F90021204610F059FF4FF4FA70F1F7E8
:1004E00063FB0121204610F051FF5020F1F75CFB27
:1004F000204610F037FF04464FF4D270F1F754FB5A
:1005000084F00100C0B210BD08B50022034925F0F7
:1005100053F8BDE8084019F08BBF00BF50DB050061
:100520002DE9F04F8BB00C46FFF7EEFF064619F0B1
:10053000A1FF28B94FF0000840460BB0BDE8F08F8E
:1005400023F088FB80460028F4D0631EFF2B28BFD1
:10055000F0242246E317CDE900234FF0000930468E
:10056000FFF7B2FF0028E7D0DDE90023082130467D
:10057000FDF74CFD01240025AA46274601213046FF
:10058000FFF774FF01215FFA80FB3046FFF76EFF33
:10059000BBF1010FC0B22BD101283AD1402FCBDDE6
:1005A0009DF80C30002BC7D005AC0DF10C090025CF
:1005B000A34619F8017B38091DF0A8F9207007F04F
:1005C0000F001DF0A3F90135082D607004F102043D
:1005D000EFD1002358468DF8243024F0D1FB01469A
:1005E000404624F0FCFED146BAF1000FA4D0B6E795
:1005F0000AAB2B44834513F81C3C2DD14F4524DA1C
:100600001C4214BF4FF0010B4FF0000BBBF1000F69
:1006100021D00AAB2B444FF0010B13F81C3C2343B1
:100620000AAA2A44012102F81C3C30465A460023FB
:100630006400FDF7EBFC14F0FF0404BF0135012456
:10064000072D07F1010799DDA8E70CBF4FF0010B5B
:100650004FF0000BDAE7BA4623EA0403E0E770B58F
:100660008AB00C46FFF750FF064619F003FF68B347
:10067000204622F00DFD18B3204624F043FD01462C
:100680000546012023F038FC044650B10146002203
:1006900068461EF003FE15F1FF3505D268461DF0D1
:1006A00019FC20460AB070BD08213046FFF7DEFE77
:1006B000C1B268461DF0D9FE68461DF03EFDEAE76E
:1006C00008213046FFF7D2FE23F0DCFA0446E8E7C3
:1006D00037B50D461446FFF717FF8DF8070019F0E0
:1006E000C9FE80B10DF107020C49284622F0E4F85A
:1006F0009DF807004CB1012110F048FE01219DF842
:10070000070011F0ADF803B030BD042111F0A8F8D6
:1007100001219DF8070010F039FEF4E79BE002008C
:1007200010B5FFF7F1FE044619F0A4FE38B12046DB
:10073000CC2200230821BDE81040FDF767BC10BDA6
:100740002DE9F04186B00C46FFF7DEFE054619F0B4
:1007500091FE40B1204622F07CFD38B92246264960
:1007600003201EF09FFB06B0BDE8F081204624F078
:100770001CF81028F2D12846FFF7A6FE21460022D9
:1007800001A81EF00EF8002427462646A04601A820
:100790001DF000FF8DF8000001A81DF0FBFE0023F6
:1007A0001A468DF80100102168468DF802801DF070
:1007B00000FBA4F12002C4F12003A14000FA02F2E0
:1007C00020FA03F31143A04008341943402C47EAB0
:1007D000000746EA0106DAD1049823F067FB2846B1
:1007E000552200230821FDF711FC3A4633462146E5
:1007F0002846FDF70BFCB6E763DE050010B5FFF7F2
:1008000083FE044619F036FE20B12046BDE81040B4
:10081000FFF75ABE10BD00002DE9F74F21F000454B
:10082000894616461F464FF0FF32414B2946804607
:1008300004462BF02DF8002876D14FF0FF323C4BC8
:10084000404629462BF01AF800286DD132463B4627
:10085000304639462BF01CF8002865D100220023D1
:10086000404649462AF0ECFF28B309F10045002232
:100870000023304639462AF0E3FF10B107F1004368
:100880001F4600220023304639462AF0CFFF78B9B0
:100890004FF0FF32264B304639462AF0DBFF38B1A5
:1008A0004FF0FF32224B204629462AF0D3FFE8B909
:1008B0000024002522E04D46D9E700221D4B2046AA
:1008C00029462AF04BFDCDE90001B246BB4652460F
:1008D0005B46DDE900012AF0C7FF52465B46E0B9FE
:1008E000204629462AF082FB04460D4622462B4626
:1008F000304639462AF0AEFF0028DED10022002320
:10090000404649462AF09CFF10B105F100431D46C0
:100910002046294603B0BDE8F08F104619462AF05C
:1009200067FB82468B46D2E70024034DF0E700BF09
:10093000FFFFEF7F0000E03F0000F87F2DE9F84364
:1009400055EC114B11EE100A294657EC106B2AF0AA
:10095000B5FF0928804619D82AF096FC22462B4676
:100960002AF064FF90B1B8F1000F63D030463946E9
:10097000B8F1010F03D141EC100BBDE8F88332460A
:100980003B462AF0EBFC08F1FF38F1E70022002398
:10099000304639462AF054FF0022D8B3284B20466F
:1009A0002946FFF739FF002200232AF03FFFF0B36A
:1009B00000224FF0804320462946FFF72DFF0022FA
:1009C00000232AF033FFB04607F1004949EC108BB1
:1009D00068B128F011FD22462B4651EC100B2AF08D
:1009E000BDFCBDE8F84341EC100B28F081BC28F0B9
:1009F00003FD22462B4651EC100B2AF0AFFC41ECD4
:100A0000100B28F075FC53EC102B10EE100A03F1BC
:100A10000041B0E70023304639462AF007FF30B1E5
:100A200000220023204629462AF014FF28B147EC73
:100A3000106BCEE7002002499DE7002000219AE7D5
:100A40000000F03F37B50D46014668461446FCF7F6
:100A5000F7FD98B1019890F82532013B022B0DD893
:100A600074B18168294413F0C5FF014630B10548CF
:100A7000054B002C08BF1846FCF7B2F903B030BD97
:100A80002146EFE798DB0500A7DB050070B50E4EA9
:100A900034783CB913F06EFA054628B90B490120A9
:100AA0001EF000FA204670BD09490A48012213F0E1
:100AB00009FE014618B10848FCF792F9F2E7012354
:100AC00033702C46EEE700BF4ED300200BDA050052
:100AD0004118060054D300203CDA05002DE9F04708
:100AE00090B004468846FFF7D1FF002865D0214624
:100AF00001A8FCF7A5FD00285FD0029B93F82522F2
:100B000002F0FD02012A58D100220092DD689B68A4
:100B1000ED1A52D028EAE878454528BF45462846D0
:100B200022F078FF0446C0B1029E22F0D7FA6B464D
:100B300001462A46304614F098FA014610B1224880
:100B4000FCF74EF9204610B0BDE8F0871AF8071000
:100B500003A81DF045FA013722E005468146A84565
:100B600025D9A8EB0506202E28BF20260DF1200A46
:100B70006B46324651460298CDF8009014F075FA53
:100B80000746E0B9009B73B14CB91B2022F0EAFF85
:100B9000044690B101463A4603A81DF002FE002724
:100BA000009BBB42D2D8009BB3421D44D7D0002C3F
:100BB000C8D0069823F07AF9C4E70024C2E70146BA
:100BC0000148FCF70DF9F2E784DB05002DE9F04F51
:100BD0009BB005460C46FFF759FF002800F00B813B
:100BE000294605A8FCF72CFD28B94FF0000B584604
:100BF0001BB0BDE8F08F069B93F82532023B012B1A
:100C0000F3D8012221460FA81EF077FB4FF0000B0E
:100C10000FA81DF091F908B9054659E007AC002767
:100C2000A2460FA81DF06DFB04F8010B0FA81DF0E4
:100C30009EFA0FA801371DF07FF908B1202FF0D1DF
:100C4000069C204613F0F4F90546002840F0CB80BE
:100C5000E379002B40F0C680A3799E0740F1C6805F
:100C6000A368FB42814604D204F124030393A368E2
:100C70004FB9D4E90232934288BFE360A37943F0CD
:100C80002003A3711DE0C3F30802002A40F09780FF
:100C9000206890F8028008F1FF3808EA532818F01D
:100CA000FF02029230D123BB216921B913F052FE19
:100CB00001460028DDD001291DD14FF00203E37168
:100CC0000225CB44B9F1000F00F09380002D9FD096
:100CD0000FA81DF005F9494B1B781B0702D4069895
:100CE00014F0CFFB002D82D029464548FCF778F858
:100CF0007DE76169DAE7481C02D10125E571E0E78B
:100D00002369616103B92161A3795A060CD5206872
:100D1000A26903994078012313F09CF80028ECD1D4
:100D2000A37923F04003A3712368616901931846F6
:100D300013F019FA0028C0D0029BB7F5007F00EB32
:100D400003082AD3019B029A9B7801987E0A3244B9
:100D50009A4288BF029A407888BF9E1A334642461C
:100D6000514613F077F80028C7D1A169A1EB08011B
:100D70008E420AD94FF400720AEB4121039814F015
:100D80006AF9A37923F04003A3717602A368334480
:100D9000B244A360B144BF1B69E7A36998450CD076
:100DA000D4E902329A4208D9019803994078012384
:100DB000424613F09FF800289FD1C4F81880A0681D
:100DC000C0F30800C0F50076BE4228BF3E4624307E
:100DD00032465146204414F03EF9A37943F04003D3
:100DE000A371D3E71D464FF000096AE78146072546
:100DF00067E701256CE78346F9E600BF50D3002082
:100E0000B6DB050037B50446FFF740FE70B3214658
:100E10006846FCF715FC48B3019C94F82632012B78
:100E200024D1204614F02DFB20B9204613F000F900
:100E300000B92060019B0E49022283F826220D4B47
:100E40000022586824F0B8FB054678B101220099C9
:100E500026F0D0FF044630B10146284624F0FEFEBD
:100E6000204623F023F8284623F020F803B030BDB5
:100E70007DDB0500482E002037B5174B1749586811
:100E8000002224F099FB044658B1014601A81DF048
:100E90009BF80198A0B9204624F0ABFF204623F030
:100EA00005F80F4B1A782AB10022114610461A7025
:100EB00013F008FCFF21002013F06CF803B030BDE4
:100EC00024F002F90546FFF79DFF284622F0EEFFC9
:100ED00001A81DF068F8DCE7482E00207DDB050046
